:100000000C94A40D0C94C10D0C94C10D0C94C10D55
:100010000C94C10D0C94C60F0C94EB110C94C10DF3
:100020000C94C10D0C94C10D0C94C10D0C94C10D18
:100030000C94C10D0C94C10D0C9473230C94C10D40
:100040000C940D150C94FC120C94D60F0C948D0F7F
:100050000C94C10D0C94881E0C94C10D0C94C10D10
:100060000C94C10D0C94C10D0C94C10D0C94C10DD8
:100070000C94C10D0C941B240C94FF110C94AD1125
:100080000C94C10D0C94755A0C94C10DBB5487553A
:10009000F653C4549B5528543E54E955E955E95547
:1000A0005C54E955E955E955E955D8546755675504
:1000B00083551C551C551A5518551655E955E955C3
:1000C000E955E955E955E955E955AB54E955E9557F
:1000D000E955E955E955E955E955E955E955E95530
:1000E000E955E955E955E955E955E955E955E95520
:1000F000E955E955E955E955E955E955E955E95510
:10010000E955E955E955E955E955DA55CC55BA555A
:100110009F5545617379436F6E74726F6C00204D0B
:100120004300696E636F6D70617469626C6520482D
:100130005700312E342E31005F03AF01D7006B0022
:10014000470035001A0011000102031304050611CF
:10015000070809120A000B0C100F0E0D0101010512
:100160000D1F0C04040E1F04041F0E041F1F1F008C
:100170001F1F1F001F1F1F001F111F001F111F0027
:100180001F1F1F001F111F001F111F00000609174E
:1001900017090600000609121412090603070F1EAC
:1001A0001C18100003050912141810000707070790
:1001B0000707070707050505050505071C1018179C
:1001C000150705071C101817110202021C1018123F
:1001D000140605021C101817140601061C10181529
:1001E000150701011C101816110201061C10181623
:1001F000110204071C10181216020207040A110A41
:100200000A0E00000C17141714170C001C101810FD
:10021000160505051F0A0A0A0A0A1F000E11111FFA
:100220001B1B1F0002060F1F0F060200080C1E1FDB
:100230001E0C08000E0E0E0E1F0E0400040E1F0EE4
:100240000E0E0E0000C030F00CCC3CFC03C333F3A8
:100250000FCF3FFFC303F333CF0FFF3FAAC0803060
:10026000F0B020E0A00CCC8C3CFCBC2CECAC08C862
:100270008838F8B828E8A803C38333F3B323E3A38B
:100280000FCF8F3FFFBF2FEFAF0BCB8B3BFBBB2BBA
:10029000EBAB02C28232F2B222E2A20ECE8E3EFE60
:1002A000BE2EEEAE0ACA8A3AFABA2AEA004060972F
:1002B0007048685878446454744C6C5C7C42625258
:1002C000724A6A5A7A466656764E6E5E7E41615131
:1002D000714969597945659F754D6D5D7D436353DE
:1002E000734B6B5B7B476757774F6F5F7F101814BB
:1002F0001C121A161E1119151D131B171FD0D8D446
:10030000DCD2DAD6DED1D9D5DDD3DBD7DF90989435
:100310009C929A969E9199959D939B5055040605A3
:1003200007C4C6C5C78486858734363537F4F6F5E5
:10033000F7B4B6B5B724262527E4E6E5E7A4A6A5D5
:10034000A701C18131F1B121E1A10DCD8D3DFDBDEF
:100350002DEDAD09C98939F9B929E9A92020202055
:1003600020200000204D4D4920200000204D4D014F
:100370002020000020444343202000002053544FFD
:100380005020000053484F52542100002048414C57
:100390005420000000000000000000002050524FD8
:1003A0004720000052455345542000007E0E0E0E9B
:1003B0000E1B1B1C0E1B1B7E0E0E0E0E232D004152
:1003C00044523A20256C6420202020202020202028
:1003D00020002D2D2D2D202000252D3564002533C6
:1003E0006400202001022020202020202000252D34
:1003F000356400252D31312E313173000002070B99
:100400001014191D22262B3035393F43484C5156C4
:100410005B5F64696D72767B7F0002070C10151AB2
:100420001E23282C31363A3F44484D52565B6064B7
:10043000696E73797F00020C151D263039434C56C6
:100440005F69727F2530386C75005741524E494EB6
:10045000473A20004552524F523A200062616420D0
:10046000706172616D657465722076616C7565008E
:10047000706F776572206973204F666600747572BD
:100480006E6F75742071756575652066756C6C008E
:10049000636F6D6D616E642071756575652066753D
:1004A0006C6C006E6F2064617461006E6F20736C01
:1004B0006F7420617661696C61626C65006C6F6B52
:1004C000206275737900696C6C6567616C20747566
:1004D000726E6F757420616472657373004D432092
:1004E000696E2048414C54004D4320696E2053549E
:1004F0004F50004C207B4C6F6B232C205B5370655E
:1005000065645D2C205B464C5D2C205B4469725D0C
:100510002C205B46315D2C205B46325D2C205B46F7
:10052000335D2C205B46345D7D0054207B54726E1D
:1005300074232C205B436F6C6F725D2C205B5374B3
:10054000617475735D7D0046207B4C6F6B232C209E
:100550005B46315D2C205B46325D2C205B46335D73
:100560002C205B46345D2C205B46355D2C205B46A1
:10057000365D2C205B46375D2C205B46385D7D0068
:10058000484C2048656C7020666F72206C6F6B2041
:10059000636F6D6D616E64730D0048462048656C35
:1005A0007020666F722066756E6374696F6E20636B
:1005B0006F6D6D616E64730D0048542048656C70FA
:1005C00020666F72207475726E6F757420636F6D24
:1005D0006D616E647300507772206F6666004861CB
:1005E0006C7465642100507772206F6E0044434341
:1005F0002070726F6772616D005245534554004818
:10060000616C746564210D5D004C20257520257595
:100610002025632025632025632025632025632072
:10062000256300756E75736564004D6F746F726F2E
:100630006C61204F6C64004D6F746F726F6C612041
:100640004E657700444343004620257520256320EE
:10065000256320256320256320256320256320252D
:1006600063202563004658202575202563202563D7
:100670002025632025632025632025630054202541
:1006800064202563202564004D43205265766973FC
:10069000696F6E2000312E342E31000D5365724E7D
:1006A000722E2025386C75004D5420256420256459
:1006B000005352202564004D6F64756C652023251E
:1006C000642028696E70757420312E2E3820262003
:1006D000392E2E313629203D200053452025640037
:1006E0003537363030002575000D5D002564005A21
:1006F0007A4100556E6B6E6F776E20636F6D6D6122
:100700006E64000D5D003132000032340000343878
:1007100000003936000031343400313932003338CA
:100720003400353736004142434445464748494A3C
:100730004B4C4D4E4F505152535455565758595A91
:10074000303132333435363738392E2C3A2D2B238D
:100750002F3D3C7C3E20004D4D204920203134204F
:10076000004D4D20492020323761004D4D20492059
:1007700020323762004D4D20012020313420004DC1
:100780004D20012020323761004D4D2001202032C4
:100790003762004443432020203134200044434347
:1007A000202020323820004443432020313238209A
:1007B000004C6F636D656E75000000000000000066
:1007C000004443432D70726F6772616D6D2E00009F
:1007D000004D6F64656C6261616E7369742E000018
:1007E00000496E7374656C6C696E67656E0000001D
:1007F00000536F667477617265205570646174652B
:10080000004C4344207665726C69636874696E6756
:10081000004D6173746572436F6E74726F6C00008B
:10082000004578697400000000000000000000002E
:10083000004B69657A656E20000000000000000032
:100840000044617461666F726D61740000000000A5
:10085000004E61616D20202020202000000000005B
:1008600000496E766F657220202020000000000095
:1008700000435620286279746529000000000000BA
:10088000004356202862697429000000000000001F
:100890000042617369736164726573000000000057
:1008A000004C616E67206164726573000000000097
:1008B00000526567697374657200000000000000F3
:1008C00000506167652D4D6F6465000000000000F9
:1008D00000486F6F666473706F6F720000000000F5
:1008E000007338382D696E7374656C6C696E67655A
:1008F0006E436F6E666967757261746965000000AA
:1009000000426F6F73746572000000000000000009
:1009100000496E74657266616365204261756400AA
:100920000057697373656C00000000000000000050
:10093000004C6F63666F726D617400000000000010
:10094000004D4D207369676E61616C7061757A65E9
:10095000007338382D6D6F64756C65000000000001
:10096000007338382D6D6F64756C65746573740031
:10097000004B6F7274736C2E20706F6C2E00000031
:10098000004B6F7274736C2E206765762E0000002A
:100990000057697373656C666F726D617400000057
:1009A000004D696E2E736368616B656C74696A646F
:1009B000004D61782E736368616B656C74696A645D
:1009C000004D656E75204C6F636F000000000000E5
:1009D0000050726F6772616D2E2044434300000027
:1009E0000045746174205265736561752E000000C6
:1009F000005265676C6167657300000000000000CD
:100A0000004D414A206C6F67696369656C000000A6
:100A1000004C756D696E6F736974650000000000AD
:100A2000004D6173746572436F6E74726F6C000079
:100A3000004578697400000000000000000000001C
:100A40000053656C656374696F6E200000000000E0
:100A500000466F726D617420646F6E6E6565730021
:100A6000004E6F6D2020202020202000000000007C
:100A70000053616973696520202020000000000098
:100A800000435620286279746529000000000000A8
:100A9000004356202862697429000000000000000D
:100AA00000416472657373652064652062617365DB
:100AB0000041647265737365206C6F6E67756500C5
:100AC00000526567697374657200000000000000E1
:100AD00000506167652D4D6F6465000000000000E7
:100AE00000566F6965207072696E636970616C652C
:100AF000005265676C61676520733838000000003C
:100B000000436F6E66696775726174696F6E00008D
:100B100000426F6F737465720000000000000000F7
:100B200000496E7465726661636520426175640098
:100B300000436F6E662E2041696775696C6C612E8B
:100B400000466F726D6174206C6F636F000000006F
:100B5000005061757365207369676E616C204D4D3F
:100B6000004D6F64756C65732073383800000000A9
:100B70000054657374206D6F64756C65207338382C
:100B800000506F6C2E6372742D63697263756974A3
:100B90000053656E732E206372742D6369726374E3
:100BA00000466F726D61742061696775696C6C2EA7
:100BB00000547073206D696E2E696D70756C732EA4
:100BC00000547073206D61782E696D70756C732E92
:100BD000004C6F6B204D656EFC00000000000000B3
:100BE000004443432D50726F6772616D6D672E0034
:100BF00000416E6C6167656E7A757374616E640036
:100C00000045696E7374656C6C756E67656E000087
:100C100000536F6674776172652055706461746506
:100C2000004C43442042656C6575636874756E675B
:100C3000004D6173746572436F6E74726F6C000067
:100C4000004578697400000000000000000000000A
:100C50000041757377E4686C656E20000000000049
:100C600000446174656E666F726D6174000000000F
:100C7000004E616D65202020202020000000000033
:100C80000045696E7472616720202000000000003A
:100C90000043562028627974652900000000000096
:100CA00000435620286269742900000000000000FB
:100CB0000042617369732D4164726573736500004E
:100CC000006C616E67652041647265737365000036
:100CD00000526567697374657200000000000000CF
:100CE00000506167652D4D6F6465000000000000D5
:100CF000004861757074676C6569730000000000DE
:100D0000007338382D45696E7374656C6C756E6749
:100D1000004B6F6E66696775726174696F6E000073
:100D200000426F6F737465720000000000000000E5
:100D300000496E7465726661636520426175640086
:100D4000005765696368656E0000000000000000E0
:100D5000004C6F6B666F726D6174000000000000E4
:100D6000004D4D2D5369676E616C20506175736540
:100D7000007338382D4D6F64756C650000000000FD
:100D8000007338382D4D6F64756C74657374000092
:100D9000004B75727A7363686C2E2D506F6C2E0049
:100DA000004B75727A7363686C2E2D456D70662EDC
:100DB000005765696368656E666F726D61740000E7
:100DC000006D696E2E20536368616C747A65697476
:100DD000006D61782E20536368616C747A65697464
:100DE000004C6F636F6D6F74697665206D656E750D
:100DF000004443432070726F6772616D6D696E6766
:100E0000004C61796F7574207374617475730000A0
:100E10000053657474696E67730000000000000081
:100E200000536F66747761726520557064617465F4
:100E3000004C4344206261636B6C69676874000016
:100E4000004D6173746572436F6E74726F6C000055
:100E500000457869740000000000000000000000F8
:100E60000053656C65637420000000000000000002
:100E7000004461746120666F726D6174000000004F
:100E8000004E616D65202020202020000000000021
:100E900000456E74727920202020200000000000A0
:100EA0000043562028627974652900000000000084
:100EB00000435620286269742900000000000000E9
:100EC000005072696D617279206164647265737338
:100ED00000457874656E642E206164647265737376
:100EE00000526567697374657200000000000000BD
:100EF00000506167652D4D6F6465000000000000C3
:100F0000004D61696E20747261636B000000000027
:100F1000007338382073657474696E67730000005D
:100F20000044656C6574650000000000000000006E
:100F300000426F6F737465720000000000000000D3
:100F400000496E7465726661636520426175640074
:100F500000506F696E747300000000000000000014
:100F6000004C6F632E20666F726D6174000000008C
:100F7000004D4D207369676E616C207061757365FB
:100F800000733838206D6F64756C65730000000065
:100F900000733838206D6F64756C652074657374E8
:100FA0000053686F727420632E20706F6C2E0000E7
:100FB0000053686F727420632E2073656E732E0069
:100FC00000506F696E747320666F726D61740000FB
:100FD000006D696E2E7377697463682E74696D6530
:100FE000006D61782E7377697463682E74696D651E
:100FF00000202D2D2D2D0025357500536F6674773B
:101000002E205600312E342E31005365724E722E32
:101010002025386C75003A2000253575002533648D
:10102000002534643A20002D2D2D00253364002046
:101030004F4B202020200020202020202020004373
:10104000563A20202020204269743A203D20004357
:10105000563A253464204269743A25643D00202DB7
:101060002D2D0025346400202D2D2D2D2D0025360D
:1010700064002533642C256473002534646D73008B
:101080003030204261756400446F776E6C6F61642C
:10109000202E2E2E002564206D7300202532640042
:1010A0004E723A2025326420200073686F727420DB
:1010B00028312E356D73292000006C6F6E67202853
:1010C000342E3032356D732900004D6F746F726F9E
:1010D0006C61000000000000000044434320202019
:1010E00020200000000000000000706F7369746928
:1010F000766520284D4D290000006E656761746992
:1011000076652028444343290000536176652020FA
:1011100020202020202020202000526573746F7230
:10112000652020202020202020005361766520208B
:1011300020202020202020202000526573746F7210
:1011400065202020202020202000206C61796F75F0
:1011500074207374617475732000206C61796F75ED
:10116000742073746174757320004B6F7272202841
:10117000312E356D7329202000004C616E672028C8
:10118000342E3032356D732900004D6F746F726FDD
:101190006C61000000000000000044434320202058
:1011A00020200000000000000000506F7369746987
:1011B000656620284D4D290000004E656761746901
:1011C000656620284443432900004D6F64656C62C6
:1011D00061616E7369742E2020004D6F64656C62CE
:1011E00061616E7369742E202000486572737465A6
:1011F0006C6C656E2020202020004F70736C616144
:101200006E2020202020202020002068657273742A
:10121000656C6C656E2020202000206F70736C61FF
:10122000616E2020202020202000436F75727420E2
:1012300028312E356D73292000004C6F6E672028F1
:10124000342E3032356D732900004D6F746F726F1C
:101250006C61000000000000000044434320202097
:1012600020200000000000000000706F73697469A6
:10127000766520284D4D290000006E656761746910
:1012800076652028444343290000456E72656769EE
:10129000737472656D656E74200052657374617548
:1012A000726174696F6E20202000456E72656769F7
:1012B000737472656D656E74200052657374617528
:1012C000726174696F6E2020200020457461742063
:1012D0005265736561752E2020002045746174206D
:1012E0005265736561752E2020004B75727A202837
:1012F000312E356D7329202000004C616E67202847
:10130000342E3032356D732900004D6F746F726F5B
:101310006C610000000000000000444343202020D6
:1013200020200000000000000000706F73697469E5
:101330007620284D4D29000000006E6567617469B4
:1013400076202844434329000000416E6C616765A4
:101350006E7A757374616E642000416E6C616765AE
:101360006E7A757374616E64200057696564657286
:101370006865727374656C6C6E0053706569636840
:1013800065726E202020202020002077696564652A
:101390007268657273742E20200020737065696313
:1013A0006865726E202020202000696E636F6D706A
:1013B00061742E20466F726D617400496E636F6DAB
:1013C000702E20466F726D6174202000466F726D22
:1013D000617420696E636F6D7061742E00696E6B4D
:1013E0006F6D7061742E20466F726D6174002E2EC9
:1013F0002E2077616974696E67202E2E2E200023BF
:101400003D64656C6574650000000000000000002C
:10141000286E6F20656E747279290000000000004C
:10142000002E2E2E2064656C6574696E67202E2E4A
:101430002E00206661756C74000000000000000042
:1014400000000020444343206F6E6C7921000000AF
:10145000000000002A3D43616E63656C202020007F
:1014600000000000002070726F6772616D696E6726
:101470000000000000002D73686F727420636972B1
:10148000637569742D20002A726561642000000074
:1014900000000000000000002A77726974650000F7
:1014A0000000000000000000002E2E2E2077726940
:1014B00074696E67202E2E2E20002E2E2E2072652F
:1014C0006164696E67202E2E2E2000212121206666
:1014D00061756C742021212120202000204F4B2099
:1014E000202020202020202020202020002E2E2EF2
:1014F00020736176696E67202E2E2E2020002E2EFE
:1015000020726573746F72696E67202E2E2000231F
:101510003D44656C2E202A3D43616E63656C20005E
:10152000233D596573202A3D43616E63656C20201D
:101530000020636F6E66696775726174696F6E20F3
:1015400020004F46460000000000000000000000A0
:101550000000002A2A2A206E6F20547261696E20D2
:101560002A2A2A002A2073686F72742063697263C2
:1015700075697420002A2A2A2074696D65206F75A8
:1015800074202A2A2A00506F696E74202025346442
:101590002F253464000000436F6E666967757261C1
:1015A00074696F6E2020200020636F6E6669677516
:1015B000726174696F6E2020002E2E2E2077616379
:1015C0006874656E202E2E2E2000233D776973737C
:1015D000656E000000000000000000286765656E71
:1015E00020696E766F65722900000000202E2E2E75
:1015F0002077697373656E202E2E2E000020666F93
:101600007574000000000000000000000000204190
:101610006C6C65656E204443432100000000002A85
:101620003D2041666272656B656E0000000000003F
:101630002050726F6772616D6D6572656E0000009B
:10164000002D2D4B6F7274736C756974696E672D04
:101650002D002A4C657A656E000000000000000035
:101660000000002A53636872690000000000000057
:10167000000000002E2E2073636872696A76656E22
:10168000202E2E00002E2E2E206C657A656E202EC8
:101690002E2E202000002021212120466F7574204D
:1016A00021212120200000204F4B2020202020201D
:1016B00020202020202000002E2E2E204F70736C22
:1016C00061616E202E2E2E00004865727374656C69
:1016D0006C656E20202020200000233D7769737305
:1016E000656E202A3D616662720000233D4A6120DA
:1016F0002A3D41666272656B656E200020776973D2
:1017000073656E2020202020202020200055495481
:1017100000000000000000000000000000002A2A75
:101720002A206765656E204C6F63202A2A2A002ACA
:101730002A6B6F7274736C756974696E672A2A00FC
:101740002A2054696A646F766572736368722E2A00
:101750000057697373656C732534642F25346400F6
:101760000000436F6E666967202020202020202023
:1017700020200020436F6E666967202020202020F3
:101780002020200050617469656E74657A00000045
:101790000000000000233D7375707072696D657202
:1017A0000000000000007669646500000000000091
:1017B000000000000000005375707072657373695B
:1017C0006F6E0000000000002045727265757200A7
:1017D0000000000000000000002044434320756E1C
:1017E000697175656D656E7400002A3D4162616EB8
:1017F000646F6E20200000000000002050726F67B0
:1018000072616D6D6174696F6E0000002D436F75BC
:1018100072742D636972637569742D20002A4C659A
:1018200063742E00000000000000000000002A4544
:101830006372697400000000000000000000002EC8
:101840002E2E204563726974757265202E2E2E002F
:101850002E2E2E204C656374757265202E2E2E2040
:1018600000212121204572726575722021212120DD
:101870002000204F4B20202020202020202020202E
:1018800020200020456E72656769737472656D650E
:101890006E74200020526573746175726174696F93
:1018A0006E20202000233D5375707072202A3D4128
:1018B00062616E642E00233D4F7569202A3D4162AE
:1018C000616E646F6E2000205375707072696D6573
:1018D0007220202020202000496E616374696620F8
:1018E0002020202020202020002A20506173206406
:1018F00065206C6F636F202A20002A20436F757269
:10190000742D6369726375697420002A2054656DB3
:101910007073206465706173736520004169677539
:10192000696C2E2534642F253464000000456E72E6
:10193000656769737472656D656E74202000526509
:1019400073746175726174696F6E20202020002E9F
:101950002E2E2077617274656E202E2E2E20200090
:10196000233D4CF6736368656E00000000000000C4
:1019700000286B65696E2045696E74726167290085
:101980000000202E2E2E206CF673636865202E2E0C
:101990002E2000204665686C657200000000000083
:1019A00000000000206E75722066FC7220444343E4
:1019B00021000000002A203D2041626272756368A8
:1019C0000000000000002050726F6772616D6D6949
:1019D0006572756E6700002D2D204B75727A7363EA
:1019E000686C75DF202D2D002A6C6573656E000014
:1019F0000000000000000000002A736368722E00DF
:101A0000000000000000000000002E2E207363681C
:101A100072656962656E202E2E00002E2E2E206CBF
:101A20006573656E202E2E2E20200000212121209E
:101A30004665686C657220212121200000204F4BF3
:101A400020202020202020202020202000002E2EBA
:101A50002073706569636865726E202E2E000077B2
:101A600069656465726865727374656C6C656E0037
:101A7000233D4CF6736368656E202A3D41626272B5
:101A800000233D4A61202A3D41626272756368000D
:101A90000000206CF6736368656E202020202020F3
:101AA000202000415553000000000000000000000D
:101AB000000000002A2A206B65696E65204C6F6B60
:101AC000202A2A20002A2A204B75727A7363686CB8
:101AD00075DF202A2A002A205A656974FC62657223
:101AE000736368722E2A0057656963686520253420
:101AF000642F2534640000004B6F6E666967757251
:101B00006174696F6E20202000204B6F6E666967DC
:101B100075726174696F6E2020005B6E6F206D6559
:101B200073736167655D005B756E6B6E6F776E20BA
:101B30006572726F725D005B756E6B6E6F776E2093
:101B40007374617475735D0011241FBECFEFD0E113
:101B5000DEBFCDBF12E0A0E0B1E0E2E1F5ED00E0D4
:101B60000BBF02C007900D92A83CB107D9F71DE04A
:101B7000A8ECB2E001C01D92A331B107E1F70C94CB
:101B80002D0E0C94000081E08093C9020895982FD7
:101B90008091C802891731F0863021F0853029F410
:101BA000963019F080E090E008959093C802892F54
:101BB0008250823058F40E94E51D1092B606809142
:101BC000C802823051F40E94822807C0943019F470
:101BD0000E94081E02C00E94F41D8091C802863037
:101BE00011F40E94B6528091C802813019F482E04B
:101BF0000E94206448EC52E063E08FEF0E946B5338
:101C00000E94C30D81E090E0089508958091C8027C
:101C10009927089580E00E94F4192FEF8F3F9207D3
:101C200019F0682F80E009C081E00E94F4192FEFBD
:101C30008F3F920721F0682F81E00E94A13D0E9412
:101C400081530E945E620E94452C8091C9028823C4
:101C500011F40E94D418A8950895CFEFD0E1DEBF0B
:101C6000CDBF0E9483500E940B0F0E94C1240E948E
:101C7000DE600E94361E0E94C35021E04EE468E000
:101C80000E94380F21E04EE468E087E00E94511185
:101C90000E94EF1278940E94BD140E94BB50FC0178
:101CA00084810E943D1962E171E082E00E94721914
:101CB0000E940651813059F060E081E00E94EA17ED
:101CC00062E271E082E00E947219A895FECF6EE197
:101CD00071E082E00E94721960E081E00E94EA17E0
:101CE00066E582E00E94421962E371E082E00E94B0
:101CF00072190E94BB508C0181E00E94D516882386
:101D000019F081E00E94BE5082E00E94D51688231F
:101D100019F080E00E94BE5083E00E94D51688230F
:101D200019F082E00E94BE5084E00E94D5168823FC
:101D300019F083E00E94BE5080E00E94C70D80E051
:101D40000E94D516882319F084E10E944F4F0E940B
:101D5000DA5D40E050E060E28FEF0E946B5380E07C
:101D60000E94853D81E00E94853D8091B80690915A
:101D7000B906A091BA06B091BB06805D9740A0401D
:101D8000B04078F40E940A0E8091B8069091B9068E
:101D9000A091BA06B091BB06805D9740A040B040CC
:101DA00088F3F80181859285892BC9F00E94CA28A1
:101DB000EC0144969E01215F3F4FAC01B901F8014F
:101DC000818592850E94E95CBC01892B29F0F8018C
:101DD000818592858A8B9B8B6115710519F4F801B9
:101DE000628173818FEF0E94265281E011C00E94B0
:101DF000602C0E949717FFEF8F3F9F07C1F70E944B
:101E00000A0E8091C9028823A1F31092C90280E0D2
:101E10000E944B2AEECF8FE78ABB1BBA80E187BBBB
:101E200018BA80EF84BB8FEF85BB8BEB81BB8CEC4A
:101E300082BB86E082B987EF83B98093610081EF2E
:101E4000809362008FE18093640089E18093650054
:101E50000E946C5A10926A001ABE8AB78A608ABFC2
:101E60000E942E16A89588E181BD8CE081BD089561
:101E7000E82F10928A0680918A06809389068091C5
:101E800089068093AC068091AC068093AB0691E006
:101E90009093B5068C9A119A82B18E7E82B9199A66
:101EA00083B18E7E83B982E08BB99498E83008F0D4
:101EB000E92FFF27EE0FFF1FE85CFE4FA591B491BD
:101EC000653010F465E003C0693008F068E04F7DCC
:101ED0006550660F453411F4606203C04F3409F455
:101EE0006063223008F068608B2F992787FD9A95F0
:101EF0008F7080939000A9B96093950088EB8AB9A0
:101F000080E090E008959091AB068091AC06981720
:101F100011F00C9B559A089508951F920F920FB6D9
:101F20000F9211248F939F93EF93FF939091AB06A1
:101F30008091AC06981761F088B7806188BF0C9BD0
:101F400009C089B7806189BF8091B50680FF02C052
:101F5000559813C08091AC06E82FFF27E757F94F3B
:101F600084A18CB98091AC068F5F8093AC06809180
:101F7000AC06883010F01092AC06FF91EF919F9163
:101F80008F910F900FBE0F901F9018951F920F9278
:101F90000FB60F9211248F9389B78F7E89BF559A00
:101FA0008F910F900FBE0F901F9018951F920F9258
:101FB0000FB60F9211242F933F934F935F936F931C
:101FC0007F938F939F93AF93BF93EF93FF938091F2
:101FD0008906282F332780918A0699270197281789
:101FE000390741F0809189068F3179F480918A0612
:101FF000882359F480918A068F5F80938A068091A6
:102000008A06803210F010928A069BB18091890670
:10201000E82FFF27E757F94F8CB18283228194FD87
:102020000CC0809189068F5F809389068091890614
:102030008032A8F01092890612C0222381F42093E6
:102040008A0680918A06809389069498822F0E943E
:10205000853D21E04EE468E0822F0E94380F809198
:102060008906282F332780918A06281B310937FFDC
:1020700002C0205E3F4F213131050CF0949AFF9150
:10208000EF91BF91AF919F918F917F916F915F91F0
:102090004F913F912F910F900FBE0F901F90189569
:1020A00050E060E070E027E0813D920708F051E0E9
:1020B0002FE0813A920708F052E023E2893292073A
:1020C00008F053E026E3813B920708F054E026E451
:1020D0008135920708F055E028E8893B920708F01F
:1020E00056E0895D964D08F057E078948BB19927BA
:1020F00026E0969587952A95E1F79C01217030702E
:1021000080FFB9016F5F7F4FA89587E26031780744
:1021100068F321E04EE468E0852F0E94380F0895AF
:1021200089B1282F3327809190009927982F8827ED
:10213000282B392B60E040E050E0FA01E85CFE4FCC
:10214000859194918217930729F06F5F4E5F5F4FDF
:10215000683098F3862F99278330910509F18430F0
:1021600091054CF481309105A9F082309105ACF4D1
:10217000892B69F024C085309105C1F08530910527
:1021800094F086309105A9F00797B1F018C080EB64
:1021900094E0089580E699E0089580EC92E1089536
:1021A00080E895E2089580E498E3089580E09BE458
:1021B000089580E096E9089580E091EE089580E02A
:1021C00090E008950895482F07C08091AC068823B9
:1021D00091F4559A7894A8958091AB06282F3327CF
:1021E0008091AC06992701972817390791F38091C0
:1021F000AB06873051F38091AB06E82FFF27E757F6
:10220000F94F44A38091AB068F5F8093AB0680911A
:10221000AB06883010F01092AB06559A80E090E043
:10222000089580918906282F332780918A06281BDC
:10223000310937FF02C0205E3F4F203131050CF4D9
:1022400094989091890680918A06981719F48FEFD7
:102250009FEF089580918A06E82FFF27E757F94FEF
:102260008281282F332780918A068F5F80938A0688
:1022700080918A06803210F010928A06C901089572
:102280000895882331F08091B50681608093B5066A
:1022900008958091B5068E7F8093B506559A08956E
:1022A0000895E82F10925D0680915D0680935C068C
:1022B00080915C0680937F0680917F0680937E06E6
:1022C00091E09093880681B3886281BB8A981598C3
:1022D000939A92981D9882E080939B009598E8309D
:1022E00008F0E92FFF27EE0FFF1FE85CFE4FA591D6
:1022F000B491653010F465E003C0693008F068E01F
:102300004F7D6550660F8B2F992787FD9A958F70AB
:1023100080939800A0939900453411F4606203C043
:102320004F3409F46063223008F0686060939D00C8
:1023300088EB80939A0080E090E0089590917E066B
:1023400080917F06981739F00D9905C080919A0009
:10235000806280939A00089508951F920F920FB69D
:102360000F9211248F939F93EF93FF9390917E068A
:1023700080917F06981761F088B7806288BF0D9BB7
:102380000DC089B7806289BF8091880680FF06C032
:1023900080919A008F7D80939A0014C080917F066F
:1023A000E82FFF27E45AF94F84A180939C00809185
:1023B0007F068F5F80937F0680917F06883010F0C4
:1023C00010927F06FF91EF919F918F910F900FBE1A
:1023D0000F901F9018951F920F920FB60F92112415
:1023E0008F9389B78F7D89BF80919A008062809397
:1023F0009A008F910F900FBE0F901F9018951F920B
:102400000F920FB60F9211242F933F934F935F9328
:102410006F937F938F939F93AF93BF93EF93FF93AC
:1024200080915C06282F332780915D0699270197BC
:102430002817390741F080915C068F3179F480913B
:102440005D06882359F480915D068F5F80935D0659
:1024500080915D06803210F010925D0690919B0095
:1024600080915C06E82FFF27E45AF94F80919C0089
:102470008283828194FD0CC080915C068F5F809383
:102480005C0680915C06803278F010925C060CC08D
:10249000882351F480935D0680915D0680935C06ED
:1024A000959881E00E94853D80915C06282F332716
:1024B00080915D06281B310937FF02C0205E3F4F27
:1024C000213131050CF0959AFF91EF91BF91AF91B9
:1024D0009F918F917F916F915F914F913F912F913C
:1024E0000F900FBE0F901F901895482F0BC0809132
:1024F0007F068823B1F480919A00806280939A00CD
:102500007894A89580917E06282F332780917F06A6
:10251000992701972817390771F380917E06873034
:1025200031F380917E06E82FFF27E45AF94F44A348
:1025300080917E068F5F80937E0680917E06883034
:1025400010F010927E0680919A00806280939A002B
:1025500080E090E0089580915C06282F33278091D9
:102560005D06281B310937FF02C0205E3F4F203136
:1025700031050CF4959890915C0680915D06981752
:1025800019F48FEF9FEF089580915D06E82FFF27E4
:10259000E45AF94F8281282F332780915D068F5F9F
:1025A00080935D0680915D06803210F010925D068A
:1025B000C90108950895882331F0809188068160CB
:1025C000809388060895809188068E7F8093880680
:1025D00080919A00806280939A000895089587B34D
:1025E000876087BBBB9888B3896088BB1DB88EB1F4
:1025F0008FB187E78DB908951F920F920FB60F9292
:1026000011242F938F939F93EF93FF932FB180917A
:10261000CA02E82FFF27E653FD4F22838F5F809386
:10262000CA02883110F01092CA029091E502E92F97
:10263000FF27E653FD4F248D27FDC09A8091E402C9
:10264000981759F0C098892F8F5F8093E5028831E1
:1026500010F01092E5022FB902C0C09A6F98FF9156
:10266000EF919F918F912F910F900FBE0F901F9020
:1026700018958091E502282F33278091E402281BCA
:102680003109C90147968831910514F0C9010197B4
:1026900008950895282F6F9919C0C0988FB16F9A27
:1026A0008091E4029091E502891711F42FB91CC0C2
:1026B000E92FFF27E653FD4F848D8FB9892F8F5F58
:1026C0008093E502883110F01092E5028091E402D7
:1026D000E82FFF27E653FD4F248F8F5F8093E4029E
:1026E000883110F01092E40280E090E0089580912B
:1026F000CA022091CB02821719F48FEF9FEF089541
:10270000E22FFF27E653FD4F8281482F5527822F66
:102710008F5F8093CB02883110F01092CB02CA01F8
:10272000907008950895882311F0DD9A0895DD983A
:10273000089508950F931F93CF93282FDE9B63C0B6
:10274000882309F060C0809100039091010353E059
:10275000969587955A95E1F7182FC0910003C77099
:10276000022FCF9901E09BB3892F8F7A8BBB94FF07
:1027700002C081E001C0822F0E949313A091000348
:10278000B0910103412F55276C2F7727C0914F0A35
:10279000002399F0FA01EF52F54F20E830E002C033
:1027A000359527956A95E2F78081822B8083FA011F
:1027B000EF56F54F8081822B0EC0FA01EF52F54F94
:1027C00080E890E002C0959587956A95E2F7982F8A
:1027D00090958081892380839D012F5F3F4F3093A7
:1027E0000103209300038C2F992744E0880F991F41
:1027F0004A95E1F72817390758F0DC9A109201033F
:102800001092000305C0222311F0DE9A01C0DE9869
:10281000CF911F910F91089500000000000000006B
:102820000895882341F0809165008460809365005D
:102830000E940C140895809165008B7F8093650041
:10284000089508959B01AC018091B8069091B90656
:10285000A091BA06B091BB0682179307A407B507EB
:10286000A0F08091B8069091B906A091BA06B091F7
:10287000BB06821B930BA40BB50B80509041A0406C
:10288000B040A0F080E090E008958091B80690916B
:10289000B906A091BA06B091BB06281B390B4A0BAA
:1028A0005B0B2050304F4F4F5F4F18F081E090E0AE
:1028B000089580E090E008950895EF92FF920F93BD
:1028C0001F93AA27BB27E090B806F090B9060091A5
:1028D000BA061091BB06E80EF91E0A1F1B1F01C0A5
:1028E000A895C801B7010E9422148823C9F31F913B
:1028F0000F91FF90EF9008950F931F93CF93C82FE0
:10290000162F042F809165008D7F8093650080E0F5
:102910000E9411148AB38F608ABB8BB3807F9C2F77
:1029200092959F70892B8BBB112321F080916500BC
:10293000816003C0809165008E7F8093650081E097
:102940000E94111480E00E941114002329F088E0F5
:1029500090E00E945D140DC08BB3807FCF708C2BF4
:102960008BBB0E940C1481E00E941114802F0E94E6
:102970001114CF911F910F91089588E290E00E9469
:102980005D1441E060E080E30E947C1441E060E07F
:1029900080E30E947C1441E060E080E30E947C14AC
:1029A00041E060E080E20E947C1488E20E94E0172F
:1029B00088E00E94E01781E00E94E01786E00E9414
:1029C000E0178CE00E94E0176CE372E080E00E9468
:1029D000191964E172E081E00E9419196CE172E05A
:1029E00082E00E94191964E072E083E00E941919E4
:1029F00064EF71E084E00E9419196CEE71E085E0EB
:102A00000E94191964EE71E086E00E9419196CEDBC
:102A100071E087E00E94191908951F920F920FB676
:102A20000F9211241F932F933F934F935F936F93B4
:102A30007F938F939F93AF93BF93EF93FF93809177
:102A4000FE028F5F8093FE02282F237009F0F4C0EE
:102A500086958695877099278330910509F47CC007
:102A6000843091054CF48130910551F1823091050B
:102A7000DCF5892B89F0E0C08530910509F4A2C00E
:102A8000853091050CF49CC08630910509F4CEC0C8
:102A9000079709F4CFC0D0C08091B8069091B906CD
:102AA000A091BA06B091BB060196A11DB11D8093FD
:102AB000B8069093B906A093BA06B093BB0680C03F
:102AC0008091B8069091B906A091BA06B091BB0664
:102AD00081709070A070B070892B19F00E94E81678
:102AE000ABC00E94A916A8C081E00E949A130E9460
:102AF000060E833009F0A0C00E94411E2091B60648
:102B00003091B7068823E9F02E5F3F4F3093B70628
:102B10002093B6060E94BB50FC019681992309F4CC
:102B20008BC08AE0989F900111248091B606909105
:102B3000B7068217930708F47FC081E00E94C70D93
:102B40007BC02115310509F477C021503040309306
:102B5000B7062093B60670C08091FF02882309F45F
:102B60006BC08AB3807F8ABB822F0E941114809130
:102B70006500826080936500809165008E7F809300
:102B800065000000000081E00E94111419B380E08C
:102B90000E9411141295107F0E940C1481E00E9473
:102BA000111489B38F70182B80E00E941114812FAB
:102BB000992787FD90958827990F881F992733C0FB
:102BC000822F35C06091FF026623B1F59091BC065B
:102BD0008091BD06981789F01091BD06E12FFF275F
:102BE000E454F94F82811F5F103108F0162F8038AE
:102BF00091F48091BC06811719F480E090E013C035
:102C0000E12FFF27E454F94F82811F5F103108F054
:102C1000162F462F02C0462F61E00E947C141093AD
:102C2000BD0681E090E08093FF0206C081E00E9433
:102C30009A1302C00E947D17FF91EF91BF91AF914F
:102C40009F918F917F916F915F914F913F912F91C4
:102C50001F910F900FBE0F901F90189510927D003E
:102C600017BE11BE89E683BF87B7816087BF82EF39
:102C70008FBD3AE13EBD4FEC50E057BD46BD85EB00
:102C800090E09BBD8ABD99BD88BD22EC20938B004E
:102C900030938A0050938100409380009093870086
:102CA000809386000E94BB50FC01808580934F0A70
:102CB0000895EF92FF920F931F93AA27BB27E090EE
:102CC000B806F090B9060091BA061091BB06E80E5E
:102CD000F91E0A1F1B1F02C00E940A0EC801B7017D
:102CE0000E9422148823C1F31F910F91FF90EF904F
:102CF0000895282F220F61112160822F8370815047
:102D0000823028F424FF02C02E6001C0217F822F70
:102D10009927089590910403E92FFF27EC5FFC4F5A
:102D20008283892F8F5F80930403883010F0109284
:102D300004039091050380910403981741F4892FAF
:102D40008F5F80930503883010F01092050308957B
:102D500008950F931F9311B1812F8074682F809174
:102D600002030E947916082F809302031078612FC6
:102D7000809103030E94791680930303007C807C7A
:102D8000003829F4882339F0803C61F408C000340D
:102D900049F4803C11F484E103C0882319F485E1EF
:102DA0000E948A161F910F910895843118F080E0D7
:102DB00090E0089520E030E0E82FFF27E25FFC4F2D
:102DC0008081882311F021E030E0C9010895089541
:102DD000FF920F931F93CF9380912703E82FFF2734
:102DE000EE5DFC4F008113B31083FF248091270315
:102DF000E82FFF27EE0FFF1FEE0FFF1FEF0DF11D56
:102E0000E85BFE4FC49110FD42C000FF14C0C23108
:102E100029F481E10E94D516882331F48C2F0E9479
:102E20008A16C43108F054C0EC2FFF27E25FFC4F34
:102E300081E080834DC0C43108F04AC0EC2FFF27E9
:102E4000DF01A25FBC4F9C919F5F9C93992311F47B
:102E50009F5F9C93E131F105DCF1E331F1056CF00A
:102E60007397B1F580912103853690F18CE10E9432
:102E70008A1681E0809321032BC080911F0389373C
:102E800038F180912003893718F185E01FC0C431E3
:102E900028F4EC2FFF27E25FFC4F108200FD18C0E2
:102EA0008C2F80680E948A160E94060E853081F45D
:102EB000C13121F482E10E94D51605C0C23141F42E
:102EC00081E10E94D516882319F486E00E94C70D7F
:102ED00016950695F39483E08F1508F087CF8091BF
:102EE00027038F5F80932703853010F0109227030C
:102EF000CF911F910F91FF900895909127039430E7
:102F000029F485B3806F85BB97980895979A85B308
:102F10008F7020E130E002C0220F331F9A95E2F754
:102F2000922F9095907F892B85BB0895089580916D
:102F3000040320910503821719F48FEF9FEF089582
:102F4000E22FFF27EC5FFC4F8281482F5527822F0D
:102F50008F5F80930503883010F010920503CA013B
:102F600008950895CF93C82F06C08091BD06882389
:102F700089F40E9481538091BC06282F33278091C9
:102F8000BD06992701972817390799F38091BC0648
:102F90008F3059F3F8948091BC06E82FFF27E45452
:102FA000F94FC2838091BC068F5F8093BC068091ED
:102FB000BC06803110F01092BC067894CF91089531
:102FC0001F93182F80E80E94B217812F0E94B2171A
:102FD0001F9108958295880F880F807C860F8068E6
:102FE0000E94E01708950E94EA178EE00E94E01701
:102FF00008958CE00E94E0170895FF920F931F93AD
:10300000CF93F82E6091DF068091DE060E94EA17CA
:10301000C0E00EEC16E08091E006C81778F4FF20BF
:1030200021F0F80161918F0101C060E282E00E940D
:103030004219CF5F8091E006C81788F3CF911F91A6
:103040000F91FF9008959093E9068093E806892BED
:1030500089F17093E7066093E606CB01AA27BB27A8
:103060002091B8063091B9064091BA065091BB063E
:10307000280F391F4A1F5B1F2093E2063093E30697
:103080004093E4065093E5068091E1068E7F80939D
:10309000E106211531054105510561F42F5F3F4FD0
:1030A0004F4F5F4F2093E2063093E3064093E406D0
:1030B0005093E50608950895AF92BF92CF92DF92A4
:1030C000EF92FF920F931F93CF93DF93D82EC62ECC
:1030D000EA018EECE82E86E0F82E1092E9061092B6
:1030E000E80681E08D1568F1EFE0E61750F1411533
:1030F000510539F1FA0101900020E9F731970E2FBF
:10310000041B013108F000E16C2D8D2D0E94EA179F
:103110005701002361F0102F8881F50181935F0131
:103120008991682F82E00E9442191150A9F7F70196
:10313000D08AC18A028B64EF71E08DEF97E10E9423
:103140002318DF91CF911F910F91FF90EF90DF90A7
:10315000CF90BF90AF900895CF93DF93CDB7DEB7F8
:10316000A0970FB6F894DEBF0FBECDBF282FDE01AB
:10317000119690E0FA014F5F5F4F8491882321F010
:103180008D939F5F9F31B0F31C92AE014F5F5F4FF5
:10319000822F0E945C18A0960FB6F894DEBF0FBE77
:1031A000CDBFDF91CF9108958091E8069091E90617
:1031B000892BA9F16091E2067091E3068091E40603
:1031C0009091E5060E942214882349F18091E1063E
:1031D000E091E806F091E906817009958091E10699
:1031E00091E089278093E1068091E6069091E706B9
:1031F0009C01442755278091B8069091B906A0916B
:10320000BA06B091BB06820F931FA41FB51F80930F
:10321000E2069093E306A093E406B093E5060895D2
:1032200008951092E9061092E80681E00E94E017E6
:1032300008950F931F93CF93DF93EB018830C0F471
:10324000992723E0880F991F2A95E1F780640E944F
:10325000E01707E010E0FE01219684910E94B2176A
:103260000150104017FFF7CF60E0862F0E94EA1749
:10327000DF91CF911F910F910895813308F080E382
:1032800081BF089599278130910539F182309105E8
:103290001CF4892BF1F00895029711F567FF15C012
:1032A000643E31F0663F41F06C3F51F0643C11F4F4
:1032B00061EE0BC0663D11F46FEE07C06C3D11F47A
:1032C00065EF03C06F3D09F462EE862F0E94B217CE
:1032D0000895862F0E94E3100895862F0E9475128C
:1032E000089508951F93CF93DF93182FEB01FB01EF
:1032F0006491662349F0812F0E9442192196FE01B4
:103300008491682F8823B9F7DF91CF911F91089599
:103310001F93CF93DF93182FEB018881882341F00F
:103320008991682F812F0E94421988818823C1F7D3
:10333000DF91CF911F9108951F93CF93DF93CDB766
:10334000DEB7C055D0400FB6F894DEBF0FBECDBF7C
:1033500067961FAD679769968EAD9FAD6997AE0171
:10336000475A5F4FBC01CE0101960E943369BE01EE
:103370006F5F7F4F812F0E948819C05BDF4F0FB6B0
:10338000F894DEBF0FBECDBFDF91CF911F9108959E
:103390001F93CF93DF93CDB7DEB7C055D0400FB6A4
:1033A000F894DEBF0FBECDBF67961FAD67976996D5
:1033B0008EAD9FAD6997AE01475A5F4FBC01CE01FC
:1033C00001960E945C69BE016F5F7F4F812F0E9452
:1033D0008819C05BDF4F0FB6F894DEBF0FBECDBFBC
:1033E000DF91CF911F91089599278130910571F058
:1033F000823091051CF4892B31F00BC0029749F4FF
:103400000E94971708950E94111108950E94AB120F
:1034100008958FEF9FEF08950895FC018F3F910568
:1034200019F010F0E0E0F0E0E45AFD4F84919927A4
:10343000089590E08F3010F08EE001C081118F5F11
:10344000442311F028E001C0242F77276230710552
:1034500081F06330710524F46130710541F00EC0D4
:103460006330710541F06430710539F007C02360A5
:1034700005C0246003C0266001C02760281729F416
:10348000442311F02AE001C025E043E050E0990F09
:10349000990F80FD926020FD9160869526954150A0
:1034A000504057FFF4CF892F992708959C01FB01C5
:1034B0008F37910528F48F77808388E090E0089516
:1034C000832F9927806C8183208380E190E0089589
:1034D0000895FC014081242F33278181992701978A
:1034E0002817390729F04F3031F48181882319F4E6
:1034F00081E090E0089580E090E0089508951F93A2
:103500008AEE96E00E94691A182F8CE597E00E94D7
:10351000691A182B812F99271F910895AF92BF9296
:10352000CF92DF92EF920F931F93CF93DF93EC0133
:103530006B015A01122F80915A03882369F40B30D2
:1035400059F00C3049F0CB010E944D269927837029
:103550009070892B09F452C0CE010E94691A282F5D
:10356000882319F080E090E04BC088819927FC0106
:1035700073E0EE0FFF1F7A95E1F7E81BF90BEC0FF4
:10358000FD1FC282D38288819927FC0163E0EE0F80
:10359000FF1F6A95E1F7E81BF90BEC0FFD1FA482F2
:1035A000B58288819927FC0153E0EE0FFF1F5A95E1
:1035B000E1F7E81BF90BEC0FFD1F178388819927B2
:1035C000FC0143E0EE0FFF1F4A95E1F7E81BF90B02
:1035D000EC0FFD1F068388819927FC0133E0EE0F75
:1035E000FF1F3A95E1F7E81BF90BEC0FFD1FE08692
:1035F00088818F5F8883803108F0288381E090E0A4
:10360000DF91CF911F910F91EF90DF90CF90BF90FE
:10361000AF9008959F92AF92BF92CF92DF92EF92B8
:10362000FF920F931F93CF93DF93EC015B016A012D
:10363000922EF02E1E2D892B31F48CE597E00E94FE
:103640000A1BCAEED6E080915A03882321F087E056
:10365000CC35D807C1F00E94060E8250833098F412
:10366000F894E12E0F2D292DA601B501CE010E945F
:103670008E1A7894882329F485E090E00E945D14E6
:10368000EACF10925D03DF91CF911F910F91FF90D0
:10369000EF90DF90CF90BF90AF909F900895EF9202
:1036A0000F93CF93DF93EC01E62E0E940925FC01D6
:1036B000892B89F08085992783709070039711F486
:1036C00023E001C026E001E040E050E0BE018AEEC8
:1036D00096E00E940A1B81E090E0DF91CF910F916C
:1036E000EF900895EF920F93CF93DF93EC010E9438
:1036F0000925FC01892BA9F080859927837090709A
:10370000039731F486818F67E82E01E024E003C03F
:10371000EE2402E02BE040E050E0BE01CA010E942E
:103720000A1B81E090E0DF91CF910F91EF90089517
:10373000EF920F93CF93DF93EC010E940925FC01D8
:10374000892B81F08085992783709070019702976B
:1037500048F4EE2402E02BE040E050E0BE01CA0154
:103760000E940A1B81E090E0DF91CF910F91EF90D2
:103770000895EF920F93CF93DF93EC010E940925F8
:10378000FC01892B79F080859927837090700197CF
:1037900049F4EE240AE024E040E050E0BE01CA0112
:1037A0000E940A1B81E090E0DF91CF910F91EF9092
:1037B0000895AF92BF92CF92DF92EF920F93CF9383
:1037C000DF935C016B010E940925EC01892B09F450
:1037D00051C088859927837090708230910571F56A
:1037E000D7FE05C06E81888199810E944F1BC0FE63
:1037F00009C0EE8006E024E040E050E0B501CA01D7
:103800000E940A1BC1FE09C0EE8007E024E040E0F0
:1038100050E0B501CA010E940A1BC2FE09C0EE8039
:1038200008E024E040E050E0B501CA010E940A1B14
:10383000C3FE20C0EE8009E024E016C00397D1F457
:10384000C6018F709078892B49F0EE2403E024E0C4
:1038500040E050E0B501CA010E940A1B8C2D807F18
:1038600049F0EE2404E0202F40E050E0B501CA0109
:103870000E940A1B81E090E0DF91CF910F91EF90C1
:10388000DF90CF90BF90AF900895EF920F931F936A
:10389000CF93DF93EC01162F0E944D268370815049
:1038A000823050F4EE2402E0212F40E050E0BE01CF
:1038B0008AEE96E00E940A1B81E090E0DF91CF91B2
:1038C0001F910F91EF900895EF920F93E62E6623CC
:1038D00019F0EE240CE001C00BE023E040E050E0E2
:1038E000BC01CA010E940A1B81E090E00F91EF9099
:1038F0000895EF920F93262FEE240DE040E050E064
:10390000BC01CA010E940A1B81E090E00F91EF9078
:103910000895EF920F93EE240EE0282F40E050E040
:10392000BA01CA010E940A1B81E090E00F91EF905A
:103930000895EF920F93FC0180915A03882319F4A4
:1039400080E090E013C06770862F806F442311F0F1
:10395000862F886FE82E01E121E040E050E0BF01B2
:103960008AEE96E00E940A1B81E090E00F91EF90B2
:103970000895EF920F93FC0180915A03882319F464
:1039800080E090E013C06770862F806E442311F0B2
:10399000862F886EE82E01E121E040E050E0BF0173
:1039A0008AEE96E00E940A1B81E090E00F91EF9072
:1039B0000895EF920F93FC01E62E80915A0388231D
:1039C00019F480E090E00BC002E121E040E050E01B
:1039D000BF018AEE96E00E940A1B81E090E00F9101
:1039E000EF900895EF920F93FC01E62E80915A0319
:1039F000882319F480E090E00BC003E121E040E06F
:103A000050E0BF018AEE96E00E940A1B81E090E040
:103A10000F91EF900895EF920F93FC01E62E8091A5
:103A20005A03882319F480E090E00BC00FE021E0F6
:103A300040E050E0BF018AEE96E00E940A1B81E060
:103A400090E00F91EF900895EF920F93FC01E62E16
:103A500080915A03882319F480E090E00BC000E1C4
:103A600021E040E050E0BF018AEE96E00E940A1B90
:103A700081E090E00F91EF900895EF920F93FC0199
:103A8000E42E04E124E0AB01BF0180E090E00E945D
:103A90000A1B81E090E00F91EF900895982F882302
:103AA00091F01092EB068091EB068093EA0681E09C
:103AB00080935C0380915C0380935A03BD9A87B71F
:103AC000846087BF089587B78B7F87BF90935A0321
:103AD000BD98C59808950895EF920F93E0905A030A
:103AE000EE2069F5882359F1E092EB068091EB0610
:103AF0008093EA0688E1EAE2F3E011928A95E9F719
:103B00000EE022E040E050E0BA018AEE96E00E942A
:103B10000A1B81E080935C038BE390E099BD88BD34
:103B200088B599B59BBD8ABD87E790E097BD86BDF6
:103B30001DBC1CBC87B7846087BFBE9A05C0BE98F9
:103B4000C69887B78B7F87BF0F91EF900895EF924C
:103B50000F93E0905A03EE2071F5882361F1E09213
:103B60005D0780915D0780935C0788E1E2E4F3E004
:103B700011928A95E9F70EE022E040E050E0BA01A8
:103B80008CE597E00E940A1B8BE390E090938700FE
:103B90008093860087E790E0909381008093800077
:103BA000109289001092880080917D00846080933B
:103BB0007D00139A07C013981B9880917D008B7F1E
:103BC00080937D000F91EF90089580E00E944E1D3C
:103BD00081E00E946C1D81E00E94A71D809162001F
:103BE000846080936200089580E00E944E1D809161
:103BF00062008B7F8093620080E00E946C1D80E0F9
:103C00000E94A71D10925C0381E00E942064089529
:103C100080E00E946C1D80E00E94A71D81E00E9450
:103C20002064809162008B7F8093620088E1EAE2E9
:103C3000F3E011928A95E9F783E080933C038FEFDC
:103C400080932A038BE390E099BD88BD88B599B530
:103C50009BBD8ABD87E790E097BD86BD81E00E944D
:103C60004E1D82E090E00E94591608950E94BB50BC
:103C7000FC01808182FF02C0C79A0895C798089509
:103C800008950E94BB50FC01808182FF07C080E044
:103C900090E0B79907C081E090E0089586B3992736
:103CA00080789070089508950E94060E833021F068
:103CB0000E94060E843021F480915D0399270895B7
:103CC00081E090E00895089580915B03992708951D
:103CD00010925B030895909372038093710308958B
:103CE00080916F0390917003089580E1EEE5F3E019
:103CF00011928A95E9F710926E0310927003109258
:103D00006F038FEF9FE79093720380937103089581
:103D100078941F920F920FB60F9211242F933F9316
:103D20004F938F939F93EF93FF9380916E0388300F
:103D300010F010926E0380916E03E82FFF27EE0FB4
:103D4000FF1FE25AFC4F24B135B1208331838F5FCE
:103D500080936E031092700310926F0320E030E0A6
:103D600047E0EEE5F3E081919191280F391F415032
:103D700047FFF9CF3093700320936F038091710355
:103D800090917203821793071CF481E080935B0388
:103D9000FF91EF919F918F914F913F912F910F90B4
:103DA0000FBE0F901F9018956F927F928F929F92E7
:103DB000AF92BF92CF92DF92EF92FF920F931F9339
:103DC000CF93DF93EC015B0188246C55774011F4AD
:103DD00071E0872EF50190818181981709F08AC0E2
:103DE000882019F481E080935D0380915A03882331
:103DF00039F0EE240DE021E040E050E0BA0177C058
:103E0000882019F00E94332602C00E94D8256C0138
:103E1000009731F4EE2401E022E0AC01BC0167C060
:103E2000FC0180859927837090708230910581F024
:103E3000833091051CF4019721F05CC00397D1F108
:103E400059C0F601E68001E022E040E050E04DC0BC
:103E5000F6011681E12E01E022E040E050E06081B1
:103E60007181C5010E948E1A0E94D4258370482F4B
:103E700055274130510591F04230510524F4411548
:103E8000510541F037C04230510559F043305105DA
:103E900071F030C0E12E06E022E026C0E12E07E0FE
:103EA00002C0E12E08E022E040E050E01DC0E12E1B
:103EB00009E0F9CFF601E68001E0202F40E050E074
:103EC00060817181C5010E948E1A0E94D4259927B4
:103ED000AC014170507080FF04C0EE2403E021E08B
:103EE000E3CFEE2404E021E0F60160817181C50199
:103EF0000E948E1AF50181819927FC0163E0EE0F83
:103F0000FF1F6A95E1F7E81BF90BEA0DFB1DE28044
:103F1000F380F50181819927FC0153E0EE0FFF1F2B
:103F20005A95E1F7E81BF90BEA0DFB1D64807580DB
:103F3000F50181819927FC0143E0EE0FFF1F4A95AF
:103F4000E1F7E81BF90BEA0DFB1D0681F501818104
:103F50009927FC0133E0EE0FFF1F3A95E1F7E81BCC
:103F6000F90BEA0DFB1D9084F50181819927FC0175
:103F700023E0EE0FFF1F2A95E1F7E81BF90BEA0D8E
:103F8000FB1D2781215027832223B1F4F501818174
:103F90009927FC0113E0EE0FFF1F1A95E1F7E81BCC
:103FA000F90BEA0DFB1D2683F50181818F5F81836B
:103FB0008181803108F02183802F8B50823070F412
:103FC0000E94BB50FC01808181FF03C0B3E0BB2E87
:103FD00002C0A1E0BA2ECC24DD2408C010915A03FF
:103FE000112331F0CC24DD24F3E0BF2E10E014C007
:103FF000C7010E9409256C01009731F0192DFC01C1
:10400000B084F3E0BF2206C0E1E0BE2E0E3011F412
:1040100073E0B72E811010788B2D99278130910590
:104020000CF442C28330910524F0039709F406C1D1
:104030003BC2C7010E940D1A982F829586958695DE
:1040400083708A83292F220F220F298361E0A62EF5
:10405000AA8A82E1888B82E0898BC114D10449F15C
:10406000F6018481958197FF02C023602983812F07
:1040700099278F779070892BE1F0F60180850E9457
:10408000C1280F97B4F01F5FF60180850E94CF24EE
:10409000892B29F410FF03C089818A258983212F68
:1040A0002078812F99278F71907095958795122F81
:1040B000182B802F99278730910509F48FC08830FD
:1040C00091059CF48230910509F47DC083309105FF
:1040D00024F4019709F43FC0E7C18330910509F446
:1040E0003AC0069709F474C0DFC18A30910509F41B
:1040F0008BC08B30910544F48830910509F478C069
:10410000099709F47BC0D0C10D970CF0CDC1C70150
:1041100043E0969587954A95E1F7907001960E9445
:104120000D1A982F82958695869583708A83990FAC
:10413000990F99830B3011F418820AC0F7E0EF222F
:10414000FF2484E592E0E80EF91EF701849188834C
:1041500082E08A8B3AC081E090E017FD892F212F01
:104160002F702F3010F02EE001C021112F5FF1E0F1
:10417000BF1661F443E050E0990F990F20FD936062
:1041800026954150504057FFF7CF1BC0882331F090
:10419000283010F085E007C08DE005C0283010F40D
:1041A0008AE001C082E043E050E0990F990F20FDC2
:1041B000926080FD9160269586954150504057FF52
:1041C000F4CF988371C180EC888384E0898B6CC1C3
:1041D000F60184818170482F61E005C0F601848179
:1041E0008270482F62E0812F8F770E94191A24C0B5
:1041F000F60184818470482F63E0F5CFF601848155
:104200008870482F64E0EFCFC7010E940D1A982FE5
:1042100082958695869583708A83990F990F93600E
:10422000998382E08A8BF601848195818F709070EA
:104230008C5B9D4FFC018491888336C183E08A8B1F
:1042400031E0B32EB98A88E1888B802F99278D3091
:10425000910509F4D5C08E309105BCF484309105E8
:1042600009F4B6C08530910544F48130910509F414
:104270003DC0039709F496C009C18530910509F442
:10428000B4C00B970CF402C10FC08231910524F425
:104290000F970CF0C5C0BFC0843191050CF4D8C095
:1042A000449709F4E4C0F2C088E090E0E80EF91EFB
:1042B000C70123E0969587952A95E1F78F7380686B
:1042C0008A83C7018095909515E0969587951A95F4
:1042D000E1F7282F207720688E2D8770282B2983DF
:1042E0000C3009F0D3C028602983D0C0F601808546
:1042F00099278C7090700897B9F48FE38A83812F87
:1043000099278F779070009731F08F37910511F4CE
:10431000117801C01F5F1983CE010396BC01C7014C
:104320000E94561A885EB1C017FF02C080E601C025
:1043300080E48983F60180850E94C128212F3327DC
:10434000BE016E5F7F4F0F97B4F0C9018F779070F9
:10435000009731F08F37910511F412E001C01D5F15
:10436000812F86958F709981982B998310FF2BC090
:104370009061998328C0C9018F779070009731F0C0
:104380008F37910511F411E001C01F5F1F70298163
:10439000212B2983F6018481958197FF14C0206128
:1043A000298311C080E88983F60124812F70822F30
:1043B000806889838481958197FF02C02069298361
:1043C000CE010296BC01C7010E94561A805F5DC0F3
:1043D00080EA8983F60184819581B4E0969587957A
:1043E000BA95E1F78F70806B09C080EA8983F60186
:1043F00084819581892F99278F70806A8983E0CF86
:104400001982CE010296BC01C7010E94561A805F34
:10441000888BB98A3BC08FEF8A83198281E025C0DF
:10442000013111F488E707C0003111F484E703C0BB
:104430000F3011F48CE78B838F2D9927982F937071
:104440008B81892B8B83EA82998280E2888B0CC0D6
:1044500080E78A83023111F488E78A838E2D877082
:104460009A81982B9A8399828AE0898B0FC0872D35
:10447000992783708C6E8B836A829982CE01049611
:10448000BC01C7010E94561A805E888B20E0988983
:10449000969596959695915031F0FE01E90FF11D94
:1044A00080812827F8CF28838A89833011F01092E1
:1044B0005C03DF91CF911F910F91FF90EF90DF9000
:1044C000CF90BF90AF909F908F907F906F90089506
:1044D000CF93DF93DC01FC018489882319F42589BB
:1044E000222361F021E0882321F08150FD01848B9B
:1044F00021C0FD0185898150858B1CC0FD01828909
:10450000833019F487898823A9F4FD019389892FC1
:10451000869586958695E80FF11D8081282F332793
:10452000892F99278770907002C0359527958A95B5
:10453000E2F72170FD013289832F9927823091059E
:1045400031F083309105CCF0039721F016C0CBE613
:10455000D0E015C0222319F0C7E7D0E002C0CEECAE
:10456000D0E0FD018389882351F48689882339F4BA
:1045700082E0858B81E0868B2BC0C7EDD0E0FD010A
:104580008389882329F58589882311F581898823E2
:1045900099F480915C038823D9F480915A0388238D
:1045A000B9F481E00E94DC50882319F0C35BDF4E30
:1045B0000FC0CD5ED94F0CC0832F99278130910554
:1045C00029F0029729F4C857DD4F02C0C05FDA4FC7
:1045D000CE01DF91CF910895DC01FC01848988230D
:1045E00019F48589882311F021E02BC0FD0133895E
:1045F000932F9150938B8289833069F427892223EA
:1046000051F4892F992787709070079721F481E0E2
:10461000878B338B16C0FD01178A9389892F869566
:1046200086958695E80FF11D8081282F3327892FE5
:1046300099278770907002C0359527958A95E2F783
:104640002170FD01828999278230910549F08330DC
:1046500091051CF4019761F01BC0039789F018C005
:10466000222319F08CE590E0089580E190E0089510
:10467000222319F08EEB90E008958CE190E00895EC
:10468000222319F08BE390E0089587E690E00895E7
:104690008BE390E008950895FC018089838B8189E4
:1046A000823010F482E0818B8289992781309105D4
:1046B000B4F0833091051CF0039761F010C081E0E5
:1046C0000E94DC50882319F08DE490E1089583E185
:1046D00096E0089580E1848B82E390E0089582E380
:1046E00090E0089508951F920F920FB60F92112433
:1046F0001F932F933F934F935F936F937F938F936A
:104700009F93AF93BF93CF93DF93EF93FF938091EA
:104710005A03882331F00E94641E882311F01092FE
:104720003B03809128038823A1F080915C038823B8
:1047300029F08BE390E099BD88BD02C019BC18BC7C
:104740008BE390E09BBD8ABD87E790E097BD86BD77
:104750005EC0CAE2D3E0CE010E946822AC019C0197
:10476000255030408CB59DB58217930718F457BD7E
:1047700046BD0EC08CB59DB5C29697BD86BDCE0117
:104780000E944C232CB53DB5280F391F37BD26BDDF
:1047900080913D03882381F510913F03112361F53A
:1047A00080913B03882381F481E08093280386B7BE
:1047B000846086BF78946AEE76E08AE293E00E9495
:1047C000D41EF8941092280380913B038150898B6A
:1047D00080913A038B8B80913C03833049F4809124
:1047E0005A03882311F084E101C080E18C8B01C061
:1047F0001C8B1D8A1F8A1E8A8AE293E00E94EC228B
:1048000099279BBD8ABD8AB59BB599BD88BDFF918F
:10481000EF91DF91CF91BF91AF919F918F917F9158
:104820006F915F914F913F912F911F910F900FBE0C
:104830000F901F9018951F920F920FB60F92112490
:104840001F932F933F934F935F936F937F938F9318
:104850009F93AF93BF93CF93DF93EF93FF93809199
:1048600029038823B1F080915C03882339F08BE31E
:1048700090E0909387008093860004C01092870098
:104880001092860087E790E09093810080938000EB
:1048900064C0C2E4D3E0CE010E946822AC019C0156
:1048A00025503040809188009091890082179307AD
:1048B00028F4509381004093800016C080918800B6
:1048C00090918900C2969093810080938000CE01E0
:1048D0000E944C232091880030918900280F391FB5
:1048E000309381002093800080915503882361F5E7
:1048F00010915703112341F580915303882391F4BC
:1049000081E08093290380917C00846080937C0007
:1049100078946CE577E082E493E00E94D41EF894EA
:1049200010922903809153038150898B8091520307
:104930008B8B80915403833019F480E18C8B01C000
:104940001C8B1D8A1F8A1E8A82E493E00E94EC223F
:1049500099279093870080938600FF91EF91DF91D4
:10496000CF91BF91AF919F918F917F916F915F9107
:104970004F913F912F911F910F900FBE0F901F905D
:10498000189580E892E0EEECF7E011920197E9F7D4
:10499000109274031092730310924E0A08958F7050
:1049A00020E030E08550823010F421E030E0C90191
:1049B00008950F931F93CF93DF93CDB7DEB724975E
:1049C0000FB6F894DEBF0FBECDBF8FEF9FEFAFEFF6
:1049D000BFEF89839A83AB83BC8300E210E044E09D
:1049E00050E0B801CE0101960E94A7640E940A0E11
:1049F0000C5F1F4F8FE00D3F180788F324960FB60A
:104A0000F894DEBF0FBECDBFDF91CF911F910F9104
:104A100008959C01009741F408958AE0A89FC00181
:104A200011248253984F0895A0E0B0914E0AAB171D
:104A3000A0F440E050E0BA01FA01E60FF71FE2539C
:104A4000F84F808191818217930739F3AF5F6F5FD1
:104A50007F4F475F5F4FAB1778F380E090E008959A
:104A60000895CF92DF92EF92FF920F931F93CF930F
:104A7000DF93CDB7DEB723970FB6F894DEBF0FBE36
:104A8000CDBF7C016C010894C108D1088FEFC81616
:104A900087E2D806A0F5C7010E9409258C01892B61
:104AA00009F072C020914E0A203450F48AE0289F09
:104AB000800111240253184F2F5F20934E0A22C009
:104AC0000EEC17E0B80120E030E0A901AFE3F901F6
:104AD000E40FF51FE253F84F9185F801818589179E
:104AE00008F48B01A1504F5F5F4F275F3F4F665F18
:104AF0007F4FA7FFECCFF8018185882319F480E070
:104B000090E043C0F801E082F182FFEFCF16F7E2B8
:104B1000DF06E0F480E2E82EF12CA89543E050E0B7
:104B2000B701CE0101960E948B6429813A81F80178
:104B30008081918128173907C9F084E090E0E80E60
:104B4000F91E9DEFE9169FE0F90638F3F801808120
:104B500091818F3F910519F010F083E00BC088E040
:104B60000E94DC50882321F083E003C08B8101C0C8
:104B700082E0F801808780E8F8018683148215823C
:104B80001282138211861782C80123960FB6F894F9
:104B9000DEBF0FBECDBFDF91CF911F910F91FF9070
:104BA000EF90DF90CF900895809175039927089535
:104BB000EF92FF921F93CF93DF9390914E0A992328
:104BC00019F480E090E049C0809173038F5F809377
:104BD0007303891738F0809175038F5F8093750395
:104BE00010927303909173038AE0989FE00111245F
:104BF000C253D84F80917503992787709070892B85
:104C0000A9F41E81E12EFF24C7018F779070892BB4
:104C100069F088850E94CF24892B41F0E0FC06C012
:104C20001F5F612F888199810E944F1B80917503BE
:104C3000992787709070049751F48885992783701D
:104C40009070019721F4888199810E94B91B898510
:104C50008F3F11F08F5F8987CE01DF91CF911F9138
:104C6000FF90EF90089590914E0A992319F480E0F7
:104C700090E00895809174038F5F80937403891787
:104C800010F010927403909174038AE0989FC00111
:104C900011248253984F089508950E940925FC011C
:104CA000009709F4089580859927089508950E9432
:104CB0000925FC01009709F4089586819927089534
:104CC00008950E940925FC01009709F40895848144
:104CD000958108950895BF92CF92DF92EF92FF924F
:104CE0000F931F93CF93DF93CDB7DEB723970FB604
:104CF000F894DEBF0FBECDBF7C01B62E0E943125D9
:104D0000FC01892BB1F180858B1599F1B086118654
:104D10009FEFC92ED92E00E210E0A89543E050E0A5
:104D2000B801CE0101960E948B6489819A818E150B
:104D30009F0511F468010DC0D7FE05C028E2803040
:104D4000920708F068010C5F1F4F2FE00D3F12071C
:104D500020F38E159F0511F0D7FC0BC0BB82E982B2
:104D6000FA82A89544E050E0B601CE0101960E9477
:104D7000A76423960FB6F894DEBF0FBECDBFDF91B8
:104D8000CF911F910F91FF90EF90DF90CF90BF9048
:104D90000895CF92DF92FF920F931F93CF93DF93EB
:104DA000EC01F62E142F892B09F47BC088850E9414
:104DB000C128482F5885752F73708F2D99278F77AD
:104DC0009070242F3327281739071CF420E8F2228B
:104DD000F42A6E816F1509F464C01986112319F045
:104DE0008F8181608F838F2D992780789070C62E58
:104DF000DD249601207830708217930771F1C60187
:104E00008F779070009711F020E8F2227330B1F4A0
:104E1000892BD1F4852F99278C7090700897E9F42D
:104E20008F2D99278F779070892BB9F48F2D816002
:104E3000682F888199810E944F1B0FC0892B49F0F0
:104E4000888199810E944F1B888199810E94721BE1
:104E500004C0888199810E94981BFE820F2D112722
:104E6000C8018F779070892BB9F088850E94CF2474
:104E7000892B91F000FD03C08F2D8F5F08C008942F
:104E8000C108D1080C151D0539F48F2D8150682FEC
:104E9000888199810E944F1B6F2D888199810E9482
:104EA0004F1BDF91CF911F910F91FF90DF90CF901B
:104EB0000895FF920F931F93CF93DF93EC01162F6A
:104EC000F42E0E94060E833009F01078CE010E9465
:104ED0003125EC010E814F2D612F0E94C9268A8158
:104EE0009B810097B1F00E943125EC018E81282F23
:104EF000332720783070802F99278078907028177A
:104F0000390711F080E818274F2D612FCE010E943C
:104F1000C926DF91CF911F910F91FF900895EF92D5
:104F2000FF920F931F93CF93DF93EC017B01892BAB
:104F3000E1F10C811D8106171707B9F11986442389
:104F400019F08F8181608F83EC82FD82888599279B
:104F5000837090708130910531F0813091052CF192
:104F600004971CF51BC0980120703078C701807031
:104F700090782817390729F06E81888199810E94DD
:104F80004F1B0F7010708FE0E822FF240E151F05D5
:104F900061F0888199810E94B91B07C00E251F25E9
:104FA000B801888199810E94D91BDF91CF911F910F
:104FB0000F91FF90EF900895FF920F931F93CF935F
:104FC000DF938B01F42E0E943125EC01892B49F1EE
:104FD0008A819B81892B01F1C8018F709F7B4F2DA6
:104FE000BC01CE010E948F278A819B810E943125BE
:104FF000EC01892BB1F0C80180709074880F991F63
:10500000007F107024E0169507952A95E1F7802B14
:10501000912B4F2DBC0102C04F2DB801CE010E9433
:105020008F27DF91CF911F910F91FF900895EF92FD
:10503000FF920F931F93CF93DF937C018B010E940C
:105040003125EC01892B61F0C8010E943125FC015A
:10505000892B31F00A831B831986E282F382118641
:10506000DF91CF911F910F91FF90EF9008950097DE
:1050700059F00E943125FC01892B31F08281938106
:10508000128213821186F3CF08950895EF92FF9252
:105090000F931F93CF93DF93CDB7DEB726970FB64D
:1050A000F894DEBF0FBECDBF7C010E9409258C01A4
:1050B000892BD9F0B701CE0101960E94E852F80180
:1050C000448155816681CE0101960E94CB52AE018A
:1050D0004F5F5F4F6AE08FEF0E946B53F80144818E
:1050E00055816681C7010E94322926960FB6F89431
:1050F000DEBF0FBECDBFDF91CF911F910F91FF900B
:10510000EF9008951F93CF93DF9310E0CEECD7E09C
:1051100090914E0A1917F0F48985899FC0011124D6
:105120008035910534F08E8199278F779070892B87
:1051300059F08E8180788E83888199810E94721BBC
:10514000888199810E9446281F5F2A9690914E0A75
:10515000191710F3DF91CF911F9108950F931F93AB
:105160008C01C8010E943D1D84E00E94891C61E001
:10517000C8010E94791C8AE00E94891C1F910F912E
:105180000895E82FFF27EF70F070E455FC4F8491ED
:105190009927089586E793E008958091840382FF1C
:1051A00005C08091780390917903089580917603EA
:1051B000909177030895089580918403826080938D
:1051C000840308950F931F93CF93DF93C6E7D3E033
:1051D0008091840399278C010170107080FF03C0B7
:1051E00080E090E021C060917C0370917D0380910C
:1051F0007E0390917F03611571058105910531F062
:105200000E942214882311F4C8010EC01A821B8246
:105210001A8A1B8A10927703109276031E861C8AC4
:105220000E94C30D81E090E0DF91CF911F910F911B
:1052300008959C018091780390917903892B11F452
:10524000C90108952F703F7B77FD3064CB018F70CB
:10525000907044E0880F991F4A95E1F7822B932BB9
:1052600008950895FC018091760390917703209131
:10527000780330917903E817F907F9F4609386030E
:10528000232BB1F080917A0390917B03F4E0969503
:105290008795FA95E1F7BC016F707070892F992797
:1052A0008695869580FD7068CA010E9419290FC0F5
:1052B00050937B0340937A030EC0E217F30759F42F
:1052C000BA0180917A0390917B030E9419299093EF
:1052D0007B0380937A030E94C30D08959C01892B60
:1052E00069F41092840310927C0310927D03109253
:1052F0007E0310927F030E94E22808956093860344
:1053000050937B0340937A038091B8069091B9063D
:10531000A091BA06B091BB0688519C4FAF4FBF4FCA
:10532000816080937C0390937D03A0937E03B09370
:105330007F038091840382FF10C081608B7F809304
:1053400084033093790320937803B9018091760325
:10535000909177030E94172807C08E7F8093840363
:1053600030937703209376030E94C30D0895089528
:10537000209184032B7F21602093840390937903F1
:105380008093780380917A0390917B030E9419297E
:1053900090937B0380937A030E94C30D08958093BA
:1053A00085030E94C128809387030E94C30D08953E
:1053B000CF93C82F882319F064ED71E002C064EF29
:1053C00071E084E00E941919CC2319F06CEC71E0B3
:1053D00002C06CEE71E085E00E941919CC2319F02F
:1053E00064EC71E002C064EE71E086E00E9419197D
:1053F000CC2319F06CEB71E002C06CED71E087E03A
:105400000E941919CF910895CF93DF93C82FDD27FC
:10541000C4FF02C083E001C085EA0E94B217C0FF4A
:1054200002C084E001C085EA0E94B217C1FF02C039
:1054300085E001C085EA0E94B217C2FF02C086E083
:1054400001C085EA0E94B217C3FF02C087E001C015
:1054500085EA0E94B217DF91CF9108958093960359
:105460000E94C30D0895882319F06CE971E002C011
:1054700064EA71E082E00E94191908950895882372
:1054800019F06CEA71E002C064EB71E081E00E9407
:105490001919089508950F931F93CF9306E713E00A
:1054A000C0919603CC2399F060E081E00E94EA1756
:1054B0008C2F81500E94DE4FBC0182E00E94721945
:1054C0001092960388EE93E00E94591602C088233A
:1054D00019F00E94111903C0682F0E94EA178091E9
:1054E000760390917703892BF9F00E94BB50FC0161
:1054F00082819381409176035091770384179507B9
:1055000049F4218532858091880390918903281779
:10551000390751F042835383809188039091890326
:10552000818792870E9442502091760330917703C1
:105530002115310529F4F80124833583108A178653
:105540008091840382FD0DC080918003909181033E
:10555000A0918203B09183030097A105B10519F1D1
:1055600005C06CEB73E082E00E94721980918003A9
:1055700090918103A0918203B0918303BF93AF9375
:105580009F938F938FEB93E09F938F9382E08F9302
:105590000E94C8198DB79EB707960FB6F8949EBFA4
:1055A0000FBE8DBF43C02115310531F462ED73E0AC
:1055B00082E00E94721918C03F932F9389ED93E007
:1055C0009F938F93C2E0CF930E94C8198091840368
:1055D0000F900F900F900F900F9080FF02C08C2FB4
:1055E00001C080E20E94B217C09185030E94060E9E
:1055F000853010F085E00EC0833061F48C2F992740
:105600008370907023E0880F991F2A95E1F7845AE0
:105610009C4F08C0992703E0880F991F0A95E1F76E
:1056200084589C4FBC0182E00E9472196CE080E0BB
:105630000E94EA178091860399278F7790709F9335
:105640008F938EED93E09F938F9382E08F930E94D0
:10565000C819809185039927837090700F900F90DF
:105660000F900F900F90019779F483E10E94D51667
:10567000882331F080E00E94B21764E671E010C028
:1056800080E20E94B2170FC080E00E94B2178091A2
:10569000860387FF03C06CE372E002C064E372E03C
:1056A00080E00E9419190E94060EC82F813049F42B
:1056B00088E00E94A94FAC0160E08C2F0E94AC18DA
:1056C000E0C040E050E060E0862F0E945C18C0E03F
:1056D0008AE00E94D516882371F08091780390911A
:1056E0007903892B39F48091850399278370907011
:1056F000039709F4C1E060E081E00E94EA1780911D
:10570000800390918103A0918203B091830300975D
:10571000A105B10509F442C08DE00E94D516882389
:1057200029F48EE00E94D516882381F182EE93E061
:105730009F938F93C2E0CF930E94C8198DE00E947F
:10574000D5160F900F900F90882379F06CEA71E0D6
:1057500081E00E94191964EA71E08C2F0E941919E6
:105760006CE271E08FE39AE20EC064EB71E081E0DD
:105770000E9419196CE971E08C2F0E9419196CE2D2
:1057800071E083E39AE20E9423187BC086E00E94C6
:10579000A94FBC0182E00E94721944C08091780335
:1057A00090917903009769F19F938F938EEE93E028
:1057B0009F938F9382E08F930E94C81980917A0300
:1057C00090917B0314E0969587951A95E1F7282F21
:1057D0002F70892F9927869586950F900F900F909F
:1057E0000F900F9080FD2061822F0E94042ACC230D
:1057F00021F08CE30E94B21715C080E20E94B2171C
:105800002CC08AE893E09F938F9383EF93E09F935C
:105810008F9382E08F930E94C8190F900F900F9082
:105820000F900F90CC23C9F0809178039091790369
:10583000892B99F480917A0390917B03A4E096954B
:105840008795AA95E1F78F7080610E94042A81E014
:105850000E94D8296CEF71E011C020917A032F705B
:1058600080917A0390917B0397FD2061822F0E94A3
:10587000042A80E00E94D82964E072E083E00E945C
:105880001919CF911F910F91089560917C03709128
:105890007D0380917E0390917F03611571058105E1
:1058A000910561F00E942214882341F010927C033C
:1058B00010927D0310927E0310927F030895089545
:1058C000EF92FF920F931F93CF93DF93EC01E6E7E4
:1058D000EE2EE3E0FE2E81319105CCF48F30910560
:1058E0000CF0D0C08A30910509F4F4C18B309105D9
:1058F00034F4009709F40BC197FDFBC11BC18C3038
:10590000910509F462C00D970CF07EC044C1853149
:105910009105D9F18631910574F48231910509F42C
:10592000D1C0823191050CF4E4C083319105D1F1ED
:105930004497B1F0DEC18F3891056CF48D38910534
:105940000CF062C08C31910509F4B4C08A3891051D
:1059500009F4CDC1CEC18339910509F4C8C1C9C1CB
:105960008091860399278F77907020918703332742
:10597000821793070CF0BDC10E94060E833009F018
:10598000B8C1809186038F5F1DC020918603822F4E
:1059900099278F779070892B09F4ABC12150209300
:1059A0008603A5C180918503992783709070019724
:1059B00029F464E671E080E00E9419198091860361
:1059C000809580788093860392C18AE00E94D516E4
:1059D000882399F08091780390917903892B69F05D
:1059E00080917A0390917B0320E030E48227932713
:1059F00090937B0380937A037AC180917A0390918C
:105A00007B0320E030E850C08091800390918103B7
:105A1000A0918203B09183030097A105B10581F1A4
:105A2000209180033091810321503040220F331F99
:105A3000CE018F7790700E9709F42160C7FF1AC0CE
:105A400041E060E0C9010E94FA6160E070E0CB01D2
:105A50000E94231864E172E081E00E9419196CE150
:105A600072E082E00E941919F701128613861486EB
:105A700015863DC141E0642FC9010E94FA6137C11A
:105A8000C7FD35C11C2F1D508AE00E94D51681111B
:105A90001C5F21E030E002C0220F331F1A95E2F7AD
:105AA00080917A0390917B0382279327F701848367
:105AB00095831DC16CE380917603909177030E94DA
:105AC000451C15C1F89483E00E94C70D882319F086
:105AD00084E00E94206483E10E94D516882339F077
:105AE0006BE480917603909177030E94451C789433
:105AF000FEC08AE00E94D516811182E00E94C70D87
:105B0000882309F4F4C084E00E942064F0C08091EE
:105B1000800390918103A0918203B0918303009749
:105B2000A105B10539F48FEF0E944F4F81E00E942B
:105B30004B2ADFC08091800390918103A091820362
:105B4000B09183039C01AD0163E0220F331F441F1A
:105B5000551F6A95D1F7280F391F4A1F5B1F280F61
:105B6000391F4A1F5B1FCE01AA2797FDA095BA2FA8
:105B7000280F391F4A1F5B1F2030F8E23F07F0E073
:105B80004F07F0E05F070CF0B4C0F70122873387BE
:105B900044875587ACC0C6E7D3E02091800330919D
:105BA0008103409182035091830360917803709147
:105BB0007903211531054105510509F47FC06115AF
:105BC000710519F10091760310917703C801AA2796
:105BD000BB2782179307A407B50741F0CB01AA277B
:105BE000BB2782179307A407B50779F48091840334
:105BF0008E7FF7018687C8010E943728F70112823D
:105C0000138210927703109276038091760390911D
:105C100077039C014427552780918003909181034D
:105C2000A0918203B0918303609184032817390700
:105C30004A075B0729F481E068276B7F6E8745C0C0
:105C40006C7F6E871A8A1B8A1C8A60918A0381E0A6
:105C50000E94EA1780E00E94A94FBC0182E00E94E6
:105C600072198091840399279695879596958795C3
:105C70009C012170307080FD11C02A833B832C83EE
:105C80003D8330937703209376031F8660918003D2
:105C9000709181038FEF0E9426520BC040918003C8
:105CA0005091810360917603709177038FEF0E948A
:105CB0004252809184038B7F8E8707C0672B29F423
:105CC000809184038460F70186871A861B861C8670
:105CD0001D860DC0109280031092810310928203E2
:105CE00010928303809184038B7F809384030E94AE
:105CF000C30DDF91CF911F910F91FF90EF90089509
:105D0000FC01EC5BFF4F8081E454F040882319F4E0
:105D100080E090E00895E95BFF4F8081E754F04018
:105D2000882329F48481883511F0883719F481E0BB
:105D300090E0089580E090E008950895CF93DF9378
:105D4000EC010E94802E882319F480E090E01FC0AF
:105D5000FE01E95BFF4F8081882351F4CC5BDF4F6C
:105D60008881C454D040823018F481E090E00FC0A4
:105D70008081882311F08C8101C08D81992787FD56
:105D80009095809590958827990F881F9927DF9186
:105D9000CF910895CF93C82FCF7719F480E090E08A
:105DA00029C0862F0E94C128282F33272B31310587
:105DB00089F02C31310524F42E30310529F017C03B
:105DC0002C31310569F013C0EC2FFF27EB5CFB4F42
:105DD00084910BC0EC2FFF27E75EFB4F849105C039
:105DE000EC2FFF27E450FC4F8491992703C0CF5F2D
:105DF0008C2F9927CF910895CF93C82FCF7719F47F
:105E000080E090E02EC0C150862F0E94C128282F2C
:105E100033272B31310579F02C31310524F42E3024
:105E2000310529F01CC02C31310569F018C08C2FC8
:105E3000992708960DC083E0C89FC00111240B96D6
:105E40006EE070E007C08C2F9927880F991F079686
:105E500069E070E00E94EE69CB01992702C08C2FA7
:105E60009927CF910895019791F40E94BB50FC01AE
:105E70008181882311F484E608C0843011F485E61A
:105E800004C08150843008F08150992708958FEF25
:105E90009FEF089508951F93CF93C82FFB01142FF0
:105EA0008181282F332782819927982F8827282BB3
:105EB000392BC90101978F5F974210F062E010C043
:105EC000112321F0C9010E94312503C0C9010E949C
:105ED0000925009751F4112311F06BE001C06AE02D
:105EE0008C2F0E94421980E090E0CF911F9108957D
:105EF000EF92FF920F931F93CF93DF93EB01E42E6A
:105F000041E00E944B2F8C01892B19F48FEF90E018
:105F100064C00E947F1A882319F088E090E05DC079
:105F2000FB80EE2051F021E0F21639F4F82EF80152
:105F3000808191810E94721B08C0EE2031F0F8012F
:105F400060858B810E94FC2EF82E6C81862F99270C
:105F500085FF02C0F0E8FF2AF801C481D581DF7710
:105F600084FDD06867FF05C0C07F8F709070C82B1C
:105F7000D92B2F2D332720783070F8016681862F9A
:105F80009927807890702817390731F0607840E0C1
:105F9000808191810E94592740E06F2DF801808116
:105FA00091810E94592740E0BE01F80180819181D2
:105FB0000E94DC27F801808191810E9446280E947E
:105FC000060E833019F480E090E007C0823019F4A7
:105FD00081E490E002C082E490E0DF91CF911F91D4
:105FE0000F91FF90EF90089541E00E94782F99273C
:105FF000089540E00E94782F992708951F93CF932A
:10600000DF93182F40E0812F0E944B2FEC01892B4A
:10601000F1F060E0812F0E94421968858E810E9414
:10602000CA2E682F812F0E9442196C816F708C815B
:106030009D8197FD60618E8187FD6062812F0E9446
:1060400042198E818F77682F812F0E9442198FEF1E
:1060500090E0DF91CF911F9108951F93CF93DF932D
:10606000182F40E0812F0E944B2FEC01892BC9F0A3
:1060700060E0812F0E94421988858370682F812FEC
:106080000E94421988850E94C128682F812F0E9492
:1060900042196FEF812F0E9442196FEF812F0E94EA
:1060A00042198FEF90E0DF91CF911F9108950F93E8
:1060B0001F93CF93DF938B0141E00E944B2FEC01A4
:1060C000892B19F48FEF90E014C08C819D81807032
:1060D000F80123813327822B932B40E0BC01888178
:1060E00099810E94DC27888199810E94462880E05E
:1060F00090E0DF91CF911F910F9108950F931F931F
:10610000CF93DF938B0141E00E944B2FEC01892B51
:1061100019F48FEF90E018C02C813D81307CF8019C
:10612000838199278F739070982F8827282B392B7C
:1061300040E0B901888199810E94DC27888199819A
:106140000E94462880E090E0DF91CF911F910F914F
:1061500008951F93CF93DF93182F40E0812F0E9463
:106160004B2FEC01892B41F060E0812F0E944219F6
:106170006C81812F0E9442198FEF90E0DF91CF91C7
:106180001F9108951F93CF93DF93182F40E0812F25
:106190000E944B2FEC01892B69F060E0812F0E9457
:1061A00042198C819D81892F99278F73682F812FA8
:1061B0000E9442198FEF90E0DF91CF911F910895D7
:1061C000DF92EF92FF920F931F93CF93DF93982F5D
:1061D0008B01823008F066C088E4989F700111241A
:1061E00087E993E0E80EF91EFB018181C82FDD27C6
:1061F0008281992787709070982F8827C82BD92B78
:106200002197F7E0C83FDF0718F082E090E04CC02C
:106210000E94BB50FC01808181FD07C023E0CD3F7F
:10622000D20718F08EE090E03FC00E94060E833047
:1062300039F00E94060E823019F086E090E034C0FA
:10624000CC0FDD1FF801628167FFC160862F99279F
:10625000E6E096958795EA95E1F771E0D72ED8228A
:1062600087010B5B1F4FF80180819181FFEF8F3F0A
:106270009F0749F040E0642F0E94FA618FEF9FEF83
:10628000F8018083918340E06D2DCE010E94FA6178
:10629000882319F489E090E007C0DD2019F0F801A7
:1062A000C083D18380E090E0DF91CF911F910F9167
:1062B000FF90EF90DF900895FF920F931F93CF937D
:1062C000F82EFB018181082F112782819927877081
:1062D0009070982F8827082B192B87E0083F180704
:1062E00018F082E090E022C0C8010E94EA60873680
:1062F00011F0873411F4C4E001C0C0E00E94BB502B
:10630000FC01808181FF02C0C16006C00C5F1340A8
:1063100018F08EE090E00AC060E08F2D0E944219D4
:106320006C2F8F2D0E9442198FEF90E0CF911F911B
:106330000F91FF9008951F93CF93182FFB01C181F8
:10634000CC2319F482E090E00FC060E00E94421973
:10635000EC2FFF27E05FF44F80818095682F812F1D
:106360000E9442198FEF90E0CF911F9108951F93E3
:10637000CF93182FFB01C181C150C03218F082E0C9
:1063800090E015C060E00E94421960E08C2F0E94EE
:106390004A5A682F812F0E94421961E08C2F0E9477
:1063A0004A5A682F812F0E9442198FEF90E0CF91B7
:1063B0001F9108950E94655A80E090E008951F9310
:1063C000CF93182FFB0181819927009719F003972C
:1063D00029F008C0C0914F0ACC0F07C0C091500AE5
:1063E000C17003C082E090E00AC060E0812F0E948B
:1063F00042196C2F812F0E9442198FEF90E0CF91AC
:106400001F910895FB0181819281282F3327211547
:10641000310521F02330310559F014C0913490F446
:10642000892F992701969595879580934F0A0DC0DE
:106430008091500A992311F0816001C08E7F809372
:10644000500A03C082E090E0089580E090E0089553
:106450000895EF92FF920F931F93CF93DF93CDB7E1
:10646000DEB760970FB6F894DEBF0FBECDBFF82E33
:1064700063E00E94421961E08F2D0E94421964E09E
:106480008F2D0E94421960E08F2D0E94421964E016
:106490008F2D0E9442190E94F850DC01CB01BF935E
:1064A000AF939F938F9384E494E09F938F938E0197
:1064B0000F5F1F4F1F930F930E94C3648DB79EB74A
:1064C00008960FB6F8949EBF0FBE8DBF33E0E32E43
:1064D000F80191919295907F81918F018053982B33
:1064E000692F8F2D0E944219EA94E7FEF1CF80E0D8
:1064F00090E060960FB6F894DEBF0FBECDBFDF917F
:10650000CF911F910F91FF90EF9008951F93CF931C
:10651000182FC0E00E94060E982F8250823008F497
:10652000C8E0923009F4C0616C2F812F0E9442199B
:106530008FEF90E0CF911F9108951F93CF93DF933A
:10654000182FFB018181282F332782819927982FCB
:106550008827822B932B0E94332FEC0197FF03C0D7
:1065600082E090E00AC060E0812F0E9442196C2F07
:10657000812F0E9442198FEF90E0DF91CF911F9100
:10658000089560E00E94421982E00E94C70D8FEFDB
:1065900090E0089580E00E94C70D80E090E00895AB
:1065A00083E00E94C70D80E090E0089580E090E0D5
:1065B00008951F93CF93DF93182F0E94BB63EC01C4
:1065C00060E084E0989F812D9927112480FD61E08F
:1065D000CE01892F992782958695877080FD64600A
:1065E000C0FD6860D7FD6062CE7FDF71209709F043
:1065F0006068812F0E944219209791F060E0C1FDF0
:1066000061E0C2FD6064C97F209709F06068812F56
:106610000E944219CD2B21F060E0812F0E94421987
:106620008FEF90E0DF91CF911F9108950F931F930B
:10663000CF93DF93182FCEECD7E000E080914E0A85
:10664000081778F58F8180FF29C068858E810E94A8
:10665000CA2E682F812F0E9442196C81812F0E94BF
:1066600042196881812F0E94421988819981892F5E
:106670009927682F6F738C819D8197FD60648E814F
:1066800087FD6068812F0E9442198E818F77682F65
:10669000812F0E9442198F818E7F8F830F5F2A96F0
:1066A000CDCF80E890E0DF91CF911F910F910895B9
:1066B0006F927F928F929F92AF92BF92CF92DF9212
:1066C000EF92FF920F931F93CF93DF93CDB7DEB777
:1066D000C254D0400FB6F894DEBF0FBECDBF882E97
:1066E00001E010E0AA249A2CB1E0BB2E7E01E00E5E
:1066F000F11E3701C92CDD24F601EF5EF34FE08176
:10670000EE2319F4095F1F4F2CC0EB2141F1F70173
:1067100001937F01812F992787708083C80101979A
:106720000E94EA60982F873411F0873621F4F70130
:10673000808180688083973411F0923521F4F701CD
:106740008081806480830894E11CF11CA394F6018D
:10675000EF5EF34F9B2D9095808189238083BB0C46
:1067600019F49394F1E0BF2E0F5F1F4FF7E0093F3C
:106770001F0720F48FE18A1508F0BCCF6A2D882D01
:106780000E944219DD2473010A2D112701151105FC
:1067900081F0F70181917F01682F882D0E944219B5
:1067A000D3942D2D3327C801800F911F2817390747
:1067B00084F38FEF90E0CE5BDF4F0FB6F894DEBF2F
:1067C0000FBECDBFDF91CF911F910F91FF90EF9042
:1067D000DF90CF90BF90AF909F908F907F906F9001
:1067E0000895CF92DF92EF92FF920F931F93CF9372
:1067F000DF93D82ECC2480914F0A882309F454C00B
:10680000F8948C2D992787FD9095880F991F9C01EE
:106810002F52354F8C010F56154FEC01CF5AD54FE3
:106820004881942F9095D8018C918923F901E080BB
:10683000E82A5981952F9095F80181818923F901E2
:10684000F180F82A2E2D332727FD3095842F9927A4
:106850002817390749F42F2D332727FD3095852F29
:1068600099272817390799F08C2D8F5F682F8D2D68
:106870000E9442196E2D8D2D0E9442196F2D8D2D73
:106880000E944219E882F982F801118210827894FC
:10689000C3942C2D332727FD309580914F0A9927DB
:1068A000281739070CF4ACCF60E08D2D0E944219F7
:1068B0008FEF90E0DF91CF911F910F91FF90EF90BC
:1068C000DF90CF9008951F93CF93C82F162F603479
:1068D00018F06AE474E002C064E574E08C2F0E9452
:1068E0007219812F99278A30910589F18B30910592
:1068F0007CF48630910511F1873091051CF40297E4
:10690000D1F039C088309105F9F00997D1F033C042
:106910008E30910529F18F30910534F48B3091053B
:10692000C9F00D97D1F027C081349105E1F0823490
:106930009105E1F020C06CE574E01AC060E774E0F6
:1069400017C06DE774E014C060E974E011C063EA39
:1069500074E00EC06BEA74E00BC06DEB74E008C02D
:1069600066EC74E005C06DED74E002C068EE74E0A2
:106970008C2F0E947219103420F06DE08C2F0E9431
:10698000421981E090E0CF911F9108950F931F93DA
:10699000D8018A30C0F48617B0F49927FC0114E0BE
:1069A000EE0FFF1F1A95E1F7E81BF90BE95DFB4FAE
:1069B0008685882341F0008111810417150718F09E
:1069C0002017310708F48D01C8011F910F91089518
:1069D00063EF74E00E94721981E090E008956AE22A
:1069E00075E00E94721981E090E0089567E475E017
:1069F0000E94721981E090E008951F93182F60E8BB
:106A000075E00E9472196AE975E0812F0E9472197F
:106A100069EB75E0812F0E94721981E090E01F916F
:106A20000895CF93C82F0E94060E992783309105B1
:106A3000A1F0843091052CF4009749F0029751F0B1
:106A400017C08430910561F0079794F40CC066ED8F
:106A500075E00BC06EED75E008C066EE75E005C030
:106A60006DEE75E002C069EF75E08C2F0E9472191F
:106A700081E090E0CF910895EF92FF920F931F93E2
:106A8000182F7B01042F80E00E94C70D402FB70113
:106A9000812F0E94113599271F910F91FF90EF9040
:106AA0000895EF92FF920F931F93182F7B01042FED
:106AB00083E00E94C70D402FB701812F0E9411353E
:106AC00099271F910F91FF90EF9008956FEF75E058
:106AD0000E94721982E00E94C70D80E090E0089544
:106AE0000F931F93CF93C82F762F642F00E010E0F1
:106AF000A801872F0E94C6348C01892B21F462E003
:106B00008C2F0E946334C801CF911F910F9108957B
:106B10007F928F929F92AF92BF92CF92DF92EF922D
:106B2000FF920F931F93CF93DF93882E942E2FEF16
:106B300037E260E00E9470355C01009719F481E053
:106B400090E062C10E9409256C01892B69F421E063
:106B5000291510F06AE012C0C5010E9431256C01B0
:106B6000892B11F46BE00AC031E0391508F0D6C06A
:106B70000E947F1A782E882331F068E0882D0E94C9
:106B80006334992741C1F601C481D58150EFE52EC8
:106B90005FE7F52EEC22FD228D2F992787FD90953A
:106BA0008827990F881F99278C0121E030E040E069
:106BB00050E0692D82E00E94C634892B21F020E04C
:106BC00030E8E22AF32ACE01817090708C0121E036
:106BD00030E040E050E0692D84E00E94C634892B0B
:106BE00021F081E090E0E82AF92ACE019695879578
:106BF000817090708C0121E030E040E050E0692D20
:106C000085E00E94C634892B21F0E2E0F0E0EE2A14
:106C1000FF2ACE01969587959695879581709070FD
:106C20008C0121E030E040E050E0692D86E00E94D8
:106C3000C634892B21F024E030E0E22AF32A83E0F5
:106C4000D695C7958A95E1F7C170D0708E0121E085
:106C500030E040E050E0692D87E00E94C634892B87
:106C600021F088E090E0E82AF92A472DB701C50114
:106C70000E94DC27F601608586810E94CA2E992732
:106C80008C012FE730E040E050E0692D81E00E9468
:106C9000C634C82F80915604863411F411E015C013
:106CA000823511F4172D11C000E010E0F601868145
:106CB00087FF02C001E010E021E030E040E050E05A
:106CC000692D83E00E94C634182FC13029F4C0E03A
:106CD000C5010E94721B06C0F60160858C2F0E94C0
:106CE000FC2EC82F1111C0682C2F3327207830704C
:106CF000F6016681862F99278078907028173907CA
:106D000029F0607840E0C5010E94592740E06C2FCF
:106D1000C5010E945927C5010E9446280E94060EFF
:106D2000823011F461E405C00E94060E833021F028
:106D300062E4882D0E946334F6018481958183FF8B
:106D400003C081E390E002C080E390E09F938F93C3
:106D5000F6018481958182FF03C081E390E002C047
:106D600080E390E09F938F93F6018481958181FF6A
:106D700003C081E390E002C080E390E09F938F9393
:106D8000F6018481958180FF03C081E390E002C019
:106D900080E390E09F938F93F601868187FF03C085
:106DA00086E690E002C082E790E09F938F93F60121
:106DB0008581282F332727FD309520953095222770
:106DC000330F221F332781E390E0821B930B9F93A5
:106DD0008F93608586810E94CA2E99279F938F93F7
:106DE000BF92AF9289E096E09F938F938F920E941B
:106DF000C81981E090E02DB73EB72D5E3F4F0FB62A
:106E0000F8943EBF0FBE2DBFDF91CF911F910F9120
:106E1000FF90EF90DF90CF90BF90AF909F908F90BA
:106E20007F900895CF93C82F2FEF37E260E08C2F2B
:106E30000E947035009719F10E940925FC01892BE9
:106E400019F463E276E018C080859927837090700A
:106E50008230910561F0833091051CF4019721F097
:106E60000EC0039739F00BC06AE276E005C067E315
:106E700076E002C064E476E08C2F0E94721981E013
:106E800090E0CF9108957F928F929F92AF92BF92A0
:106E9000CF92DF92EF92FF920F931F93CF93DF93E6
:106EA000A82EB42E2FEF37E260E00E9470354C011F
:106EB000009719F481E090E021C10E9409256C013E
:106EC000892B69F421E02B1510F06AE012C0C4018F
:106ED0000E9431256C01892B11F46BE00AC031E06E
:106EE0003B1508F08FC00E947F1A782E882331F05E
:106EF00068E08A2D0E946334992700C1F601E4807E
:106F0000F580E701C070C701817090708C0121E0AD
:106F100030E040E050E06B2D81E00E94C634892BC8
:106F200009F0C160C70196958795817090708C01BA
:106F300021E030E040E050E06B2D82E00E94C6345A
:106F4000892B09F0C260C70196958795969587951C
:106F5000817090708C0121E030E040E050E06B2DBA
:106F600083E00E94C634892B09F0C46063E0F69484
:106F7000E7946A95E1F7F1E0EF22FF24870121E031
:106F800030E040E050E06B2D84E00E94C634892B55
:106F900009F0C860870121E030E040E050E06B2D4F
:106FA00085E00E94C634892B09F0C061870121E089
:106FB00030E040E050E06B2D86E00E94C634892B23
:106FC00009F0C062870121E030E040E050E06B2D25
:106FD00087E00E94C634892B09F0C064870121E054
:106FE00030E040E050E06B2D88E00E94C634892BF1
:106FF00009F0C068472DBE01C4010E94DC27C4010E
:107000000E9446280E94060E882321F462E48A2DFD
:107010000E946334F6018481958187FF03C081E378
:1070200090E002C080E390E09F938F93F60184810B
:10703000958186FF03C081E390E002C080E390E089
:107040009F938F93F6018481958185FF03C081E32F
:1070500090E002C080E390E09F938F93F6018481DB
:10706000958184FF03C081E390E002C080E390E05B
:107070009F938F93F6018481958183FF03C081E301
:1070800090E002C080E390E09F938F93F6018481AB
:10709000958182FF03C081E390E002C080E390E02D
:1070A0009F938F93F6018481958181FF03C081E3D3
:1070B00090E002C080E390E09F938F93F60184817B
:1070C000958180FF03C081E390E002C080E390E0FF
:1070D0009F938F939F928F9288E496E09F938F93D4
:1070E000AF920E94C81981E090E02DB73EB72B5EA9
:1070F0003F4F0FB6F8943EBF0FBE2DBFDF91CF912B
:107100001F910F91FF90EF90DF90CF90BF90AF90C5
:107110009F908F907F9008957F928F929F92AF92D1
:10712000BF92CF92DF92EF92FF920F931F93CF9374
:10713000DF93A82EB42E2FEF37E260E00E94703567
:107140004C01009719F481E090E02EC10E940925BE
:107150006C01892B69F421E02B1510F06AE012C054
:10716000C4010E9431256C01892B11F46BE00AC027
:1071700031E03B1508F09DC00E947F1A782E8823CD
:1071800031F068E08A2D0E94633499270DC1F60121
:10719000C481D5817FEFE72E70ECF72EEC22FD2223
:1071A0008D2F9927817090708C0121E030E040E0B4
:1071B00050E06B2D81E00E94C634892B21F020E045
:1071C00031E0E22AF32ACE01892F99278695817032
:1071D00090708C0121E030E040E050E06B2D82E0C7
:1071E0000E94C634892B21F080E092E0E82AF92A37
:1071F000CE01892F992786958695817090708C0194
:1072000021E030E040E050E06B2D83E00E94C63486
:10721000892B21F0E0E0F4E0EE2AFF2ACE01892F4D
:107220009927869586958695817090708C0121E0CE
:1072300030E040E050E06B2D84E00E94C634892BA2
:1072400021F020E038E0E22AF32ACE01892F9927A5
:1072500082958F70817090708C0121E030E040E069
:1072600050E06B2D85E00E94C634892B21F080E030
:1072700090E1E82AF92ACD2FDD27C295C695C7707F
:10728000C170D0708E0121E030E040E050E06B2D05
:1072900086E00E94C634892B21F0E0E0F0E2EE2A7D
:1072A000FF2A472DB701C4010E94DC27C4010E94B8
:1072B00046280E94060E882321F462E48A2D0E944B
:1072C0006334F60184819581892F9927829586956B
:1072D000877080FF03C081E390E002C080E390E00C
:1072E0009F938F93F60184819581892F99278295A9
:1072F0008F7080FF03C081E390E002C080E390E0E4
:107300009F938F93F60184819581892F9927869584
:107310008695869580FF03C081E390E002C080E3FC
:1073200090E09F938F93F60184819581892F99270F
:107330008695869580FF03C081E390E002C080E3DC
:1073400090E09F938F93F60184819581892F9927EF
:10735000869580FF03C081E390E002C080E390E067
:107360009F938F93F60184819581892F992780FFC0
:1073700003C081E390E002C080E390E09F938F938D
:107380009F928F9285E696E09F938F93AF920E9493
:10739000C81981E090E02DB73EB72F5E3F4F0FB682
:1073A000F8943EBF0FBE2DBFDF91CF911F910F917B
:1073B000FF90EF90DF90CF90BF90AF909F908F9015
:1073C0007F900895AF92BF92CF92DF92EF92FF929B
:1073D0000F931F93CF93DF93A82EC42F0E94060E06
:1073E000882311F466E05DC028EF37E04C2F60E0A1
:1073F0008A2D0E9470356C01892B19F021E02A1525
:1074000018F481E090E083C088E4A89EC0011124B4
:1074100089569C4FC23008F44EC0A5E4EA2EF12CE8
:10742000E80EF91EF70180819181FFEF8F3F9F07E2
:1074300049F040E0642F0E94FA618FEF9FEFF7015F
:107440008083918380913804873411F4BB2410C069
:10745000823519F4F1E0BF2E0BC002E010E021E00C
:1074600030E040E050E06C2F81E00E94C634B82E3E
:1074700000E010E021E030E0A8016C2F82E00E94E3
:10748000C634EC01860101501040000F111F0B0D96
:10749000111D40E0682FC8010E94FA61882331F471
:1074A00069E08A2D0E946334992731C0CC2319F0FA
:1074B000F70100831183C60101970E94EA60C0E0D2
:1074C000D0E0082F112707FD1095C8010E94156A0A
:1074D000892B11F0C1E0D0E0DF93CF93C8010E9467
:1074E000286A9F938F93DF92CF928DE796E09F93C8
:1074F0008F93AF920E94C81981E090E02DB73EB7FC
:10750000275F3F4F0FB6F8943EBF0FBE2DBFDF91F0
:10751000CF911F910F91FF90EF90DF90CF90BF9090
:10752000AF9008951F93182F68E876E00E947219B3
:1075300065E976E0812F0E9472190E94F850DC0103
:10754000CB01BF93AF939F938F938BE996E09F936B
:107550008F931F930E94C8198DB79EB707960FB6D9
:10756000F8949EBF0FBE8DBF81E090E01F910895FB
:10757000EF92FF920F931F93CF93DF93E82EF42E99
:107580000E94BB50EC01FF20E1F08B8599278C0114
:1075900024E130E040E050E06F2D80E00E94C634EE
:1075A0008B878C859927880F991F8C012EEF31E0EE
:1075B00042E050E06F2D81E00E94C6349695879599
:1075C0008C878C859927880F991F9F938F938B8524
:1075D00099279F938F9388EA96E09F938F93EF92DA
:1075E0000E94C8198DB79EB707960FB6F8949EBF34
:1075F0000FBE8DBF81E090E0DF91CF911F910F9181
:10760000FF90EF9008950F931F93CF93C82F642F8F
:10761000442379F08091500A9927817090708C01F1
:1076200021E030E040E050E080E00E94C6340E945B
:107630005A5A8091500A9927817090709F938F9326
:1076400081EB96E09F938F93CF930E94C8190F9080
:107650000F900F900F900F9081E090E0CF911F91CD
:107660000F910895DF92EF92FF920F931F93CF93A4
:10767000E82E842F00E010E020E230E041E050E00E
:10768000682F80E00E94C634C82F882309F447C0C1
:1076900099279F938F9387EB96E09F938F93EF9219
:1076A0000E94C819DC2EDA9460E08D2D0E944A5A9F
:1076B000082F112781E0F82E0F900F900F900F9058
:1076C0000F90C7E08F2D992780239123892B11F0EC
:1076D00061E301C060E38E2D0E944219C150FF0C8E
:1076E000C7FFF0CF60E28E2D0E94421961E08D2D20
:1076F0000E944A5A082F1127C1E0FC2EC7E08F2DA7
:10770000992780239123892B11F061E301C060E365
:107710008E2D0E944219C150FF0CC7FFF0CF81E0AF
:1077200090E0CF911F910F91FF90EF90DF9008951F
:10773000FF920F931F93F82E642F80914F0A992781
:10774000880F991F8C0120E430E040E050E080E099
:107750000E94C6348F5F869580934F0A9927880FC1
:10776000991F9F938F938AED96E09F938F93FF923B
:107770000E94C8190F900F900F900F900F9081E00A
:1077800090E01F910F91FF900895CF93C82F44234D
:10779000C9F4C13031F460EE76E08C2F0E9472198A
:1077A00013C00E9490109F938F9386EE96E09F9354
:1077B0008F93CF930E94C8190F900F900F900F9046
:1077C0000F9002C0C13019F481E090E00DC069EE65
:1077D00076E08C2F0E9472198091270490912804E2
:1077E0000E94501080E090E0CF9108950F931F9376
:1077F000CF93C82F842F0FEF1FEF27EE33E040E029
:1078000050E0682F80E00E94C6340E94332F97FF1B
:1078100006C062E08C2F0E946334992711C09070DB
:107820009F938F938CEE96E09F938F93CF930E94BC
:10783000C81981E090E00F900F900F900F900F907B
:10784000CF911F910F910895EF92FF920F931F9385
:10785000982F642F4423C9F088E4989F7001112465
:1078600087E993E0E80EF91E00E010E021E030E047
:10787000A80180E00E94C634F701E95BFF4F892B25
:1078800019F081E0808301C0108281E090E01F91B7
:107890000F91FF90EF900895DF92EF92FF920F9378
:1078A0001F93CF93DF93082FEB01D42E823008F083
:1078B0000EC188E4089F9001112429563C4F48814D
:1078C000142F1F71642F7727CB01807E9070803436
:1078D000910509F4A3C08134910534F40097A9F00F
:1078E000809709F463C0F3C08038910509F4BFC0E4
:1078F000813891052CF48036910509F4B0C0E7C0B9
:10790000803C910509F4CCC0E2C021E02D1508F0BF
:10791000E0C08981C82FDD27CE010E943125FC01FE
:10792000892B09F4D4C0E480F58014FF05C080E001
:1079300090E8E82AF92A04C08FEF9FE7E822F922AD
:107940001F70068100781F3019F460E8602729C095
:1079500080851F7011F01F3019F460E070E020C0C6
:107960000E94C128282F33272C31310571F02D3189
:10797000310524F42B31310529F010C02E373105A3
:1079800031F00CC0110F115009C0110F07C089E070
:10799000189F802D1124682F772702C0612F772729
:1079A000602B40E0CE010E94592750C0437F48839E
:1079B00075E4E72EF12CE20EF31EF7018081918130
:1079C000FFEF8F3F9F0749F040E0642F0E94FA616C
:1079D0008FEF9FEFF701808391832881203209F494
:1079E00076C0233209F473C0F1E0FD15D0F469814B
:1079F000213231F4C62FDD272197CC0FDD1F05C0C2
:107A0000C62FDD27CC0FDD1F219740E061E0CE01BE
:107A10000E94FA61F701C083D18359C0F1E0FD15DE
:107A200018F080E090E055C08981C82FDD27CE0195
:107A30000E94612640EFE42E4FEFF42EE822F92257
:107A4000812F99278F709070E82AF92A40E0B701BA
:107A5000CE010E94DC27CE010E94462838C060FF7C
:107A600002C080E001C083E00E94C70D30C0112336
:107A700011F4812F18C0C0E0C11748F560E08C2FC9
:107A80000E94395A682F802F0E94421961E08C2F82
:107A90000E94395A682F802F0E944219CF5FECCF85
:107AA000112321F481E00E945A5A11C0115060E064
:107AB000812F0E94395A682F802F0E94421961E05D
:107AC000812F0E94395A682F802F0E94421981E02D
:107AD00090E0DF91CF911F910F91FF90EF90DF9099
:107AE00008959B012F5F3F4F42E0B9010E944C3C3B
:107AF0008FEF90E008959B012F5F3F4F41E0B90168
:107B00000E944C3C8FEF90E008958230C0F4282F03
:107B1000332788E490E0289FF001299FF00D389FDB
:107B2000F00D1124E956FC4FEC5BFF4F10823396A9
:107B300010828FEF9FEF929382930E944F6408957B
:107B400008952F923F924F925F926F927F928F9201
:107B50009F92AF92BF92CF92DF92EF92FF920F93DC
:107B60001F93CF93DF93CDB7DEB725970FB6F89469
:107B7000DEBF0FBECDBF8B83B62E823008F0DFC1D3
:107B800088E49B81989F8001112409561C4FB4E41E
:107B9000CB2ED12CC00ED11ED6018C918823B1F0F2
:107BA000F80180819181A281B38188539F4FAF4FAB
:107BB000BF4FBC01CD010E942214882339F0C801B7
:107BC0000E94802E882311F4D6018C938091B806F0
:107BD0009091B906A091BA06B091BB06F8018083D6
:107BE0009183A283B383D6018C91803408F01C92D8
:107BF000C8010E949E2E882391F0B8E0BB1641F484
:107C0000F6018081882309F49AC18150808397C14D
:107C1000BB2009F494C1FDE0BF1609F4BB24D601D2
:107C2000FC90F801EF0DF11DB482F394FC92C801B1
:107C30000E94802EA82E882309F476C1C8010E94D4
:107C40009E2E882309F43CC1BB2009F078C1F601BF
:107C5000B08286E491E08C839D83A4E04A2E512C6F
:107C6000400E511E095B1F4FD8018C9107541040E4
:107C7000882329F4F5E04F2E512C400E511EF201BD
:107C80008081882309F416C143E050E06FEE76E06E
:107C9000C2010E941365892B19F4C201039601C029
:107CA000C2010E94716649825A82EE2486E9E7E2A7
:107CB000F4E011928A95E9F705C00894211C311C63
:107CC00029823A8229803A80D1019C91992391F0AE
:107CD0009C3281F0943271F0953261F0892F80539B
:107CE0008A3040F0892F992787FD90950E941F6A5E
:107CF000892B19F3F1018081882309F4A8C004C0FD
:107D00000F5F1F4F09831A8309811A81D801FC90E4
:107D10008F2D992787FD90950E941F6A892B81F7E7
:107D2000FF2009F496C0BCE2FB1609F482C08FE084
:107D3000E89E60011124E7E2F4E0CE0EDF1E480168
:107D4000E2E0AE2EB12CAC0CBD1C6624772409C039
:107D50000894811C911CD501FD925D010894611C61
:107D6000711CBBE06B1671047CF4F401F080FF2001
:107D700059F0FCE2FF1641F08F2D992787FD909571
:107D80000E941F6A892B21F3D5011C92F801808182
:107D9000843239F4C801019689839A8340E150E026
:107DA00008C0853251F4C801019689839A8342E064
:107DB00050E0BE016F5F7F4F06C04AE050E0BE0159
:107DC0006F5F7F4FC8010E942165DC01CB01F60186
:107DD0008083918381E0F601868704C00F5F1F4F87
:107DE00009831A8309811A81D801FC90FF2081F050
:107DF0008F2D992787FD90950E941F6A892B41F44A
:107E0000BCE2FB1659F704C00F5F1F4F09831A83AA
:107E100009811A81F801F080FF2041F08F2D992708
:107E200087FD90950E941F6A892B71F7FCE2FF166F
:107E300021F40F5F1F4F09831A83E394E981FA81CC
:107E40008081882321F089E08E1508F05DCFD10173
:107E50001C924E2D5527142F809146019091470179
:107E6000892BD1F0EC81FD8160817181C2010E947A
:107E7000F464892B41F4EC81FD8122813381211549
:107E8000310581F417C08C819D8104968C839D837C
:107E9000DC018D919C91E4CF63EF76E08B810E94B1
:107EA000721908C0412FB2018B81F901099588230D
:107EB00009F445C063E077E08B810E9472193FC0EE
:107EC000EEEAF1E0A8014C5F5F4F2F2D095B1F4FD9
:107ED000D8018C9107541040882321F4A8014B5FEE
:107EE0005F4F21508091AE01882349F19081DA01E2
:107EF0008C919817A1F48181281708F10280F381F1
:107F0000E02D309749F0BA018B810995682F8F3F9A
:107F100019F08B810E944219F601108210C034962C
:107F20008081882319F70BC00C5F1F4F4F2DB801BC
:107F30008B810E944C3C882311F0D601AC9225968F
:107F40000FB6F894DEBF0FBECDBFDF91CF911F916A
:107F50000F91FF90EF90DF90CF90BF90AF909F90E8
:107F60008F907F906F905F904F903F902F900895EB
:107F7000FB0121E057FF04C020E0509541955F4F81
:107F80008330910549F18430910534F481309105B5
:107F900091F0029729F12AC08430910519F00597D4
:107FA00061F024C081818F5F8183992784179507B1
:107FB000ECF0222359F0118219C081818150818314
:107FC00099278417950794F0222321F0842F81505C
:107FD00081830CC021830AC012821382168A06C0D4
:107FE00090E08281882309F491E0928380E090E020
:107FF00008950F931F93CF93DF938C010E94CD2898
:10800000EC01009731F461EF7FE082E00E94721989
:108010000FC09F938F9387EF9FE09F938F9382E092
:108020008F930E94C8190F900F900F900F900F9090
:108030000115110521F0B80182E00E947219CE01EC
:10804000DF91CF911F910F9108950F931F93CF93BD
:10805000DF93EC018B01009731F097FD35C002975B
:10806000029790F52BC060E081E00E94EA17F801CA
:108070008281882359F46BEF7FE082E00E947219BD
:1080800064E070E182E00E94721918C00E94F8500A
:10809000DC01CB01BF93AF939F938F938AE090E174
:1080A0009F938F9382E08F930E94C8198DB79EB7DC
:1080B00007960FB6F8949EBF0FBE8DBF40E050E00C
:1080C000B801CE010E94B83F80E090E0DF91CF91EF
:1080D0001F910F9108958230910541F083309105F1
:1080E00041F440E050E00E94B83F03C08FEF9FEFA3
:1080F000089580E090E008950895CF92DF92EF9286
:10810000FF920F931F93CF93DF93EC017B010E94AB
:10811000CA288C01C230D10509F453C0C330D1053F
:108120002CF42097D1F0219731F090C0C630D105C2
:108130000CF08CC02AC0FC016785262F2695269559
:108140002370637009F461E083E0689FC00111242B
:10815000280F2350F701218379C060E081E00E945D
:10816000EA1786E190E10E94F93F892B09F46EC07D
:10817000F70191818AE0989FC0011124895A984F94
:10818000BC0182E00E94721961C049E050E0B70171
:10819000CE010E94B83FF801808191818F3F910507
:1081A00009F008F453C0F7018181882311F486E0B7
:1081B0008183F7018181863008F048C088E081839F
:1081C00045C0FC0182819381892B09F03FC0F701F2
:1081D0008281882399F1F801C081D1812097B1F182
:1081E000F7013181832F63E00E94E269282F2F5F1E
:1081F000832F0E94E269892F9927880F991F880F82
:10820000991F282BF801C288D388622FCE010E94C3
:108210006B26CE010E944D260E94CF29C114D104A5
:1082200069F0C80144969C01F8014785608171811D
:10823000C6010E94295CF801828B938B90E0F701C4
:108240008281882309F491E0F701928380E090E035
:10825000DF91CF911F910F91FF90EF90DF90CF9022
:108260000895482F30E0832F992787FD9095FC01D2
:10827000EA5DF84F2491241729F03F5F222399F7F4
:108280008FEF9FEF08950895EF92FF920F931F9342
:10829000CF93DF93EB018230910509F486C08330E0
:1082A000910534F4009709F43EC0019769F0BAC013
:1082B0008430910509F443C0843091050CF470C0FA
:1082C000059709F456C0AEC00E94CA288C01FC0173
:1082D00080819181892B09F4A5C044E1E42EF12C21
:1082E000E00EF11E8E01065F1F4F65960C171D07ED
:1082F000B8F4F7018081882339F00E94314187FD6D
:1083000003C0F701808101C080E2F80181938F01F1
:10831000F7018081882351F30894E11CF11CE6CF1A
:10832000F80110827FC00E94F93F60E081E00E9466
:10833000EA172A96BE0182E00E94881973C08981DB
:10834000FB01E80FF11DEF012A9682850E94314161
:108350008F5FE82FFF27E7FDF095EA5DF84F8491E6
:10836000882319F4E6E2F7E08491992787FD909538
:1083700015C08981FB01E80FF11DEF012A96828566
:108380000E943141181614F08FE201C08150E82F8D
:10839000FF27E7FDF095EA5DF84F8491888342C09E
:1083A00049E050E00E94B83F3DC00E94CA288C01BD
:1083B000FC0182819381892BA9F59A81992349F443
:1083C00089E08B8381E0888F99839F8B8A838E8B52
:1083D00029C089818F5F89838F8B8B3018F11B8235
:1083E0001A821E8A8CE098012C5E3F4FD901FE0153
:1083F0003A9601900D928A95E1F7F8018289938966
:10840000009731F04785608171810E94295C07C027
:10841000A901F8016785808191810E94E15CF801E2
:10842000828B938B80E090E0DF91CF911F910F9131
:10843000FF90EF900895AF92BF92CF92DF92EF92AC
:10844000FF920F931F93CF93DF93CDB7DEB72197A2
:108450000FB6F894DEBF0FBECDBF9C018B018230FA
:10846000910509F455C0833091052CF40097C1F0B3
:10847000019759F0A3C084309105D9F1843091055A
:108480000CF441C00597C9F199C04BE050E060E29F
:1084900070E0C8010A960E94BC64F801158A8EC07B
:1084A000FB018281882309F489C08181882309F432
:1084B00085C0065F1F4FA801B90199270E94E95C9A
:1084C0009F938F9389E190E19F938F9362E0F62EC3
:1084D000FF920E94C81960E081E00E94EA17B8018B
:1084E0008F2D0E9488190F900F900F900F900F9072
:1084F00065C0FB018181992721C0FB0181819927FA
:108500000E945E5D1DC049E050E00E94B83F56C029
:1085100090E0FB018281882309F491E0F8019283C5
:108520000E94CA287C01F8018281882361F0F7014A
:1085300082899389009711F0828902C00E94295D87
:10854000F80181833BC05AE0A52EB12CA00EB11ECC
:10855000F8018181A501BE016F5F7F4F99270E94BD
:10856000E95C6C01F7011282138210821182BC0156
:108570008FEF0E942652F70180819181892B59F05B
:108580006981C6010E946B26C6010E944D260E9489
:10859000CF290E94DC28F70180819181892B59F035
:1085A000B501C70144960E94FE64F80181819927B4
:1085B000F701828B938B8FEF9FEF02C080E090E0FA
:1085C00021960FB6F894DEBF0FBECDBFDF91CF91DD
:1085D0001F910F91FF90EF90DF90CF90BF90AF90E1
:1085E00008950F931F93CF93DF93EC010E94CA2845
:1085F0008C01209719F02297C9F03DC0CE010E944E
:10860000F93F892BC1F160E081E00E94EA17F8018F
:1086100082899389892B11F081E001C082E00E9458
:10862000A94FBC0182E00E94721925C0FC01C281E1
:10863000D381209701F580819181892BE1F0828996
:108640009389892BC1F060E081E00E94EA1783E002
:108650000E94A94FBC0182E00E94721984EF91E050
:108660000E945916F801828993890E94265CF801BC
:10867000C28BD38B148A80E090E0DF91CF911F9161
:108680000F9108951F93CF93DF93EB0182309105F3
:1086900009F440C0833091052CF4009789F00197CC
:1086A00031F04CC0863091050CF048C02EC00E94BD
:1086B000BB50FC01848163E00E94E26989833EC073
:1086C00060E081E00E94EA17898113E0819F802D9C
:1086D00011240E943D1982E090E00E94591681B752
:1086E000612F0E94E269898399279F938F938DE17F
:1086F00090E19F938F9382E08F930E94C8190F900F
:108700000F900F900F900F9019C04FEE5FEF0E94E7
:10871000B83F14C08A81882359F00E94BB50398128
:1087200023E0329F90011124FC0124830E944250D7
:1087300090E08A81882309F491E09A8380E090E0B8
:10874000DF91CF911F9108951F93CF93DF93EC0199
:108750008A81882309F45CC060E081E00E94EA1706
:108760008C819D819F938F9381E290E19F938F9362
:1087700012E01F930E94C8198B810F900F900F90E9
:108780000F900F90843059F487E290E19F938F937C
:108790001F930E94C8190F900F900F9010C08885EA
:1087A00099279F938F938BE290E19F938F931F93D1
:1087B0000E94C8190F900F900F900F900F90898D05
:1087C0009A8D97FD03C06FE270E10AC08E5F9F4FE4
:1087D00019F467E370E104C084E00E94A94FBC0172
:1087E00082E00E94721981E0888F8E8B8B8199279D
:1087F0008130910564F08330910524F0049702974D
:1088000030F402C083E001C088E08F8B01C01E8A73
:10881000DF91CF911F9108950F931F93CF93DF9313
:108820008C01FC018281882311F581E0838364300F
:1088300019F488E090E003C080E094E0F8018683BA
:108840009783F80124813581868197818217930768
:1088500024F481E090E08483958381E0F8018283B1
:10886000683009F410C180E00E94C70D0CC1F80106
:10887000848195819093C7048093C604C62FDD2719
:10888000C430D10561F1C530D10594F4C130D105B2
:1088900009F4C2C0C230D1051CF4209701F1F3C025
:1088A000C230D10509F4BAC0239709F4E9C0EBC07E
:1088B000C730D10509F4B0C0C830D10544F4C53083
:1088C000D10509F4A9C0C630D10549F0DCC0C830D3
:1088D000D10509F47EC0299709F49EC0D4C0F801DF
:1088E000838181508230E0F58EEF9FEF818F928FF0
:1088F000C8010E94A4436AE081E00E94EA1789E06F
:108900000E94A94FBC0182E00E947219C430D105B7
:1089100081F0C530D1051CF4CD2B21F019C026976C
:1089200071F016C0F8018481958101970E94FA596F
:108930000CC0F801848181500E941A5A06C0F801C7
:108940008481958101970E942F5AF801818F928F1F
:10895000F801818D928D97FD5DC0818D80875AC011
:108960006AE081E00E94EA178AE00E94A94FBC01F8
:1089700082E00E947219C430D10589F0C530D1055A
:108980001CF4CD2B21F046C02697C1F043C0F8015E
:1089900084819581608501970E94F05916C0F80185
:1089A0008481958109971CF08FEF9FEF0FC0F8012C
:1089B0008481608581500E940F5A07C0F80184812C
:1089C0009581608501970E94255AF801818F928FC9
:1089D00021C00E94CA28FC01208131812115310566
:1089E000C9F08785992783709070039799F4F801EF
:1089F000648175816115710569F0838181508230D0
:108A000048F0615070404085C9010E94AE28F801CD
:108A1000138239C081E035C084E033C0F80183811E
:108A20008150823010F481E02DC06AE081E00E9424
:108A3000EA17F8018381863079F489E00E94A94F12
:108A4000BC0182E00E947219F801848195816185E0
:108A500001970E94E6590FC08AE00E94A94FBC010D
:108A600082E00E947219F80184819581418D6185AF
:108A700001970E94DC59F801818F928F86E001C036
:108A800087E0F8018383DF91CF911F910F910895C3
:108A90009C01FB018130910561F0823091051CF44D
:108AA000892BD1F024C083309105E9F00597C1F0FE
:108AB0001EC08EEF9FEF818F928F4091C604509120
:108AC000C704CA0101978050944018F44483558329
:108AD0000EC0248335830BC0CB010E94A44307C082
:108AE00081E0838304C040E050E00E94B83F80E012
:108AF00090E008950F931F93CF93DF938C01EB01C8
:108B00000E94CA28FC0180819181892B31F08785E0
:108B1000992783709070039761F060E081E00E9474
:108B2000EA1785E00E94A94FBC0182E00E947219F9
:108B30001BC00230110541F00430110589F469E0D1
:108B4000CE010E940C4410C068E0CE010E940C448B
:108B50008B81882349F40E94F9178FEF9FEF06C09D
:108B6000BE01C8010E94484580E090E0DF91CF91AE
:108B70001F910F910895CF93DF93EB018230910500
:108B800009F481C08330910534F40097A1F081305D
:108B9000910569F07CC08430910509F462C084308D
:108BA00091050CF46BC0059709F460C070C00E9479
:108BB000484519866CC08A81882309F468C060E042
:108BC00081E00E94EA178B81882331F46FE370E122
:108BD00082E00E94721918C0898599279F938F930C
:108BE0008C819D819F938F938FE490E19F938F93CE
:108BF00082E08F930E94C8198DB79EB707960FB673
:108C0000F8949EBF0FBE8DBF898D9A8D97FD0BC0C6
:108C1000823091051CF0029721F005C0898D805D9E
:108C200003C08FE301C085E40E94B21781E0888F02
:108C30008E8B8B8199278630910561F08730910565
:108C400024F40197029758F403C0079729F007C04E
:108C500086E003C08CE001C08EE08F8B18C01E8AB6
:108C600016C08B81863039F463E00EC08B8186306C
:108C700011F481E001C086E08B8309C040E050E040
:108C80000E94B83F04C062E0CE010E940C4480E024
:108C900090E0DF91CF9108959B018230910529F0FA
:108CA0008430910539F461E001C060E0C9010E949F
:108CB0000C4402C00E94484580E090E008959B016A
:108CC0008230910529F08430910539F465E001C0C6
:108CD00064E0C9010E940C4402C00E94484580E043
:108CE00090E008959B018230910529F08430910530
:108CF00039F467E001C066E0C9010E940C4402C07B
:108D00000E94484580E090E008951F93182F60E08E
:108D100081E00E94EA17812F99278130910571F037
:108D2000823091051CF4892B39F013C082309105F3
:108D300039F0039739F00DC08BE005C08CE003C01B
:108D40008DE001C08EE00E94A94FBC0182E00E942C
:108D500072191F910895CF93C82F1816B4F480E0AC
:108D60000E9485466C2F80E090E00E94F059892B8C
:108D700039F440E065E08CE190E00E94DC5907C0E6
:108D80008C2F0E94045A892B11F082E001C083E0ED
:108D90000E94854684EF91E00E945916CF91089574
:108DA000CF93DF93EB0182309105E1F183309105A0
:108DB0001CF4892B29F04EC08330910571F14AC013
:108DC0008A81882309F446C060E081E00E94EA17A6
:108DD0008C819D8197FF0CC08EE590E19F938F93CE
:108DE00082E08F930E94C8190F900F900F900FC0D0
:108DF0009F938F9383E690E19F938F9382E08F936D
:108E00000E94C8190F900F900F900F900F9083E061
:108E10008F8B81E0888F8E8B1DC040E050E00E94D8
:108E2000B83F18C08A81882321F08C810E94AB460C
:108E300005C081E00E94854681E08A8380E090E061
:108E40000E94FA598C839D8381E08B838FE790E0A9
:108E50008E839F8380E090E0DF91CF9108950F9300
:108E60001F93CF93DF938B018130910571F0823096
:108E700091051CF4892B79F0B4C08230910509F476
:108E80003FC083309105B9F1ACC08FEF9FEFFB017C
:108E900084839583A6C0FB018281882309F4A1C045
:108EA00060E081E00E94EA17F8018481958197FFD4
:108EB0000CC087E690E19F938F9382E08F930E948E
:108EC000C8190F900F900F900FC09F938F938EE64D
:108ED00090E19F938F9382E08F930E94C8190F9027
:108EE0000F900F900F900F9085E0F801878B81E035
:108EF000808F868B76C040E050E00E94B83F71C002
:108F0000FB018281882389F1C481D581C038D105D4
:108F100020F48C2F0E94AB462EC0F8E2C030DF0751
:108F2000A0F480E00E9485468D2F9927806C682FE1
:108F300080E190E00E94F059009729F46C2F81E1C4
:108F400090E00E94F059892B11F082E007C041E0C7
:108F500065E08CE190E00E94DC5983E00E94854648
:108F600084EF91E00E94591606C081E00E94854678
:108F700081E0F8018283F8018481958101978F3720
:108F8000910540F480E090E00E94FA59F801848352
:108F9000958315C080E190E00E94FA59982F8827A8
:108FA000F8018483958381E190E00E94FA59F801E9
:108FB00024813581282B392B3F7324833583F80195
:108FC00084819581805098422CF08FEF9FEFF801BB
:108FD0008483958381E0F80183838FEF97E2868312
:108FE000978380E090E0DF91CF911F910F910895DA
:108FF0001F93CF93DF93EB01122F8230910519F16C
:10900000833091052CF4009761F0019729F02EC070
:10901000863091055CF512C0842F0E94DC50898354
:1090200025C060E081E00E94EA178981810F0E94DB
:109030000150BC0182E00E94721918C042E050E069
:109040000E94B83F13C08A81882351F08981882308
:1090500021F0842F0E94E65003C0842F0E94EE501E
:1090600090E08A81882309F491E09A8380E090E07F
:10907000DF91CF911F91089522E0422F0E94F8477F
:10908000089522E048E00E94F847089520E041E07A
:109090000E94F84708950F931F93CF93DF938C019D
:1090A000EB0124E0422F0E94F8470230110529F419
:1090B0008A81882311F40E94361E80E090E0DF91BF
:1090C000CF911F910F910895FF920F931F93CF930C
:1090D000DF93EC018B01F42E0E94BB50FC01C230E7
:1090E000D10509F471C0C330D1052CF42097C9F023
:1090F000219771F07DC0C430D10509F44DC0C43052
:10910000D1050CF44DC0C530D10509F449C070C07B
:10911000FF2019F08485E80155C08385F80181831B
:1091200067C060E081E00E94EA17E8019981FF20B2
:10913000F9F0892F6AE00E94E269892F99279F93AD
:109140008F9389810E94E26999279F938F9382E789
:1091500090E19F938F9382E08F930E94C819EDB79F
:10916000FEB737960FB6F894FEBF0FBEEDBF40C0F6
:1091700082E3989FC00111249F938F938AE790E127
:109180009F938F9382E08F930E94C8190F900F9046
:109190000F900F900F902CC0F80181818F3F41F10B
:1091A000FF2019F040E05FEF02C04BEE5FEFB80127
:1091B000CE010E94B83FFF20D9F0E80189818823C1
:1091C000B9F481E0898314C0E8018A81882341F0E1
:1091D0009981FF2011F0948701C093870E9442502B
:1091E00090E0F8018281882309F491E0E8019A83F4
:1091F00080E090E0DF91CF911F910F91FF90089553
:1092000040E00E946448089541E00E946448089547
:10921000CF93DF93EB018230910559F183309105B3
:109220002CF4009759F0019729F02FC08630910552
:1092300064F51AC00E94C350898327C060E081E0B2
:109240000E94EA1789819927880F991F880F991F13
:109250008A5F984FBC0182E00E94721960E870E159
:1092600082E00E94721911C048E050E00E94B83FAD
:109270000CC08A81882319F089810E94C75090E030
:109280008A81882309F491E09A8380E090E0DF915D
:10929000CF910895CF93DF93EB0182309105C1F117
:1092A0008330910534F4009749F08130910551F1F4
:1092B00057C0863091050CF053C024C08A818823A2
:1092C00009F44EC061E080E00E94EA1789818A5F5C
:1092D0000E940150BC0182E00E94721960E081E0AE
:1092E0000E94EA176981623020F082E10E94A94F52
:1092F00004C0862F865F0E940150BC0182E00E945C
:1093000072192EC042E050E0BE010E94B83F28C052
:109310008A81882319F18981823018F48E5F8983CC
:109320001FC060E081E00E94EA178981833051F418
:109330008FE00E94A94FBC0182E00E9472190E9436
:10934000A15E09C080E10E94A94FBC0182E00E9499
:1093500072190E94695F8FEF9FEF04C081E08A83DA
:1093600080E090E0DF91CF910895CF938091BD048C
:10937000803178F01092BD041092BE0461E0862F17
:109380000E94EA17CEE085EA0E94B217C150C7FFDB
:10939000FACF6091BD0481E00E94EA178091BE047B
:1093A00099278130910559F0823091051CF4892B61
:1093B00021F014C0029739F011C085E001C084E0AB
:1093C0000E94B2170BC080E20E94B21785E00E9493
:1093D000B2178091BD048F5F8093BD048091BE045D
:1093E0008F5F8093BE04833010F01092BE04CF9143
:1093F0000895CF93DF93EB018230910559F18330CB
:1094000091051CF4892B31F053C0863091050CF086
:109410004FC01BC08A81882309F44AC061E080E004
:109420000E94EA1789E10E94A94FBC0182E00E94D4
:10943000721960E081E00E94EA1781E10E94A94F61
:10944000BC0182E00E94721933C040E050E00E94EB
:10945000B83F2EC08A81882329F10E94F41D64E957
:1094600071E084E00E9419196CE871E085E00E94C7
:10947000191968EC70E085EB99E40E94231860E00C
:10948000862F0E94EA1783E00E94A94FBC0182E068
:109490000E9472190E94D9240E94875D0E94645024
:1094A0000E94B65290E08A81882309F491E09A8361
:1094B00080E090E0DF91CF910895CF92DF92EF921C
:1094C000FF920F931F93CF93DF93029709F0CEC0C3
:1094D00060E0862F0E94EA1780E20E94B21760E0E7
:1094E00081E00E94EA1780E00E94C70D68E870E101
:1094F00082E00E94721921E04EE468E086E00E945A
:10950000380F6D9880E00E94411180E00E94DB12CC
:10951000CC24DD248EEF0E944A1380E00E94F419CF
:109520008F5F9F4FD1F781E00E94F4198F5F9F4FAB
:10953000D1F7A8950E9497178331910509F488C047
:109540008B30910509F484C00A9701F581C0CF3FA3
:10955000D10551F0209741F06C2F80E00E94421914
:109560006C2F81E00E944219CF33D10519F0CB3224
:10957000D10519F4B4E8CB2ED12CC332D10511F0AA
:10958000AA9721F4A6E0CA2EA1E0DA2E0E94771352
:10959000EC018F5F9F4FD9F6C114D10409F4BACF03
:1095A000E090B806F090B9060091BA061091BB069B
:1095B00088EC90E0A0E0B0E0E80EF91E0A1F1B1F47
:1095C0003BC0A8950E94F419EC019FEFCF3FD9074B
:1095D00021F481E00E94F419EC01AFEFCF3FDA07EC
:1095E00021F18C2F0E944A130894C108D108E09001
:1095F000B806F090B9060091BA061091BB0688EC47
:1096000090E0A0E0B0E0E80EF91E0A1F1B1F0DC09D
:10961000CF3FD10551F0209741F06C2F80E00E94A0
:1096200042196C2F81E00E9442190E947713EC01CD
:109630009FEFCF3FD90761F7C114D10409F468CF78
:10964000C801B7010E942214882309F4BACF60CF61
:1096500081E00E94411181E00E94DB126D9A0E941C
:10966000C35021E04EE468E00E94380F80E090E0B3
:10967000DF91CF911F910F91FF90EF90DF90CF90EE
:109680000895CF93DF93EB018230910509F440C038
:10969000833091052CF4009771F0019731F048C0A8
:1096A000863091050CF044C02EC00E94BB50FC01D6
:1096B000868189833DC060E081E00E94EA1769816C
:1096C000662369F484E10E94A94F9F938F9382E0FF
:1096D0008F930E94C8190F900F900F9029C085E0BA
:1096E000689FC00111249F938F9385E990E19F9318
:1096F0008F9382E08F930E94C8190F900F900F9064
:109700000F900F9015C049EC50E00E94B83F10C078
:109710008A81882339F00E94BB502981FC0126836D
:109720000E94425090E08A81882309F491E09A8354
:1097300080E090E0DF91CF910895CF93DF93EB012C
:109740008130910569F0823091051CF4892B81F0FC
:1097500049C08230910539F183309105F9F042C05A
:109760000E94BB50FC01808599278C839D833AC061
:1097700060E081E00E94EA178C819D819F938F9326
:109780008BE990E19F938F9382E08F930E94C81999
:109790000F900F900F900F900F9024C040E050E07A
:1097A0000E94B83F1FC08A81882361F483E08B83C5
:1097B00080E290E08E839F8391E0988F82E08F8B90
:1097C0009E8B0AC01E8A0E94BB502C81FC01208700
:1097D00020934F0A0E94425090E08A81882309F426
:1097E00091E09A8380E090E0DF91CF910895EF922D
:1097F000FF920F931F93CF93DF938C01EB010E9495
:10980000BB507C010230110509F463C0033011051F
:1098100044F40115110571F00130110509F446C039
:1098200072C00330110509F43DC0063011050CF07B
:109830006AC03CC08A81882309F465C0F70180852D
:10984000882309F460C060E081E00E94EA178C81FF
:109850009D819F938F9380EA90E19F938F9382E005
:109860008F930E94C81960E089810E94395A082F9D
:1098700061E089810E94395A182FC0E80F900F903B
:109880000F900F900F9094E0802F8C2309F096E0BA
:10989000812F8C2309F09F5F892F0E94B217C695F4
:1098A00091F731C01E8A81E00E945A5AF7018085E3
:1098B0009927AC01BE01C8010E94B83F8981992750
:1098C00001968C839D838B818230E9F488E08B83C1
:1098D0001AC02A81222391F481E090E08C839D8339
:1098E000F701808599278E839F8311E01A83822F49
:1098F0000E945A5A188F85E08F8B1E8B88E08B83CD
:109900008C818150898380E090E0DF91CF911F911D
:109910000F91FF90EF900895CF92DF92EF92FF9218
:109920000F931F93CF93DF937C01C62F0E941119D1
:109930000E94BB506C01C23208F06FC085E0C89F26
:10994000800111240E5D1D4FF7018281882311F0E3
:1099500080E001C082E00E94B217F601858199275C
:1099600081309105B1F0823091051CF4892B39F0DA
:1099700031C082309105B9F00397F9F02BC08C2FDC
:10998000992744E0880F991F4A95E1F78F51924F2C
:109990001DC08C2F992734E0880F991F3A95E1F765
:1099A0008F52944F13C08C2F992724E0880F991F52
:1099B0002A95E1F78F53964F09C08C2F9927C4E061
:1099C000880F991FCA95E1F78F54984FBC0182E028
:1099D0000E947219E8018C8187FD0BC060E081E074
:1099E0000E94EA178C810E94A94FBC0182E00E946C
:1099F0007219E801EA81FB81309721F0B70180E01C
:109A000090E00995F7018689882329F06789808D80
:109A10000E94F31702C00E94F917DF91CF911F91A6
:109A20000F91FF90EF90DF90CF90089560E0E2E219
:109A3000F2E0482F552747FD509520E030E0808127
:109A400099278417950711F4C90108956F5F2F5F57
:109A50003F4F3596613298F38FEF9FEF0895089549
:109A6000BF92CF92DF92EF92FF920F931F93CF930B
:109A7000DF93CDB7DEB76B970FB6F894DEBF0FBE9E
:109A8000CDBFB82E20E2281718F480E090E0F7C18F
:109A90006E010894C11CD11C8BE1F60111928A95CC
:109AA000E9F7A89585E0B89EF0011124EE5DFD4F21
:109AB0000280F381E02D309721F0B60181E090E043
:109AC00009956B2DC6010E948C4C0E940A0E85E000
:109AD000B89E7001112482E292E0E80EF91E0E9405
:109AE0009717AC018A30910509F4E5C08B309105D8
:109AF00064F4009709F406C1181619060CF41AC18B
:109B00004F5F5F4F09F4AAC1E0CF8331910509F49B
:109B10008AC08431910544F48B30910509F483C0E7
:109B2000419709F497C1D1CF8431910519F0459738
:109B300041F1CBCFF6018281882381F0F7012281A8
:109B400033812115310531F0BE016F5F7F4F84E015
:109B500090E07DC1F60181818F5F26C0F701908181
:109B6000FFE1FB1534F0F7018581891711F4B394F7
:109B70002FC0892F0E94164D682F772767FD70959B
:109B80003EC0F6018281882389F0F701228133816A
:109B90002115310531F0BE016F5F7F4F85E090E008
:109BA00056C1F60181818150818365C16B2DF7011A
:109BB0009081BB2091F02BEF3FEFE20EF31EF701F7
:109BC000808125E030E0E20EF31E891731F4BA946B
:109BD0006B2D772767FD709512C03FE13B1564F050
:109BE000D7011596F7018581891731F46F5F6032CF
:109BF0001CF415968C91F8CF772767FD7095B62EDB
:109C000085E0689FF0011124EE5DFD4F0280F38135
:109C1000E02D309709F42FC1BE016F5F7F4F81E0C7
:109C200090E0099528C1F7019181992361F1092FED
:109C3000112701541B4FF801808118162CF0892F31
:109C40000E94164DF8018083F7018181E82FFF27DC
:109C5000E154FB4F80810E94304D282F332727FD90
:109C60003095F7018181E82FFF27E154FB4FC901AF
:109C700037FF04C088279927821B930B808337FF07
:109C8000FAC0B1943AC0F701228133812115310520
:109C900051F0BE016F5F7F4F82E090E0F9010995BE
:109CA00099237CF319C0F6018281882309F491E09D
:109CB000F6019283E0C0F60182818823F1F0F7017A
:109CC0002281338121153105A9F0BE016F5F7F4FDD
:109CD00083E090E0F9010995F6018281882309F07B
:109CE000CAC0F70122813381BE016F5F7F4F81E0DF
:109CF00090E0ADC0F6011282BEC08B2D992787FD82
:109D00009095BDC0F6018381813009F4DECE8830A4
:109D100089F481E00E945A5A60E0F60181810E9434
:109D2000395A61E0F60181810E94395A80E00E942F
:109D30005A5AA1C0F601838199278530910509F40B
:109D400054C08630910584F48230910581F18330CE
:109D500091051CF40197B9F08EC08330910599F0FC
:109D6000049709F43EC087C08730910509F456C0B6
:109D7000873091050CF44CC08830910521F009978B
:109D800009F453C078C0F60186819781892B21F4AC
:109D90008FEF9FE786839783F601868197818417EB
:109DA00095070CF468C01482158282E08383F60163
:109DB000848195819C0163E0220F331F6A95E1F74E
:109DC000280F391F280F391F240F351F37FD53C0A7
:109DD00086819781821793070CF44DC024833583C5
:109DE0004AC0F601108685E08383F60190858AE0FB
:109DF000989F90011124240F351F2F3F310509F042
:109E000008F420878EEF9FEFF601818F928F33C089
:109E10004830510584F5F60141872DC04230510587
:109E200054F5F601418F528F26C0F6018181E80F6B
:109E3000F11D842F805D8287F701228133812115F6
:109E40003105C9F0BE016F5F7F4F82E090E0F901FC
:109E5000099511C080E00E94C70D0DC0F6018381F5
:109E6000883009F032CEBE016F5F7F4F80E090E016
:109E70000E94F74B2ACE6B2DCE01019624CE6B9615
:109E80000FB6F894DEBF0FBECDBFDF91CF911F910B
:109E90000F91FF90EF90DF90CF90BF900895CF93F8
:109EA000C82F6CE571E080E00E94191964E671E04A
:109EB00082E00E94191964E871E084E00E94191997
:109EC0006CE771E085E00E94191964E771E086E0B3
:109ED0000E9419196CE671E087E00E9419198091BF
:109EE000BF04813210F01092BF04C7FD04C08C2F54
:109EF0000E94304D0EC08091BF040E94304D9927C2
:109F000087FD909597FF03C0909581959F4F809313
:109F1000BF046CE372E080E00E9419196CE172E00A
:109F200082E00E94191964EF71E084E00E9419191F
:109F30006CEE71E085E00E94191964EE71E086E034
:109F40000E9419196CED71E087E00E941919CF91F8
:109F50000895CF93C82F8B3118F08AE19BE12CC074
:109F60000E94BB50FC01858199278230910581F0C8
:109F7000833091051CF4019721F018C0039779F004
:109F800015C081E1C89FC0011124815B964E14C0A9
:109F900081E1C89FC00111248C57984E0DC081E10A
:109FA000C89FC001112487549A4E06C081E1C89F02
:109FB000C001112482519C4ECF910895882319F03D
:109FC00087E29BE108950E94BB50FC01858199279F
:109FD0008230910561F0833091051CF4019721F0E6
:109FE0000CC0039739F009C08DED93E108958CEC16
:109FF00093E108958BEB93E108958AEA93E1089544
:10A000000895CF93C82F8C3018F087E39BE138C0B8
:10A010000E94BB50FC01858199278230910599F0FF
:10A02000833091051CF4019721F021C00397A9F01A
:10A030001EC08C2F992754E0880F991F5A95E1F77D
:10A0400086519D4E1DC08C2F992744E0880F991F83
:10A050004A95E1F7865D9D4E13C08C2F992734E019
:10A06000880F991F3A95E1F786599E4E09C08C2FAB
:10A07000992724E0880F991F2A95E1F786559F4E6E
:10A08000CF910895EF92FF921F93CF93DF9388ECC7
:10A09000E82E84E0F82EC0E0D0E01FE1CE010E945F
:10A0A0008364F70161917F01861719F0CE010E9448
:10A0B0009C64A8951150219617FFF0CFDF91CF91A6
:10A0C0001F91FF90EF9008959091CD04943008F087
:10A0D00091E08FE0E8ECF4E011928A95E9F788E1ED
:10A0E0008093CC049093CD0481E08093C90484E1F3
:10A0F0008093CE0482E08093D30482E38093D404DF
:10A100000E944250089540E250E060E070E088EC28
:10A1100094E00E948B648091CA049091CB048F5F7D
:10A120009F4F11F40E9464508091C904883018F048
:10A1300081E08093C9048091D5049091D604885F12
:10A14000974020F01092D6041092D5048091CD044F
:10A15000843010F01092CD048AEF9FEFA1E0B0E0C0
:10A16000ABBFFC0187918F3F21F0882311F08093D2
:10A170006F000895089588EC94E008958093CD04CD
:10A180000E94425008958091C90499270895CF9361
:10A19000C82F883008F0C7E08091C904C81751F073
:10A1A000C093C9040E94425021E04EE468E08C2F25
:10A1B0000E94380FCF91089520E030E09091C804BC
:10A1C000982311F021E030E0C90108959091C8046E
:10A1D000982B9093C8040E9442500895982F909510
:10A1E0008091C80489238093C8040E944250089536
:10A1F0008CEF9FEFA1E0B0E0ABBFFC01879197919E
:10A20000A791B691B070BC01CD0108958FEF9FEF7B
:10A21000A1E0B0E0ABBFFC018791992708950E94AF
:10A220000925FC01892BB9F0A8EEB4E043E02D919B
:10A230003C911197808191812817390729F08281FB
:10A2400093812817390719F41D921C9211974150D8
:10A25000139647FFECCF089508959F92AF92BF9257
:10A26000CF92DF92EF92FF920F931F93CF93DF93E2
:10A27000CDB7DEB726970FB6F894DEBF0FBECDBFC1
:10A28000C82E7B01942ECE0101960E94E852DD2457
:10A2900098EEA92E94E0B92EF501808191818E155A
:10A2A0009F0509F08AC082818F5F8283843008F421
:10A2B000B9C0C7010E9431258C01009709F4B4C0D0
:10A2C000FFEFCF1619F5992029F0FC016481758103
:10A2D000C70117C0FC01448155816681C7010E94F6
:10A2E0006E29F80180850E94CF29F801828193812F
:10A2F000009749F00E943125FC01648175818081BD
:10A3000091810E94B8290E94DC2851C0992049F00F
:10A31000FC014481558160E0CE0101960E94CB5240
:10A3200039C0FC01448155816681CE0101960E94AD
:10A33000CB52AE014F5F5F4F67E08C2D0E946B5395
:10A34000F80180858F778B830E9481538823E1F306
:10A35000AE014F5F5F4F69E08C2D0E946B53F80197
:10A36000828193810E9409258C010097D1F0FC0124
:10A3700060817181CE0101960E94E852F80144810A
:10A38000558160E0CE0101960E94CB520E9481531C
:10A390008823E1F3AE014F5F5F4F68E08C2D0E9490
:10A3A0006B5340E050E06DE08C2D0E946B53F50143
:10A3B0001082118281E090E037C0D39483E090E076
:10A3C000A80EB91E93E09D1508F066CFDD2408EEB7
:10A3D00014E0F80180819181892BA1F40E94CD289D
:10A3E0008E159F0519F40E94E22807C0AE014F5F49
:10A3F0005F4F65E08FEF0E946B53F801E082F182BE
:10A40000128206C0D3940D5F1F4FF3E0FD1508F7CD
:10A4100083E08D1538F4AE014F5F5F4F66E08FEF3C
:10A420000E946B5380E090E026960FB6F894DEBF52
:10A430000FBECDBFDF91CF911F910F91FF90EF9095
:10A44000DF90CF90BF90AF909F9008950F931F9390
:10A45000CF93DF93082FEB01672B79F010E040E0FA
:10A46000BE01802F0E942D51882339F40E94815310
:10A470008823E1F31F5F143190F3DF91CF911F9197
:10A480000F9108958F929F92BF92CF92DF92EF9299
:10A49000FF920F931F93CF93DF93CDB7DEB726972D
:10A4A0000FB6F894DEBF0FBECDBFB82E4B016A01C8
:10A4B000CB010E9431258C01892B09F445C0C601CE
:10A4C0000E9431257C01892B09F43EC0F80180856A
:10A4D0000E94C1288C01F70180850E94C128081BB9
:10A4E000190BC80117FF03C0909581959F4F0297E4
:10A4F000E4F0FFEFBF1621F481E00E942E2A24C071
:10A5000086E0FE01319611928A95E9F781E0898310
:10A51000AE014F5F5F4F61E28B2D0E946B5314C001
:10A52000B601C4010E9417280FC010E041E0B60137
:10A530008B2D0E942D51882399F70E9481538823E7
:10A54000E1F31F5F143190F326960FB6F894DEBF47
:10A550000FBECDBFDF91CF911F910F91FF90EF9074
:10A56000DF90CF90BF909F908F9008950E94F41D30
:10A57000F894FFCF682790E027E0862F86959F5FAD
:10A5800060FF03C0682F622701C0682F9830A8F3CE
:10A59000862F99270895FC01262F862F8F77828397
:10A5A00026952074CA01892F9927869586958F73E1
:10A5B000822B8383CA0123E0969587952A95E1F73C
:10A5C0008F778483842F8295807F8F77858308950A
:10A5D000FC01CB01262F2F772083880F892F881F1E
:10A5E000990B91958F7781830895803480F4E82FBB
:10A5F000FF27662329F0E55DFA4F8AE080830895FE
:10A60000E55DFA4F8081882311F0815080830895A1
:10A610000895EF92FF920F931F93CF93DF93782FBC
:10A62000C62F7A01A89580911805282F332780918D
:10A630001905992701972817390741F080911805C6
:10A64000833039F480911905882319F480E090E073
:10A650003BC09091180589E0989F800111240C500F
:10A660001B4F872F8068F8018083682F80E00E944D
:10A67000BA52F801C1836C2F0E94BA52982FE80198
:10A68000229605E0E114F10431F0F70181917F0198
:10A690008F77888301C018826991892F0E94BA52EE
:10A6A000982F015007FFEECF87FD909598838091FA
:10A6B00018058F5F8093180580911805843010F07D
:10A6C0001092180581E090E0DF91CF911F910F91DA
:10A6D000FF90EF9008950F931F93CF93DF93082F70
:10A6E000162FEA0102C00E940A0EAE01612F802FD0
:10A6F0000E9409538823B9F3DF91CF911F910F91E5
:10A7000008959F92AF92BF92CF92DF92EF92FF9205
:10A710000F931F93CF93DF93CDB7DEB76C970FB630
:10A72000F894DEBF0FBECDBF992458C227FF05C0E5
:10A73000109221058FEF80932305809121058930A8
:10A7400040F4E82FFF27EE5DFA4F20838F5F809360
:10A75000210580912105893009F040C280912205B0
:10A7600087FF3CC242E2E42E45E0F42E90E017E081
:10A77000F70181917F01682F892F0E94BA52982F8B
:10A78000115017FFF5CF87FD909580912A059817F6
:10A7900009F01FC2FF248091220588230CF019C202
:10A7A0003FE7B32EB82230912405C32EDD2440911B
:10A7B0002505842F99279695982F88279795879513
:10A7C000C82AD92A20912305822F9927AA27BB2797
:10A7D000FC013197E334F10508F0FBC1EA5BFF4F60
:10A7E000EE0FFF1F0590F491E02D099410912605BE
:10A7F00080912705282F332726FD1068322F222726
:10A80000330F330F8091280599278F77907003E0DD
:10A81000880F991F0A95E1F7282B392B809129057C
:10A82000992780779070B4E095958795BA95E1F770
:10A83000282B392B41E0B901C6010E94DC2741E0F9
:10A84000612FC6010E945927C6010E940F51BDC148
:10A8500080912605992790E4899F902D88271124BF
:10A86000C82AD92A60912705662319F041E0642F90
:10A8700001C041E0C6010E94FA61A7C1809126058E
:10A88000682F772780912705282F3327C9018770E4
:10A8900090709695982F882797958795682B792B98
:10A8A00020743070220F331F80912805822B482F8F
:10A8B000C6010E94AE2889C180912605E82EFF249A
:10A8C000002711278091270599279695982F88278B
:10A8D00097958795AA2797FDA095BA2FE82AF92A78
:10A8E0000A2B1B2B80912805992790E4899F902D96
:10A8F00088271124AA2797FDA095BA2FE82AF92ABC
:10A900000A2B1B2B20912905822F9927AA27BB27C9
:10A9100087709070A070B07035E1880F991FAA1FE2
:10A92000BB1F3A95D1F7E82AF92A0A2B1B2B26954B
:10A9300026952695D801C7010197A109B1098F5F16
:10A940009F4FAF4FB04008F040C1A601C801B7010A
:10A950000E944B5E3AC10E94060E843009F435C154
:10A96000809124050E94C70D882309F42EC184E03C
:10A970000E9420642AC1C114D10409F426C1B60181
:10A980008B2D0E94265221C160912605C6010E948E
:10A990006B26809124058A87809125058B87C601C7
:10A9A0000E944D268C87AE01465F5F4F69E0A7C0CD
:10A9B0001AE0E12EF12CEC0EFD1EAE01405F5F4F60
:10A9C000BE01645F7F4FC6010E94E95C6C018F7716
:10A9D0008A87CC0CCD2CCC1CDD08D1948C2D8F77A4
:10A9E0008B8788898D8789898E871F86A70161E17A
:10A9F0008B2D0E946B538E010F5F1F4FF80194E067
:10AA0000818981879150319697FFFACFA70162E142
:10AA10008B2D0E946B53F80193E0868981879150BA
:10AA2000319697FFFACFA70163E169C0A3E0FA2E40
:10AA300033E0F30E83E0F80E8601243199F480911F
:10AA40002605C82EDD248091270599279695982FF5
:10AA5000882797958795C82AD92A809128058C8FB1
:10AA6000188A23C0AE01405F5F4FBE01645E7F4F16
:10AA7000C6010E94E95C6C0194E0EAE0EF1588F001
:10AA8000DE01AF0DB11D5096E92FFF27EE5DFA4FA5
:10AA900080818D939F5FF394973018F4FAE0FF154F
:10AAA00098F7FE01EF0DF11D108A9E01205F3F4FC8
:10AAB0004C8DB601C8010E94295C8C018F778A8772
:10AAC000000F012F001F110B1195802F12C0213193
:10AAD00021F4C6010E94295D03C0C6010E945E5D8B
:10AAE0006C018F778A87CC0CCD2CCC1CDD08D194DF
:10AAF0008C2D8F778B87AE01465F5F4F60E18B2D8A
:10AB00000E946B5362C0C6010E94265C5EC08091A9
:10AB10002605282F33278091270599279695982F6A
:10AB2000882797958795282B392BA901B6018B2D5E
:10AB30000E9442524AC0C6010E94372846C0BB2428
:10AB4000EBE2F5E08191882369F444E255E064E0AA
:10AB50008B2D0E946B5380911B058B1538F4B0929E
:10AB60001B0504C0B3943FE33B1560F782E080937C
:10AB70001C052BC080911C05833038F583E0809341
:10AB80001C0530931D0540931E058091260580937A
:10AB90001F051092200519C080911C058230A8F471
:10ABA00082E080931C0530931D0540931E05109292
:10ABB0001F050BC090911C05992339F481E0809307
:10ABC0001C0530931D0590931E0561E08B2D0E949E
:10ABD000F552109221058FEF809323050E94771381
:10ABE0009C018FEF2F3F380709F0A0CD0E94391349
:10ABF0000A970CF421C190911805809119059817B6
:10AC000011F19091190589E0989F70011124E4EFEA
:10AC1000F4E0EE0EFF1E08E010E0F70181917F01E5
:10AC20000E944A130150104017FFF7CF8091190579
:10AC30008F5F8093190580911905843008F4FCC05A
:10AC400010921905F9C07E010894E11CF11C57010E
:10AC500080911A05803429F060911C05662309F45F
:10AC600075C08FEF89830894E11CF11C80911C054D
:10AC7000992781309105C9F0823091051CF4892B08
:10AC800039F059C08230910519F10397C1F153C0D1
:10AC900080E4F701819380911D05982F97708F5F55
:10ACA00080931D0591937F0148C081E4F701819352
:10ACB00080911D058770819380911E05982F9F7745
:10ACC0008F5F80931E0591937F0180911E0531C097
:10ACD00082E4F701819380911D05877081938091B3
:10ACE0001E058F77819380911F05982F9F778F5F27
:10ACF00080931F0591937F0180911F051AC083E403
:10AD0000F701819380911D058770819380911E05C5
:10AD10008F77819380911F058F7781938091200594
:10AD2000982F9F778F5F8093200591937F0180916B
:10AD3000200587FF02C010921C0580911C05882306
:10AD400009F059C080911A058F5F53C08134A1F575
:10AD50008FEF89830894E11CF11C83E0F701819354
:10AD60007F018F010894E11CF11C0E94060E8F7771
:10AD7000F801808380911A058F5F80931A050E94E5
:10AD8000CA288C01FC01868581FF13C080819181D6
:10AD90000E940F5141E0F8016089808191810E94F9
:10ADA000592741E0F80164817581808191810E9479
:10ADB000DC2751E0952E1FC0803410F060931A05F7
:10ADC00080911A05806889830894E11CF11C82E057
:10ADD000F70181937F0180911A050E94F5528091BD
:10ADE0001A058F5F80931A0590911B05981718F428
:10ADF00080E480931A05CE010996E816F90620F43E
:10AE0000F70111927F01F9CFDD24750107E010E011
:10AE1000F70160818D2D0E94BA52D82EF7018191E1
:10AE20007F010E944A130150104017FFF1CFD7FC59
:10AE3000D0948D2D0E944A13A895892D99276C9640
:10AE40000FB6F894DEBF0FBECDBFDF91CF911F913B
:10AE50000F91FF90EF90DF90CF90BF90AF909F90B9
:10AE60000895CF93DF93CDB7DEB726970FB6F8944A
:10AE7000DEBF0FBECDBF36E0FE01319611923A958E
:10AE8000E9F74983AE014F5F5F4F0E946B532696EF
:10AE90000FB6F894DEBF0FBECDBFDF91CF910895FE
:10AEA0001F93CF93DF93EC0110E001C0A8950E949F
:10AEB000541E8823D9F310C0A89504C081E090E007
:10AEC0000E9459160E94541E8823C1F361E080E05D
:10AED00090E00E94791C21970E94641E882311F43F
:10AEE000209751F70E94641E811111E0C5E00EC049
:10AEF00063E080E090E00E94791C0E94681E01C01F
:10AF0000A8950E94541E8823D9F3C1500E94641E44
:10AF1000882311F0CC2361F7CC2309F41C2F812F57
:10AF20009927DF91CF911F910895EF92FF921F9380
:10AF3000CF93DF937C01CFEFDFEF10E0612FC701EC
:10AF40000E94F21C80E090E00E945057882311F08C
:10AF5000C12FDD271F3F49F483E090E00E94505746
:10AF6000882331F0CFEFD0E005C01F5FD7FDE6CFDB
:10AF7000D7FD14C01C2FCFEFDFEF612FC7010E9458
:10AF8000F21C83E090E00E945057882311F0C12FFB
:10AF9000DD27112319F01150D7FDEFCFCE01DF913E
:10AFA000CF911F91FF90EF9008954F925F926F9213
:10AFB0007F928F929F92AF92BF92CF92DF92EF9249
:10AFC000FF920F931F93CF93DF93CDB7DEB72697F2
:10AFD0000FB6F894DEBF0FBECDBF782E5B01C42E36
:10AFE000522E402E8091620082608093620080E049
:10AFF0000E943D1986E0FE01319611928A95E9F78B
:10B00000AE014F5F5F4F62E28FEF0E946B530E9471
:10B01000751E83EC87B98FEE86B96FEF862E962E5C
:10B02000662480E00E94C70D82E390E00E945916DA
:10B0300084E00E94C70D84E690E00E945916E090DB
:10B04000B806F090B9060091BA061091BB0680EDE3
:10B0500097E0A0E0B0E0E80EF91E0A1F1B1FDD24F8
:10B0600010926C0510926B052BC00E94701EAC01F3
:10B0700020916B0530916C05C901885A9D4F84174A
:10B08000950734F0C901885592404817590744F490
:10B0900050936C0540936B05DD2059F0DA9409C09C
:10B0A000240F351F3595279530936C0520936B053C
:10B0B000D39494E09D1550F08AE090E00E945916D8
:10B0C000C801B7010E942214882379F280916B0590
:10B0D00090916C0544975CF584E393E00E946B1EAD
:10B0E00083E090E00E94505710E0412F612F80E0F4
:10B0F00090E00E94B91C83E090E00E9450578111BB
:10B1000011E041E060E080E090E00E94B91C83E043
:10B1100090E00E94505781111F5F113041F484E18B
:10B1200090E090936C0580936B0545E0D42E809160
:10B130006B0590916C054497855A9B4028F4B4E0C8
:10B14000BD1510F1442001F560E081E00E94EA178E
:10B1500080916B0590916C058431910514F485E123
:10B1600006C0895B9B4014F086E101C087E10E9424
:10B17000A94FBC0182E00E94721980E00E94C70DB5
:10B1800088EE93E00E94591680916B0590916C05B2
:10B19000805E9C4F0E946B1E86E990E00E945916CB
:10B1A0000E94060E843009F0D8C0072D1127033005
:10B1B000110509F447C0043011054CF401301105A4
:10B1C00039F102301105FCF4012B71F0ACC00530EF
:10B1D00011050CF4A8C0073011050CF453C0093058
:10B1E00011050CF0A0C06FC0452D6C2DC5010E944B
:10B1F000991C8FE090E00E945057882309F497C073
:10B20000852C992494C06C2DC5010E940B1D4CC047
:10B2100040E06C2DC5010E94B91C83E090E00E94C3
:10B220005057882309F046C041E06C2DC5010E94AB
:10B23000B91C83E090E00E945057882309F477C03E
:10B24000480177C010E0012F169540E0602FC5013E
:10B250000E94B91C83E090E00E945057882309F4B3
:10B2600010680F5F083080F3612FC5010E94241D14
:10B2700083E090E00E945057882309F458C0812E43
:10B28000992455C061E085E090E00E94D91C8FE0D0
:10B2900090E00E945057C50187709070F5E07F16CE
:10B2A00061F46C2D0E94D91C8FE090E00E945057F1
:10B2B0008823E9F1882499243CC00E9495574C01C9
:10B2C00033E0632E34C0C501969587959695879592
:10B2D000682F6F5F85E090E00E94D91C8FE090E0BE
:10B2E0000E945057C5018370907027E0721661F478
:10B2F0006C2D0E94D91C8FE090E00E94505788234B
:10B3000041F08824992405C00E9495574C0193E090
:10B31000692E61E085E090E00E94D91C8FE090E00A
:10B320000E94505704C08FEF882E982E08C097FCBB
:10B3300006C0442021F08CE291E00E94591680E082
:10B340000E94C70D97FE09C08CE291E00E94591639
:10B35000639482E0861508F064CE16B886B187B98A
:10B360000E94BB50FC0184810E943D1981E08983C9
:10B37000AE014F5F5F4F62E28FEF0E946B5380918F
:10B3800062008D7F80936200C40126960FB6F89408
:10B39000DEBF0FBECDBFDF91CF911F910F91FF9008
:10B3A000EF90DF90CF90BF90AF909F908F907F9065
:10B3B0006F905F904F9008950F93242F01E0462FD8
:10B3C000BC0180E00E94D5570F9108950F9300E0D3
:10B3D000202F462FBC0181E00E94D5570F91089580
:10B3E0000F9301E020E0462FBC0182E00E94D55778
:10B3F0000F9108950F9300E0202F402FBC0183E0B0
:10B400000E94D5570F9108950F9301E020E0482F37
:10B4100060E070E085E00E94D5570F9108950F938A
:10B42000992701E020E0462FBC0185E00E94D55716
:10B430000F9108950F93992700E0202F402FBC0112
:10B4400086E00E94D5570F9108950F9301E020E008
:10B45000462FBC0187E00E94D5570F9108950F93A6
:10B4600000E0202F402FBC0188E00E94D5570F91AB
:10B470000895880F61118F5FF894E82FFF27EF562A
:10B48000F54F90818091500A80FD10827894892F29
:10B4900099270895880F61118F5FF894E82FFF278F
:10B4A000DF01AF52B54F8C91EF5AF54F80837894FE
:10B4B000992708959091500A882311F0916001C056
:10B4C0009E7F9093500A0895089580E4E1E5FAE0A4
:10B4D00011928A95E9F7089584E0809374001092A0
:10B4E000710082E28093700008951F920F920FB650
:10B4F0000F9211248F939F93EF93FF93809171008C
:10B500009927887F90708032910509F487C0813235
:10B5100091056CF480319105D9F0813191051CF4CD
:10B520000897D1F07DC0489709F43FC079C08034B6
:10B530009105A9F18134910524F4889709F441C05B
:10B540006FC080359105D9F08835910561F068C0EC
:10B5500080916D0587FF02C080EA01C081EA809377
:10B56000730085E861C0E0917305F09174058091E6
:10B5700073008193F0937405E093730548C0E091E4
:10B580007305F0917405809173008193F0937405B5
:10B59000E093730580916E05815080936E058091D4
:10B5A0006E058230F4F285EC3FC080917105909178
:10B5B0007205892F9927809373008FEF80936D0513
:10B5C000D0CF80916D0587FF09C080917105909162
:10B5D00072058093730010926D05C3CF80916F0543
:10B5E0008823E1F080916E05882389F0E09173054E
:10B5F000F09174058191F0937405E0937305809345
:10B60000730080916E05815080936E05AACF84E906
:10B610008093740081E08093700508C085EA04C0BF
:10B620008FEF8093700584E980937400FF91EF9110
:10B630009F918F910F900FBE0F901F901895809142
:10B640007400992787709070009711F081E090E066
:10B650000895089560936E05909372058093710527
:10B6600020936F0550937405409373058EEF80937C
:10B670006D051092700585EA80937400089580919D
:10B680007005992787FD909508950E942A5B01C057
:10B69000A8950E943F5B892BD9F38091700599276B
:10B6A00087FD90950895AB0120E060E134E0880FBC
:10B6B000991F3A95E1F70E94455B0895AB0121E09F
:10B6C00060E174E0880F991F7A95E1F70E94455B6D
:10B6D000089520E0AC0164E080E090E00E94455BCA
:10B6E000089521E0AC0164E080E090E00E94455BB9
:10B6F0000895EF92FF920F931F93CF93DF93CDB7EF
:10B70000DEB722970FB6F894DEBF0FBECDBF7C0127
:10B7100019821A8209811A8120E0AE014F5F5F4FC2
:10B7200062E0C801E4E0880F991FEA95E1F70E9402
:10B73000455BA89589819A81009719F08E159F0520
:10B7400049F7C80122960FB6F894DEBF0FBECDBFF1
:10B75000DF91CF911F910F91FF90EF9008950F937C
:10B760001F93CF93DF93CDB7DEB722970FB6F89430
:10B77000DEBF0FBECDBF8C0101978F5F934000F5F8
:10B7800020E0AE014F5F5F4F62E0C801A4E0880F88
:10B79000991FAA95E1F70E94455BC8010E94795B59
:10B7A00024E08030920760F421E0AE014F5F5F4FEC
:10B7B00062E0F4E0880F991FFA95E1F70E94455B7B
:10B7C00022960FB6F894DEBF0FBECDBFDF91CF91AA
:10B7D0001F910F9108950F931F93CF93DF93CDB7D0
:10B7E000DEB764970FB6F894DEBF0FBECDBF8C01F5
:10B7F00001978F5F9340F8F4C8010E94AF5BCE01C0
:10B8000041960E94695B40E150E06FEF70E0CE012D
:10B8100001960E94BC648B899C8989839A83BE01AE
:10B820006F5F7F4FC8010E945E5B0B8B1C8BCE014C
:10B8300041960E94715B64960FB6F894DEBF0FBE0E
:10B84000CDBFDF91CF911F910F9108950E94EB5BC7
:10B8500008957F928F929F92AF92BF92CF92DF9284
:10B86000EF92FF920F931F93CF93DF93CDB7DEB785
:10B87000AA970FB6F894DEBF0FBECDBF7C014B0177
:10B88000742E5901232B79F1672B69F180E0E816BA
:10B8900084E0F80640F5E114F10421F0C7010E94AC
:10B8A000AF5B1EC0CE0181960E94695B0BA11CA1FB
:10B8B0000115110511F4C70112C020E0AE014D5D64
:10B8C0005F4F62E0C80134E0880F991F3A95E1F7B5
:10B8D0000E94455BCE0181960E94715BC8017C018C
:10B8E000E114F10411F4C70158C06E010894C11CA1
:10B8F000D11CF5018B829C827D82DE01169620810F
:10B90000222351F0CE014196A817B90728F43196A9
:10B910002D9320812223C1F7C6014096A817B907AD
:10B9200008F41C92E9A6FAA6CE0185960E94695BEE
:10B93000EE24FF240DA11EA101151105B1F0A8955B
:10B94000BE016F5E7F4FC8010E94535BC601059622
:10B950004BE050E0BC01CE0146960E94056599235C
:10B9600024F4780109891A89E7CFF601008311834D
:10B97000A895B60189A59AA50E945E5B21E0AE015B
:10B98000475D5F4F62E0C701B4E0880F991FBA9529
:10B99000E1F70E94455B89A59AA5AA960FB6F8948F
:10B9A000DEBF0FBECDBFDF91CF911F910F91FF90F2
:10B9B000EF90DF90CF90BF90AF909F908F907F904F
:10B9C00008959A01462FBC0180E090E00E94295C16
:10B9D0000895EF92FF920F931F93CF93DF93CDB70C
:10B9E000DEB760970FB6F894DEBF0FBECDBF9C01E7
:10B9F0007B018A0101978F5F934018F080E090E00F
:10BA00001BC0BE016F5F7F4FC9010E94535BE114F1
:10BA1000F10419F08D81F70180830115110551F0B2
:10BA20008BE0F801DE0116960D9001928A95E1F700
:10BA3000F80113868B819C8160960FB6F894DEBF67
:10BA40000FBECDBFDF91CF911F910F91FF90EF906F
:10BA500008950F931F93CF93DF93CDB7DEB764970D
:10BA60000FB6F894DEBF0FBECDBF8C01815094405D
:10BA700018F080E090E017C0CE0141960E94695B0B
:10BA80000115110571F0BE016F5F7F4FC8010E9463
:10BA9000535B89819A81009721F02FEF8F3F9207A6
:10BAA00011F489899A8964960FB6F894DEBF0FBEA7
:10BAB000CDBFDF91CF911F910F910895CF93DF9369
:10BAC000CDB7DEB724970FB6F894DEBF0FBECDBF5B
:10BAD00024E08130920718F080E090E00FC00097DA
:10BAE00039F4CE0101960E94695B89819A8106C072
:10BAF0000E94795B009711F40E94795B24960FB63F
:10BB0000F894DEBF0FBECDBFDF91CF910895EF92C5
:10BB1000FF920F931F93CF93DF93CDB7DEB7649758
:10BB20000FB6F894DEBF0FBECDBF198A1A8A01E0A6
:10BB300010E00B8B1C8BA895CE0141960E94715B87
:10BB400040E150E06FEF70E0CE01800F911F0E9446
:10BB5000BC6440E1E42EF12C83E00F3F18073CF475
:10BB60000F5F1F4F09831A830150104002C01982D2
:10BB70001A820E940A0E21E0AE014F5F5F4F60E122
:10BB8000C7010E94455B0F5F1F4F80E190E0E80E08
:10BB9000F91E94E000301907FCF264960FB6F89491
:10BBA000DEBF0FBECDBFDF91CF911F910F91FF90F0
:10BBB000EF900895EF92FF920F931F93CF93DF932F
:10BBC000CDB7DEB764970FB6F894DEBF0FBECDBF1A
:10BBD000CE0141960E94695B89E00E94D5168823B8
:10BBE00029F08EE00E94D516882351F48B899C8918
:10BBF0008F5F9F4F21F589899A898F5F9F4FF9F455
:10BC000064E971E084E00E9419196CE871E085E054
:10BC10000E94191968EC70E085EB99E40E942318E2
:10BC200060E0862F0E94EA1783E00E94A94FBC01C2
:10BC300082E00E9472190E94875D0E94B6520989B3
:10BC40001A89C80101978F5F9340C0F4BE016F5FEE
:10BC50007F4FC8010E94535BE980FA808B819C81F1
:10BC600001978F5F974218F0C8010E94EB5B870134
:10BC7000A895C70101978F5F934040F364960FB674
:10BC8000F894DEBF0FBECDBFDF91CF911F910F9112
:10BC9000FF90EF900895EF92FF920F931F93CF9331
:10BCA000DF93CDB7DEB728970FB6F894DEBF0FBE8F
:10BCB000CDBF7B018C01FA018091750590917605CD
:10BCC000892B91F1E982FA820B831C831F821886EB
:10BCD000022F112700FF09C04F83588740E050E032
:10BCE000BA01CF010E94E95CFC0101FF05C08F8110
:10BCF000988590688F839887ED83FE83EF2BA1F062
:10BD000021E0AE014F5F5F4F68E080917505909133
:10BD100076050E94455B80917505909176050896A1
:10BD2000909376058093750528960FB6F894DEBF3C
:10BD30000FBECDBFDF91CF911F910F91FF90EF907C
:10BD40000895CF92DF92EF92FF921F93CF93DF93EC
:10BD5000CDB7DEB728970FB6F894DEBF0FBECDBFC4
:10BD600010E0C12C30E4D32E80914E0A181798F5BC
:10BD7000812F9927FC0123E0EE0FFF1F2A95E1F7A1
:10BD8000E80FF91FE80FF91FE253F84F8081918106
:10BD900089839A83828193818B839C83848195811B
:10BDA0008D839E838085282F33272F833887868134
:10BDB00087FD03C031602F83388721E0AE014F5FDC
:10BDC0005F4F68E0C6010E94455B1F5F88E090E01E
:10BDD000C80ED91EC9CF0E94BB502FEF3FEF298359
:10BDE0003A83FC01858596858B839C8321E0AE0197
:10BDF0004F5F5F4F68E0C6010E94455B88E090E0BE
:10BE0000C80ED91E0E94CA28FC01D0927605C092A5
:10BE10007505828993892685892B41F020FF02C010
:10BE200023E001C021E04289538907C020FF02C0FE
:10BE300022E001C020E04081518160E070E080E0BC
:10BE400090E00E944B5E10E040E050E06BE0812FFC
:10BE50000E946B531F5F1034B8F310E00E948153AF
:10BE60008823E1F31F5F1630C8F310E0212F4FEF56
:10BE70005FEF6FEF7FEF8FEF9FEF0E944B5EC09001
:10BE80007505D0907605109276051092750581E1C2
:10BE9000E82E8BE0F82E1FE121E0A70168E0C60143
:10BEA0000E94455B1150E8E0F0E0EE0EFF1ECE0E62
:10BEB000DF1E17FFF1CF28960FB6F894DEBF0FBE36
:10BEC000CDBFDF91CF911F91FF90EF90DF90CF908A
:10BED00008957F928F929F92AF92BF92CF92DF92FE
:10BEE000EF92FF920F931F93CF93DF93CDB7DEB7FF
:10BEF0006C970FB6F894DEBF0FBECDBF0E94060E42
:10BF0000782E80E00E94C70D40E050E060E0CA015A
:10BF10000E946E2986E08E010F5E1F4FF80111927C
:10BF20008A95E9F7FF24A80167E08F2D0E946B53E3
:10BF300084E190E00E945916F3942FE32F1598F7AF
:10BF40000E94C12419821A82A12C00E4B02E20E0A4
:10BF5000AE014F5F5F4F68E0C5010E94455B89817C
:10BF60009A81EFEF8F3F9E07E1F00E9431258C010F
:10BF7000892BB9F08F818F70682FF80180819181B2
:10BF80000E946B268B819C81F801828393838D8133
:10BF90009E81848395838F819885892F992780FD41
:10BFA000168288E090E0A80EB91E89819A818F5F81
:10BFB0009F4F69F619861A861B861C86B9E08B2E60
:10BFC000912C8C0E9D1E20E0A40168E0C5010E940A
:10BFD000455B89859A85AB85BC8580509040A040A3
:10BFE000B14008F0A8C08D859E85009709F4A3C0D4
:10BFF00028E28030920708F09EC0FF242F85388900
:10C0000037FF02C0A2E0FA2E8C012115310589F01C
:10C0100089011F7740E050E0BA01C8010E94E95C45
:10C020002D853E852817390719F481E0F82A01C0CB
:10C030008901F4012081318142815381CF2CDD249B
:10C040002115310541055105C1F50E94CA287C0121
:10C05000C0FE08C04496AC0160E070E0C8010E94D8
:10C06000E95C8C01C8010E9409258C010097D1F080
:10C07000FC01448155816681808191810E946E29F5
:10C08000F80180850E94CF29F801828193810E9466
:10C090000925009739F0FC016481758180819181C7
:10C0A0000E94B829C1FE04C0F70186858160868799
:10C0B000F7018685826086873EC0802F8F778F8BC1
:10C0C000000F012F001F110B1195802F8F77888F84
:10C0D000F40180818F77898FE7E0569547953795F2
:10C0E0002795EA95D1F7822F8F778A8F77E056953B
:10C0F0004795379527957A95D1F7822F8F778B8F34
:10C1000067E056954795379527956A95D1F7822F21
:10C11000877053E0CC0CDD1C5A95E1F78C298C8F8D
:10C12000AE01495E5F4F6CE08FEF0E946B530E943F
:10C1300081538823E1F388E090E0A80EB91E898539
:10C140009A85AB85BC8580509040A040B14008F4F2
:10C1500035CF01E11BE04FE1F42E20E0A80168E0BB
:10C16000C5010E94455BFA94085F1F4F88E090E08C
:10C17000A80EB91EF7FEF1CF83E00E94C70D84E63A
:10C1800090E00E9459168B819C810E942763872D25
:10C190000E94C70D6C960FB6F894DEBF0FBECDBFE0
:10C1A000DF91CF911F910F91FF90EF90DF90CF9093
:10C1B000BF90AF909F908F907F9008952FEF3FEFAB
:10C1C000E7E7F5E08FE1208331833796815087FFE1
:10C1D000FACF0895AC01FC0123E0F695E7952A9586
:10C1E000E1F7EF5EF44F808199279A012770307054
:10C1F00002C0959587952A95E2F7440F551F382F71
:10C20000317080FF02C04F5F5F4F20E0E7E7F5E04D
:10C21000808191818417950759F4868180FF0CC035
:10C22000332319F082E590E0089587E490E00895C3
:10C230002F5F3796203260F3332319F082E790E0C6
:10C24000089587E690E0089508951F93CF93DF93B4
:10C25000EC01162F892B09F4A2C0662319F08E81F8
:10C2600080FD9DC0112309F481C0809157069091F3
:10C270005806A0915906B0915A068896A11DB11D85
:10C28000BC01CD010E942214882309F488C0488192
:10C29000598190E0E7E7F5E0BA01B3E0769567955C
:10C2A000BA95E1F7208131818FEF2F3F380779F080
:10C2B0002417350761F0868180FF09C0A3E0369519
:10C2C0002795AA95E1F72617370709F468C09F5FFD
:10C2D0003796903238F361E0888199810E94641C1E
:10C2E0008091B8069091B906A091BA06B091BB06AC
:10C2F0008A839B83AC83BD838093570690935806B3
:10C30000A0935906B0935A068E8181608E8383FF75
:10C3100006C088819981969587950E9426644881F8
:10C320005981CA0164E0969587956A95E1F7682F6F
:10C330009A01369527952770307081E090E002C011
:10C34000880F991F2A95E2F7982F772740FF06C09C
:10C35000FB01EF5EF44F8081892B06C0FB01EF5E8D
:10C36000F44F90958081892380833EC08E818260C6
:10C370008E83992780FF13C082FF11C080915706DA
:10C3800090915806A0915906B0915A068896A11D21
:10C39000B11DBC01CD010E942214882319F480E054
:10C3A00090E024C0612F888199810E94641C809153
:10C3B000B8069091B906A091BA06B091BB068093D9
:10C3C000570690935806A0935906B0935A068E814B
:10C3D00083FF06C088819981969587950E9426647F
:10C3E0008FEF9FEF8883998381E090E0DF91CF9179
:10C3F0001F910895FF920F931F93CF93DF938C01AA
:10C40000F62E805F9F4018F080E090E051C020E061
:10C41000E7E7F5E0808191818017910731F12F5F87
:10C4200037962032B8F3FF2089F41CC000831183B3
:10C430008091B8069091B906A091BA06B091BB065A
:10C4400082839383A483B58316820FC020E0E7E73D
:10C45000F5E0808191818F5F9F4F41F32F5F379689
:10C460002032B8F3C0E0D0E003C0EF01309721F4F0
:10C47000CE01FF20E9F41AC0442319F086818860B8
:10C4800086830E94BB50FC01FF2061F09801369525
:10C490002795858596858217930720F4258736870B
:10C4A0000E9442506F2DCE010E94256181E090E0F4
:10C4B000DF91CF911F910F91FF9008956F927F921E
:10C4C0008F929F92AF92BF92CF92DF92EF92FF92A4
:10C4D0000F931F93CF93DF930E94BB508C01FC01FD
:10C4E00083859927AA27BB27BC01CD0122E330E031
:10C4F00040E050E00E94C3696B017C01F801848533
:10C500009927AA27BB27BC01CD0124E630E040E0F3
:10C5100050E00E94C3693B014C01AA24BB24C7E739
:10C52000D5E00FE1888199818F5F9F4F51F18E8116
:10C53000992780FF14C082FD24C08A819B81AC8131
:10C54000BD818C0D9D1DAE1DBF1DBC01CD010E9486
:10C5500022148823B1F08E8184608E8312C0A114CE
:10C56000B10471F0F50122813381448155818A81C2
:10C570009B81AC81BD8182179307A407B50708F49E
:10C580005E010150279607FFCDCF8091570690910D
:10C590005806A0915906B0915A068896A11DB11D62
:10C5A000BC01CD010E942214882399F08091B80625
:10C5B0009091B906A091BA06B091BB068897A109DF
:10C5C000B1098093570690935806A0935906B093EB
:10C5D0005A0600E0C7E7D5E0888199818F5F9F4FB9
:10C5E000E1F08E81992780FF18C082FF16C081FD7F
:10C5F0000EC08A819B81AC81BD81860D971DA81DCF
:10C60000B91DBC01CD010E942214882331F060E0E5
:10C61000CE010E942561882359F40F5F27960032CE
:10C62000D8F2A114B10421F061E0C5010E94256196
:10C63000DF91CF911F910F91FF90EF90DF90CF90FE
:10C64000BF90AF909F908F907F906F9008959F9232
:10C65000AF92BF92CF92DF92EF92FF920F931F9310
:10C66000CF93DF937C0188EFE81687E0F80608F0A7
:10C6700076C00E94BB505C01FC01E586F6860E94F4
:10C680004250CC24DD249924092D1127E016F1060F
:10C6900008F450C0C80123E0969587952A95E1F7E4
:10C6A000482F98012770307081E090E002C0880F19
:10C6B000991F2A95E2F7982FE801CC0FDD1FE42F90
:10C6C000FF27EF5EF44F8081892309F0219640E037
:10C6D00061E0CE010E94FA6140E0642FCE010E9429
:10C6E000FA6160E081E00E94EA170894E11CF11C05
:10C6F000FF92EF920894E108F1080894C11CD11C44
:10C70000DF92CF9288E10E94A94F9F938F9382E09E
:10C710008F930E94C81984E690E00E9459168DB745
:10C720009EB707960FB6F8949EBF0FBE8DBF0C5FE5
:10C730001F4FACCFF501838599270E94591693941A
:10C74000F3E0F91508F0A0CF84E690E00E945916B6
:10C7500002C00E940A0E0E94541E8823D1F3DF916A
:10C76000CF911F910F91FF90EF90DF90CF90BF90EE
:10C77000AF909F900895EF92FF920F931F93CF93E6
:10C78000DF9380915B06682F772710925B06E1E1CB
:10C79000FCE08191882311F0706805C08DE0E031E4
:10C7A000F807B9F3B4F340E050E080914E0A9927BE
:10C7B000481759079CF4DC019A01F901E40FF51FB1
:10C7C000E253F84F878180FF02C0706407C04F5F5B
:10C7D0005F4F275F3F4F4A175B077CF340E050E015
:10C7E00080914F0A9927880F991F4817590704F518
:10C7F0007C01E1E9FAE001E51AE0C1EDDAE09991A6
:10C80000D8018D918D01981759F48081282F3327F5
:10C81000892F99278095909528233923232B11F070
:10C82000706206C04F5F5F4F31964E155F053CF357
:10C83000CB01DF91CF911F910F91FF90EF90089561
:10C8400090915B06982B90935B0608959C0187E07E
:10C85000283F3807A0F4F90183E0F695E7958A951B
:10C86000E1F7EF5EF34F2770307081E090E002C097
:10C87000880F991F2A95E2F72081282B208308959D
:10C88000089528E28030920740F40E940925FC01B7
:10C89000892B19F087818160878308950895CF934C
:10C8A000DF9310925B0680E091E0E1E1FCE0119201
:10C8B0000197E9F7C1E5DAE0A1EDBAE0E1E9FAE0D4
:10C8C00080914F0A9927880F991F009741F09C018A
:10C8D0008D919191892B899321503040C9F7EEECCD
:10C8E000F7E080914E0A9927009751F09C018781CB
:10C8F0008E7F8783215030403A9621153105B9F754
:10C90000DF91CF910895E199FECF9FBB8EBBE09A56
:10C9100099278DB308954115510569F0DC01E1991E
:10C92000FECF7FBB6EBBE09A6F5F7F4F0DB20D9263
:10C9300041505040B1F70895E199FECF9FBB8EBBA7
:10C940006DBB0FB6F894E29AE19A0FBE08954115B7
:10C95000510589F0DC018FB7E199FECF7FBB6EBB3B
:10C960000D900DBAF894E29AE19A8FBF6F5F7F4FF6
:10C970004150504089F70895DC0101C06D9341504A
:10C980005040E0F708950F931F93CF93DF93CDB7F7
:10C99000DEB72C970FB6F894DEBF0FBECDBF0B8964
:10C9A0001C89ED89FE893EE03C8309831A834FEFA1
:10C9B0005FE74D835E83AE01495E5F4FBF01CE01ED
:10C9C00001960E947E662F813885020F131FD801C1
:10C9D0001C922C960FB6F894DEBF0FBECDBFDF9130
:10C9E000CF911F910F910895FB01DC018D91019072
:10C9F000801911F40020D1F7990B0895FB01DC0197
:10CA000001900D920020E1F70895FB01DC014150F7
:10CA1000504030F08D910190801919F40020B9F741
:10CA2000881B990B0895FB01DC014150504030F008
:10CA30008D910590801919F40020B9F7881B990B86
:10CA400008952F923F924F925F926F927F929F92A2
:10CA5000AF92BF92CF92DF92EF92FF920F931F930C
:10CA6000CF93DF93CDB7DEB76E970FB6F894DEBFE6
:10CA70000FBECDBF898B9A8B6B8B7C8B4D8B5E8B66
:10CA80003C011F8A188EF30191903F01892D99274F
:10CA90000E943D6A892BB9F70DE2901609F4FFC098
:10CAA0001BE2911609F4F7C02D893E892115310545
:10CAB00009F4DAC02031310509F4D6C0ED89FE89C8
:10CAC000EF2B41F430E3931609F4C9C04AE050E07B
:10CAD0004D8B5E8B8D899E89AA2797FDA095BA2FD5
:10CAE000898F9A8FAB8FBC8F8F89988D892B09F492
:10CAF000B1C060E070E080E090E8298D3A8D4B8D08
:10CB00005C8D0E946E6A29873A874B875C876D87A8
:10CB10007E878F87988B58E0DE011196FE0139964B
:10CB200001900D925A95E1F7CC24DD247601AA24D8
:10CB3000BB2429803A804B805C802D813E812D8FE3
:10CB40003E8F092D1127C8010E94316A892BC9F136
:10CB5000C8010E94366A892B09F46BC070ED970EEC
:10CB6000892D99276D897E898617970754F5B7FC1B
:10CB700024C02C143D044E045F04F8F0C214D30406
:10CB8000E404F504A9F021E0A22EB12CC701B601FE
:10CB9000298D3A8D4B8D5C8D0E94C3696B017C01A0
:10CBA000C90CD11CE11CF11CD3019D903D01C9CFE2
:10CBB000AD8CBE8CA816B90634F73FEFA32EB32E6A
:10CBC000F3CFB7FE29C0EF89F88DEF2BE1F0C12C30
:10CBD000D12CE12C90E8F92E02E210E01093120D16
:10CBE0000093110D8B899C89892B09F460C0AB28B7
:10CBF00039F0C3010197AB89BC898D939C9357C0D1
:10CC000089899A89F8CF8FEFC82E8FEFD82E8FEFB2
:10CC1000E82E8FE7F82EE0CFAF89B88DAB2B11F35C
:10CC2000F094E094D094C094C11CD11CE11CF11C80
:10CC3000D9CFC8010E94176A892B19F2C8010E9436
:10CC4000156A892B21F0802F8753982E89CF802F4A
:10CC50008755FBCF6FEF7FEF8FEF9FE74ECF08E059
:10CC600010E00D8B1E8B36CF40E3941609F026CFD3
:10CC7000F3018081883719F0883509F01FCFD3017F
:10CC800011969C9082E090E0680E791E60E170E061
:10CC90006D8B7E8B13CFD3019D903D0105CF21E09D
:10CCA00030E02F8B388FF30191903F01FDCEC7010B
:10CCB000B6016E960FB6F894DEBF0FBECDBFDF9102
:10CCC000CF911F910F91FF90EF90DF90CF90BF9089
:10CCD000AF909F907F906F905F904F903F902F907C
:10CCE0000895DC015C91552341F05F7D51341CF0C7
:10CCF0005B350CF45C931196F5CF08952F923F921B
:10CD00004F925F926F927F928F929F92AF92BF925B
:10CD1000CF92DF92EF92FF920F931F93CF93DF9307
:10CD2000CDB7DEB762970FB6F894DEBF0FBECDBFAA
:10CD3000AA24BB2465014C016D877E874F87588BE1
:10CD400044245524FC0146825782838181FD5BC2C5
:10CD50008FEF9FEF6FC240FE44C2862D80538A3012
:10CD6000E0F4F0E36F1641F42A89222329F47720B6
:10CD700019F480E091E08BC08AE09A89989F902D09
:10CD80001124892F860D80538A8B882314F4EFE7B2
:10CD9000EA8B43FC38C27A8836C243FE05C0FA8962
:10CDA000FF2311F421E02A8B862D992787FD90958A
:10CDB0008836910554F5853691050CF06BC08835A1
:10CDC000910509F4D3C089359105B4F48B329105EE
:10CDD00009F442C08C32910544F48032910509F483
:10CDE0003FC0839709F442C0F2C18D329105D9F159
:10CDF0008E9709F440C0EBC18336910509F454C005
:10CE00008436910509F478C0E2C18037910509F4B0
:10CE1000A5C08137910584F48C369105B1F18D362A
:10CE200091052CF48936910509F466C0D0C18F367E
:10CE3000910509F490C0CBC18537910509F498C0DC
:10CE40008637910524F483379105B9F1C0C188373D
:10CE5000910509F48BC0BBC180E190E0482A592AB2
:10CE6000E0E2F0E005C080E890E011C0E0E4F0E02E
:10CE70004E2A5F2AC8C188E090E0482A592AEFEF7D
:10CE8000FEEF4E225F221A8ABEC184E090E0482A5B
:10CE9000592AB9C10F2EFFE3AF2EF02D7A940F2E31
:10CEA000F3E66F2EF02D3AC1EF85F889CF01029697
:10CEB0008F87988BA0807A9431C1EF85F889CF0154
:10CEC00002968F87988BA080B18043FE0BC0EA89C1
:10CED0008E2F992787FD9095BC01C5010E94B869E6
:10CEE000898B07C0F50101900020E9F73197EA1915
:10CEF000E98BF9897F1A12C142FE0BC0EF85F889D0
:10CF0000CF0104968F87988B208131814281538194
:10CF10000DC0EF85F889CF0102968F87988B8081AD
:10CF200091819C01442737FD4095542F59016A0196
:10CF3000552364F4E2E0F0E04E2A5F2AD094C094D6
:10CF4000B094A094A11CB11CC11CD11C8FEB9FEF0D
:10CF5000482259222BC098E0998B0AC0E0E4F0E007
:10CF60004E2A5F2A0F2EF8E76F2EF02DF0E1F98B95
:10CF700042FE0BC0EF85F889CF0104968F87988B0E
:10CF800020813181428153810BC0EF85F889CF0127
:10CF900002968F87988B808191819C014427552729
:10CFA00059016A01EFECFFEF4E225F221E01089447
:10CFB000211C311CF989EF2EFF2400271127C601FF
:10CFC000B501A80197010E944C6ADC01CB01F10177
:10CFD00080838A301CF0860D815203C0F10180816C
:10CFE000805DF10181931F01C601B501A801970180
:10CFF0000E944C6A59016A0121153105410551050C
:10D00000F1F6CE010196A22CA81AC201827390708B
:10D01000892B09F07A9446FE0FC0872D992787FD4A
:10D020009095F989F03131F40F2EFEEF7F2EF02D1F
:10D03000780E02C0782E7A9443FE12C08A89282F77
:10D04000332727FD30958A2D9927821793072CF0D7
:10D05000E7EFFFEF4E225F2203C0FA89FA19FA8B3D
:10D0600043FE03C02A89721A01C07A18C20180786F
:10D070009170892B69F4872D7A9418164CF4B401B9
:10D0800080E290E00E948569872D7A941816BCF39F
:10D0900041FE04C0B4018DE290E00BC044FE04C028
:10D0A000B4018BE290E005C045FE05C0B40180E20A
:10D0B00090E00E94856946FE0FC0B40180E390E0D5
:10D0C0000E9485698989803139F4862D992787FDE9
:10D0D0009095B4010E94856950FE0DC0872D7A9409
:10D0E00018164CF4B40180E390E00E948569872D06
:10D0F0007A941816BCF343FE11C08A89982F915078
:10D100009A8B18165CF4B40180E390E00E94856964
:10D110008A89E82FE150EA8B1816ACF3842D8078C9
:10D1200069F4872D7A9418164CF4B40180E290E0EB
:10D130000E948569872D7A941816BCF3F3E66F1662
:10D1400041F48A2D992787FD9095B4010E94856945
:10D150002DC023E76216B1F489898150898B8F3FF6
:10D1600029F1F5018081992787FD90950894A11CEC
:10D17000B11CB4010E94856999899150998B9F3F98
:10D1800081F714C0CE0101962816390679F08E0178
:10D190000F5F1F4FF10182911F01992787FD909525
:10D1A000B4010E94856920163106A1F7842D80788C
:10D1B000A9F0872D7A9418168CF4B40180E290E0DF
:10D1C0000E948569872D7A941816BCF307C0862DB6
:10D1D000992787FD9095B4010E94856944245524C0
:10D1E00012C0F5E26F1641F44424552443941A8A80
:10D1F0007A882AE0298B07C0862D992787FD90958C
:10D20000B4010E948569F401838183FF08C0ED8524
:10D21000FE85CF0101968D879E87649005C0ED85C0
:10D22000FE856190ED87FE87662009F094CDF401BC
:10D230008681978162960FB6F894DEBF0FBECDBF90
:10D24000DF91CF911F910F91FF90EF90DF90CF90E2
:10D25000BF90AF909F908F907F906F905F904F9016
:10D260003F902F9008950F931F93CF93DF93CDB7E7
:10D27000DEB72C970FB6F894DEBF0FBECDBF8C0182
:10D2800036E03C8389839A832FEF3FE72D833E83EB
:10D29000CE0101960E947E66AF81B885A00FB11FB6
:10D2A0001C922C960FB6F894DEBF0FBECDBFDF9157
:10D2B000CF911F910F9108950F931F93CF93DF93F9
:10D2C000CDB7DEB72C970FB6F894DEBF0FBECDBF3B
:10D2D0008C013EE03C8389839A832FEF3FE72D83C7
:10D2E0003E83CE0101960E947E66AF81B885A00F75
:10D2F000B11F1C922C960FB6F894DEBF0FBECDBFA7
:10D30000DF91CF911F910F9108950F931F93CF93AA
:10D31000DF938C01EB018B81992781FF22C082FF73
:10D3200014C02E813F814C815D81241735073CF468
:10D33000A881B9810D93A883B9832E813F812F5F86
:10D340003F4F2E833F83C8010EC0E885F985802FAB
:10D350000995892B31F4EE81FF813196EE83FF83AD
:10D36000F2CF8FEF9FEFDF91CF911F910F91089533
:10D37000FC016150704001900110D8F780959095A4
:10D380008E0F9F1F0895629FD001739FF001829FAF
:10D39000E00DF11D649FE00DF11D929FF00D839F44
:10D3A000F00D749FF00D659FF00D9927729FB00DE1
:10D3B000E11DF91F639FB00DE11DF91FBD01CF01F4
:10D3C00011240895991B79E004C0991F961708F05D
:10D3D000961B881F7A95C9F78095089597FB092EAB
:10D3E00007260AD077FD04D00CD006D000201AF40E
:10D3F000709561957F4F0895F6F7909581959F4FB1
:10D400000895AA1BBB1B51E107C0AA1FBB1FA6178B
:10D41000B70710F0A61BB70B881F991F5A95A9F7DD
:10D4200080959095BC01CD01089585FD17C080625F
:10D430009923A1F4813694F08B3784F408959923CD
:10D4400069F4803269F0893059F08B3039F40895ED
:10D450008F93EDDF8F9109F08062089599278827D7
:10D4600008959923D9F78095807808959923B1F785
:10D470008033A4F38A3394F70895992379F780329F
:10D4800079F38A3069F38C3059F38D3049F3893060
:10D4900039F38B3019F70895A1E21A2EAA1BBB1B92
:10D4A000FD010DC0AA1FBB1FEE1FFF1FA217B30770
:10D4B000E407F50720F0A21BB30BE40BF50B661F86
:10D4C000771F881F991F1A9469F76095709580954A
:10D4D00090959B01AC01BD01CF01089597FB092EEA
:10D4E00005260ED057FD04D0D7DF0AD0001C38F433
:10D4F00050954095309521953F4F4F4F5F4F089580
:10D50000F6F790958095709561957F4F8F4F9F4F5F
:02D5100008957C
:10D512005A7A41003F004800484C004854004846AF
:10D52200002E0053544F50002100474F0048414CF9
:10D5320054004C004C430046004658005400590029
:10D5420056004D540053520053530053450040407F
:10D55200004200534F000001243C0401FD34060147
:10D56200FD340801E8340B01EF340E01F6341101E9
:10D572003C3513013C35180151351A0151351D0155
:10D5820066352201883524011237270143372901E4
:10D592008C382C01E2392E0111353001923A3201D8
:10D5A200B83A3501033B3801323B3B01983B3E011F
:10D5B200B6524101C53B4301F63B00000000800525
:10D5C200F42F8105F92F8403FE2F85032D30880463
:10D5D200573089047E308C03A9308D03C23090030A
:10D5E200E03094035C3195029B319802B731990186
:10D5F200DA319C02DF319D030232A0012932A201FD
:10D602008632A4039D32A501C132A601CA32A70106
:10D61200D032C401D632C6027B3DC703713DC80178
:10D62200D932C9011633CA015833CB01F133000094
:10D63200000000010000FF00020000FF00004A4954
:10D64200FF00030000FF00005D4AFF00004243FFAD
:10D6520000002540FF00006B40FF01001B42FF015C
:10D66200007D40FF01004441FF0100F142FF020042
:10D672004C46FF0200BB45FF0200D046FF02002FCE
:10D6820047FF02005F46FF02007246FF02007A4532
:10D69200FF03040000FF0300F94913030500001A09
:10D6A20003000849FF030600001A03004148FF0374
:10D6B200004648FF04009D4BFF0400F74BFF0500A6
:10D6C2004B48FF0500414BFF06003C48FF060000A7
:08D6D20049FF06000449FF00B6
:00000001FF
